:020000040000FA
:1000000000F80202B96A0000F5310000A93F0000C3
:1000100000000000000000000000000000000000E0
:1000200000000000003D0100483D0100F5310000E6
:100030000000000000000000F5310000ED7000003D
:1000400081310000F5310000F5310000D96A00006F
:10005000B9470000056800008531000079320000D2
:10006000F516000031160000F5310000F9310000EE
:100070008D470000417F0000596A0000856A00003A
:10008000F5310000F5310000F53100002D7300005E
:100090004D730000F5310000F5310000F53100002E
:1000A000D1730000DB730000833100006D69000034
:1000B000F53100006D680000000000000000000045
:1000C0000348854600F072FE0048004711BB00005F
:1000D00000F8020230B50B46014600202022012420
:1000E00009E00D46D5409D4205D31D469540491B6C
:1000F0002546954040191546521E002DF1DC30BDB5
:1001000070B500242546002801DA01244042002968
:1001100001DA01254942FFF7DDFFAC4200D0404241
:10012000002C00D0494270BD03460B439B0703D00F
:1001300009E008C9121F08C0042AFAD203E00B78AC
:100140000370401C491C521EF9D27047D2B201E024
:100150000270401C491EFBD270470022F6E710B522
:1001600013460A4604461946FFF7F0FF204610BD25
:10017000CAB2401E4178401C8A4202D00029F9D1FF
:1001800000207047421C0178401C0029FBD1801AD6
:10019000704730B504460020034600E05B1C9342E4
:1001A00003D2E05CCD5C401BF8D030BD30B50546D5
:1001B0000020034600E05B1C934205D2EC5CC85C67
:1001C000201A01D1002CF6D130BD00000FB400B5CB
:1001D0008DB009900B9010A900200091C0430A90A7
:1001E00000200C9006480690064807906A4609A829
:1001F0000F9900F043FC0DB008BC04B01847000094
:100200009D0A0000BD0A0000FFB5002083B00090E9
:1002100050680190916914460026976804988847B1
:1002200005460C990698084305D009E0A169761C9B
:10023000049888470546216A284688470028F5D152
:10024000681C03D00198C00704D017E00020C04309
:1002500007B0F0BD2068011D2160006800900DE02E
:100260000198C00704D1009805700098401C0090C8
:10027000A169761C7F1E049888470546002F1CDD67
:10028000681C1AD0069800280FD0E817C00E401935
:1002900041118A0006994009511840012A1A09683B
:1002A000012090400142DBD107E00C980028D7D113
:1002B000216A284688470028D2D0E16904988847F7
:1002C0000C98002807D1002E05DD0198C00702D147
:1002D000009800210170A068B84204DD0C98002845
:1002E00004D0002F02D00120C043B1E73046AFE771
:1002F00070B5064610F0C2F8046805460A220021CF
:10030000304600F047FC2C6070BDF8B502464A400C
:10031000D40F42004B0052085B089A4202D20246B8
:10032000084611464A0023D0C30D4A00DDB2120E22
:10033000AD1A202D35DA49020126490AF6058A1937
:10034000002C00D0524220214F1B1146B9402A41B7
:100350001018C20D9A4221D0002C17D0012D08DCB4
:10036000DA05801AD20F8019D207DBB200F052FCF6
:10037000F8BDDA05801A012340001B06C01880185A
:100380005A428018CA0F1043490007E04908C207C3
:100390001143DA05801A80194008801800F032FCF9
:1003A000F8BD61000122511A001BF7E70122D207B4
:1003B0005140AAE70122D2075040A6E7024670B595
:1003C0004A40D30FDB0740002DD04A002AD0010E4F
:1003D000140E000212020919400A520A8418E5019B
:1003E00004465443000A120A2E045043A419421929
:1003F000200CC543AA18120C0125AD03521C52193A
:1004000012047F39240400D0521C104301D4400050
:10041000491EC2B20C06C0092018401C4008802AA0
:1004200002D003E0002070BD40084000002900DA3F
:100430000020184370BD70B502464A40D50F4000F9
:100440004A00ED0740085208002814D0002A12D0B4
:10045000C40DD30D41020120C0055202490A520ABF
:10046000E41A091812187D34914201D3641C00E08B
:100470004900002C01DA002070BD0023914201D315
:10048000891A0343400849000028F7D100290AD0FF
:10049000914202D10121C90705E0914201D2012117
:1004A00001E00121C943E005C018401900F0AAFB92
:1004B00070BD0000F0B507460846584087B0C00F31
:1004C000049048000E46590040084908BC1A88416B
:1004D00005D2384631461E4617460B46024658009E
:1004E000400810434CD0300D039040055900400D9A
:1004F000490D0590401A0290402872DA1803012134
:10050000000B09050843019004980092002805D0CB
:1005100001995242002088410092019002984021A6
:100520000A1A0199009800F06FFA05460C466B46CE
:1005300007CB00F08AFAC0197141039A0E0D00230F
:10054000D71756401A467A40164344D0049A002AD8
:100550002DD0029A012A039A15DC1205C01A914186
:1005600001263605001C7141D20F059ED20700936B
:10057000019202962A46234600F092FB07B0F0BD96
:1005800038463146FAE71605224A0F46B218C01A15
:10059000B74101210905001C4F4100187F41114658
:1005A00018187941E20F10436D19644113E0E20716
:1005B0006D0815436408C2071443039A0126120507
:1005C000C01A91413605001C7141CE0740083043E6
:1005D0004908C01851412A46234600F054FBCDE794
:1005E000FFE7049801224000C117121A00238B4133
:1005F00004983146C417381AA141EEE730B40124FB
:10060000E407634030BC55E730B40124E40761409F
:1006100030BC4FE70000E0FFF0B51FB488B00B9985
:100620000998002448400999C00F490049080991D8
:10063000C0070B990090490049080B910999089847
:10064000A64608431CD00B990A98084318D009986D
:1006500001244000420D4800410D09982405000383
:10066000000B204309900B980003000B20430B90D4
:1006700050181C494018002201901446104605E00D
:10068000002001460DB0F0BD032801DA034600E06A
:1006900003239C46C11A0AAE0AE05F0008ADED5B79
:1006A0004F00F75B7D430027AA187C41491C5B1E65
:1006B0006145F2DD410004AB5A522104120C0A4399
:1006C000240C401C0828DFDB01980290009970463A
:1006D00001910090059B049A0799069800F0E0FAB2
:1006E000D0E700000DFCFFFFF0B50C465C4085B084
:1006F000E40FE40703944C00002664085900944674
:10070000490802460296224321D062460A431ED07F
:100710006200570D4A000E032303550D01240246C3
:100720002C492405781B1B0B360B4018234326430A
:10073000614600901C46501AB44103D30098401CF7
:10074000009002E0921800985B41002803DA002034
:10075000014605B0F0BD0020012109050746864687
:1007600011E064461D46141BB54106D36546521B75
:10077000B341744607430C43A646CD0740084908D9
:10078000284392185B4105460D43EAD110461843B1
:1007900013D06046194650407140084306D0604669
:1007A000101AB34106D20122002306E000220123E1
:1007B000DB0702E00122D243531000987446010582
:1007C000381C6141029C039D0019694100F05BFAED
:1007D000BFE70000FD0300000122D207002800DB74
:1007E000101A002900DB511A814201D801207047FC
:1007F000002070470122D207002800DB101A0029D0
:1008000000DB511A814201D201207047002070475D
:100810000122D207002800DB101A002900DB511A40
:10082000814201D301207047002070470122D20786
:10083000002800DB101A002900DB511A814201D97F
:1008400001207047002070470122D207002800DBFA
:10085000101A002900DB511A814201D10120704792
:1008600000207047C217C10F504010B54018CA078A
:100870009623002100F0CEF910BD10B5002296237A
:10088000114600F0C7F910BD0EB5054902910021CF
:1008900000910A460B46019100F002FA03B000BD38
:1008A00033040000C20F410040020123400ADB056F
:1008B000D207090EC0187F2901DA00207047962957
:1008C00003DC9623591AC84001E096398840002A73
:1008D000F4D040427047410040020122400AD20554
:1008E000090E80187F2901DA00207047962903DC61
:1008F0009622511AC84070479639884070470000C8
:1009000070B5CD0F4A0009030123090B1B051943DC
:100910000B4BED070024520D9A4201DA002070BD06
:10092000074B34339A4203DC9A1A00F07DF802E058
:100930000449511888402C43F1D0404270BD00005A
:10094000FF030000CDFBFFFFC20FD20740004008AD
:100950000BD0C10D0723DB01C91840020905400A6D
:100960001143C208400711437047002001467047F9
:10097000CB0FDB07490010B5490802460A4307D0F0
:100980000A0D07240903E401090B121B002A01DCEC
:10099000002010BDC900440F0C43C100E018D2056F
:1009A000801800F02FF910BDF0B51FB406460020E6
:1009B00082B005464024019100901BE00199224637
:1009C0000F46304600F030F8049A059B801A994192
:1009D00010D310461946224600F016F8361A8F41F9
:1009E0000197224601200021009F00F00DF83818E1
:1009F0004D4100902046641E0028DFDC019B0098DA
:100A00002946324607B0F0BD10B5202A04DB014666
:100A1000203A9140002010BD914020239C1A0346AB
:100A2000E3401943904010BD10B5202A04DB08466E
:100A3000203AD040002110BD0B46D340D0402024A6
:100A4000A21A91400843194610BD10B5202A06DBB2
:100A5000CB170846203A1041C1170B4306E00B465E
:100A60001341D0402024A21A91400843194610BDDA
:100A700002681378511801601846704710B5D160AC
:100A8000044951610449116200211161114600F0CD
:100A9000ADF910BD710A0000D90D00004268002AAE
:100AA00008D001680B78491C002B03D0521E06C0E9
:100AB000184670470121C160881E70474268002AAD
:100AC0000BD0C3680168002B07D183688B4204D028
:100AD000491E521C06C0002070470020C0437047CA
:100AE0000FB400B589B00A460DA9009100230C99F6
:100AF000002ACB60234B0693234B079301D004239A
:100B000000E00023214A0292214A08920193024602
:100B10006B46002000F095FB09B008BC04B01847F4
:100B2000F0B585B007460020C04301901E46002066
:100B300015460C460091029104903B466A463146A8
:100B400004A8FFF7CDFF049902466018002D05D0D8
:100B5000002901D0034600E023462B6000290ED077
:100B6000002A02DD0099814209D0001B0190009407
:100B70003B466A463146029404A8FFF7B1FF05B030
:100B8000F0BD00009D0A0000BD0A0000FFFFFF7FCE
:100B9000D90D0000F7B5009C0F4600262578641C8F
:100BA000002D05D000F014F90068405DC007F5D1B4
:100BB0002B2D02D02D2D18D0641E39462046029AC6
:100BC00000F06AFC002F04D03968A14201D10099DD
:100BD00039607105022400290BDA4042002803DD48
:100BE0000FF04CFC0460A007FEBD0120800206430C
:100BF000E3E70028F8DA0FF041FC04600048FEBD8E
:100C0000FFFFFF7F002904DA401C490001D14008A2
:100C10004000704770B40024050C05D11024000476
:100C200002D1002921D01124050E01D1000208347F
:100C3000050F01D10001241D850F01D18000A41CE6
:100C4000002801DB4000641C002908D020252E1B51
:100C50000D46F540A14000D001212943084301067B
:100C60001B1B000ADB1D02D5002070BC7047DB0592
:100C7000181880180029F8DA401C4900F5D170BC1A
:100C800040084000704710B5002B08DA0024401CD3
:100C9000614192185B411A4301D14008400010BDE8
:100CA000F0B51FB482B005460C0003D008460FF023
:100CB000CDFB02E00FF0CAFB203002460090214637
:100CC0002846FFF7A1FE049B059A04460F461843E9
:100CD0001143084314D0184610431BD000984021FC
:100CE0000A1A18460599FFF79FFE05460E46009A18
:100CF00005990498FFF788FE084305D0012004E019
:100D00002046394607B0F0BD0020C11705430E4309
:100D10002C43374300990E986305401A7905E40A7D
:100D200000220C43FD0A0A3002D500200146E9E703
:100D30000105101969410C9C0D9D00196941FFF7CF
:100D4000A2FFDFE74A0009030123090B1B05194332
:100D50000A4B10B5520D9A4202DA0020014610BD2E
:100D6000064B34339A4203DC9A1AFFF75DFE10BD3E
:100D7000034BD218FFF748FE10BD0000FF03000030
:100D8000CDFBFFFF10B5002904DB0124E40740423E
:100D90008C412146002B04DB1C460123DB07524219
:100DA000A341994200D1904210BD0000064C01259C
:100DB000064E05E0E36807CC2B430C3C9847103403
:100DC000B442F7D3FFF780F96C3701008C3701008C
:100DD00000487047180E010010B50446FFF7F8FFF1
:100DE0000068005DC007C00F10BD0000F3B58DB0F6
:100DF00000200A9001200B90002608460C300C467B
:100E000009906269012109989047051E2ED0252D71
:100E10002DD0216A8847002818D0626901210998DD
:100E20009047216A88470028F7D1411E62690998D6
:100E3000904700E0761CA1690D988847216A884791
:100E40000028F7D1E1690D988847DAE7A1690D9884
:100E500088470746A84201D1761CD2E7E1690D9880
:100E600088477F1C02D10A98002877D049E10027E3
:100E700062693D463946099890472A280CD1626933
:100E8000012109989047012506E00A214F433F18A8
:100E9000303FEBD410200543626901210998904747
:100EA000014630390A2903D29B498F42DEDCECE748
:100EB000E90600D4994F6C280AD04C2810D0682835
:100EC00024D06A282ED074280CD07A280AD00DE0BD
:100ED00062690121099890476C2823D004211CE005
:100EE000202005436269012109989047A760656049
:100EF00065284FD026DC582839D01ADC452849D03F
:100F000012DC252834D04128B0D143E062690121A8
:100F100009989047682802D008210D43E6E7012090
:100F2000C002DEE70220DCE7462833D047282CD178
:100F300030E05B2870D061282CD063286CD0642806
:100F400023D161E06F284FD009DC662822D06728C2
:100F500020D0692826D06E2817D12EE0CDE0702849
:100F60004DD073286FD075284ED078280DD154E01D
:100F7000A1690D9888470546252800D16CE7E169ED
:100F80000D9888476D1C00D16DE7BAE00A224CE04D
:100F90000A2252E0012023466A46C0430D9900F020
:100FA00050F9A3E02846402108436060A807234683
:100FB00001D5002239E000223FE0E80700D020E719
:100FC0002068011D21600068290501D5067018E719
:100FD000290701D5068014E7A90703D5F117066094
:100FE00041600EE706600CE7284640210843606038
:100FF000A807234601D5082217E008221DE048492A
:1010000028460840606016E028464021084360609A
:10101000A8072346BCD5B9E715E028464021084378
:101020006060A80707D5234610220120C0430D9910
:10103000C046C0465AE0234610220120C0430D9905
:10104000C046C04652E000210C910B460091632837
:1010500002D05B2807D043E0E80601D40120A0605D
:10106000012000903CE062690121099890475E28C8
:1010700005D101200C9001466269099890472169C9
:10108000002906D10B4601AA8F00491CD35108291B
:10109000FADB002835D0216900290ED1C117C90E0D
:1010A00009184A11930001AA9A1849094901411ADD
:1010B0000120136888400343136062690121099885
:1010C00090475D28E5D10C98002808D0002001AB9E
:1010D00081005A58401CD2435A500828F8DB01AB13
:1010E00001202246C0430D99FFF78EF800280ADA46
:1010F000401C06D10B98002803D00020C0430FB03D
:10110000F0BD0A98FBE7E90702D10A99491C0A9148
:10111000361800200B9074E6CCCCCC0CFFFFFF7F80
:10112000F1F7FFFFFFB5087889B01546FF2805D015
:10113000491C2D2804D00022002407E000240BE0E5
:101140000122F9E70A235C430419491C0878FF28A7
:10115000F8D1002A00D06442002004902A78014689
:101160002D2A01D02B2A0FD16D1C2D2A02D000224E
:10117000049209E00122FBE700260A2233466D1C97
:1011800000F0DDF9381871412F78FF2FF4D10C9A57
:10119000A218069202460A4304D0FF23069A91330E
:1011A000DA4205DA002109980A4606C00DB0F0BD02
:1011B0000024B74AB54D2646079200F00DFA02907A
:1011C00006980391002801DA474200E007463905F6
:1011D0000020AF4A001C51410191009012E0F80735
:1011E00007D022462B4630460799FFF715FA0646E8
:1011F000079122462B4610461946FFF70DFA044682
:101200000D467F10002FEAD10698019B0028009A16
:101210000399029806DAFFF767FA3246079BFFF751
:1012200063FA05E0FFF7F8F93246079BFFF7F4F998
:10123000049A002A02D00122D2075140099A03C21F
:10124000B4E7FFB591B0002009900025ED432E20B2
:101250009E685C681F460190B9696D1C12988847AA
:101260000090396A88470028F6D10098401C0AD0BF
:101270000D20C0018443002E12DD00982B2809D0D8
:101280002D280DD103E00020C04315B0F0BD012092
:1012900080020443B9696D1C12988847761E00903D
:1012A00003A9600501D52D2000E02B206A461073AC
:1012B000491C0CA80F9102900AE0B9696D1C1298A4
:1012C000884700900120400204431398761E056071
:1012D000002E02DD00983028EFD001990098884256
:1012E00045D18020044308E00998401E0990012060
:1012F000400204431399681C0860B9696D1C761E8E
:101300001298884700903028EED030E0019988424A
:1013100005D1200603D480200443761E1DE00098EA
:101320000FF07AF9002825D0012149020C430098DA
:1013300007AA0F9903323038761E914208D20870FE
:101340000F98401C0F90200607D50998401E03E017
:10135000200602D40998401C0990A00502D51399D3
:10136000681C0860B9696D1C129888470090002EAF
:10137000CCDC59E0002E57DD0098652801D04528C7
:1013800052D1A00550D5032000028443B9696D1CD9
:10139000761E129888470090002E0CDD2B2804D072
:1013A0002D2808D1FF2001300443B9696D1C129823
:1013B0008847761E0090E00501D52D2100E02B2105
:1013C000029801700298401C0290019025E00120D3
:1013D000400204430EA902980131761E88420ED2C3
:1013E0000098029930380006000E087003D1029967
:1013F000019881420AD90298401C029006E0E0055B
:1014000001D5244801E0234840420990B9696D1C88
:1014100012988847009013980560002E04DD00980C
:101420000FF0FAF80028D2D1F969129888470F997D
:10143000FF200870029903AA087000200A900B9000
:101440000CA90AA8099BFFF76DFEA00502D4012094
:10145000C0431AE72420044209D0E00713D13868BA
:101460000B9A0A99031D3B60006806C00BE00B99BC
:101470000A98FFF77DFA0146E00704D13868021D9B
:101480003A60006801602846FFE600000000144052
:101490000000F03FF1D8FFFFF7B582B0029C0027B3
:1014A0002078641C15460197302802D0002D15D0F5
:1014B00015E020780127641C782804D0582802D031
:1014C000002D09D00BE0002D01D0102D07D10027F1
:1014D00010252078641C02E0082500E00A2500267B
:1014E000009610E00099012769430818020C29466C
:1014F00080B2714300908E183804864201D30120D7
:1015000001902078641C294600F056F80028E9DA9A
:101510000398002805D0002F01D0641E00E0029C33
:1015200004600198002806D00EF0A8FF0221016097
:10153000C81E05B0F0BD009930040843F9E7F0B5C6
:101540001FB486B000200090019002900698069982
:1015500080B204900798090C02040014114307900C
:101560000027089D099806913E463C460390039843
:10157000A9B20204000C039004982D0C15434843B3
:1015800000212246FFF740FAC719714110340E4678
:10159000402CECDB3846029AFFF736FA009A019BA2
:1015A0008018009059410298019110300290402813
:1015B000CCDB00980BB0F0BD3A2800D230382023A5
:1015C00002469A43412A01D310463738884201D354
:1015D0000020C043704700000EB5054A0292002269
:1015E000009213460192FFF75BFB03B000BD0000C1
:1015F0003304000030B58C180278401C13071B0F11
:1016000001D10378401C120906D10278401C03E086
:1016100005780D70401C491C5B1EF9D101E00B7070
:10162000491C521EFBD1A142E6D3002030BD000070
:1016300010B52148016A8A0715D44A0715D4C9078D
:1016400032D01E498A89002A15D0531E8B818268A8
:101650008C6904C48C610A691B040DD0002A22D154
:101660000121016010BD022100E00421C161134885
:101670008021416110BD0A69012A09D10268012354
:101680009A430260C361FF20683099300C4A1060B1
:1016900001204861CA69002A05D0886909898B0040
:1016A000C01A904710BD10BDFF226832054806A140
:1016B00009A30CF091FBC04608D0014078950102C7
:1016C00080E200E0681D01004144435F49525148F7
:1016D000616E646C65720000556E65787065637448
:1016E00065642041444320696E746572727570743C
:1016F0000D0A000070B582B00023019344480168D0
:101700008A6A4C6813252540132D02D1CB689B07AC
:10171000DB0F4361930772D453070AD4D30711D167
:10172000130724D5048F838E1C1B102C0EDD102371
:1017300010E0042088620220032142A20DF0A8FBE1
:1017400002B070BD0120886202B070BD048F1B1B07
:101750001C0610D0DBB20024058FC66A75192D5DFA
:101760000D74641CA342F7D1048FE3180387D206DB
:1017700007D400212FE04B6A0824A3434B62D20612
:10178000F7D5CB68C28E448F141B5B04DB0EA342DB
:1017900001D3438FD31ADAB2002A16D0097D438FC2
:1017A000046BE1540199012A10D001231C468901E0
:1017B00045582D7D41184E8F9B19096BCD54641CE3
:1017C000E3B201999A42F2D800E000218B01C318DC
:1017D0005C8FA2185A878A0181184B8FCC8EA34246
:1017E0000BD301230B61805800224262CA6B002A8E
:1017F00003D03A31098801A8904702B070BD022099
:101800008862044804A1084A08A30CF0E5FAC0461F
:1018100078900102811D01004145535F49525148B2
:10182000616E646C65720000CE0200004145532079
:10183000696E707574206F766572666C6F770D0ACD
:1018400000000000414553206F7574707574207559
:101850006E646572666C6F770D0A0000F0B581B03A
:1018600001243F2900D993E003468068456B2D6829
:101870008E0001A7BE59B746B7190000D319000062
:10188000AF190000AF190000911900009119000074
:1018900091190000911900009119000091190000A0
:1018A0009119000091190000911900009119000090
:1018B000E5190000011A00009119000091190000BB
:1018C0009119000091190000911900009119000070
:1018D0009119000091190000911900009119000060
:1018E0009119000091190000911900009119000050
:1018F0009119000091190000911900009119000040
:10190000911900009119000091190000911900002F
:10191000911900009119000091190000911900001F
:10192000911900009119000091190000911900000F
:1019300091190000911900009119000091190000FF
:1019400091190000911900009119000091190000EF
:10195000791900007919000079190000791900003F
:10196000791900007919000079190000791900002F
:101970007919000079190000434800690024022801
:1019800009D001280DD0002802D103CA04F0FAFEC4
:10199000204601B0F0BD03CA04F0E6FE204601B0C7
:1019A000F0BD03CA04F004FF204601B0F0BD0229D7
:1019B00031D0022430E0344D00242C616C61984910
:1019C000354A01F0E9FD6869401C6861204601B0B4
:1019D000F0BD01F01BFE284602F088F800242046E6
:1019E00001B0F0BD284909690C234B432749CA5867
:1019F000C918496801F0D0FD0024204601B0F0BDAF
:101A00000024204604F08CFE0128C1D11E4830304D
:101A1000204900241CE001241B490F690C26314693
:101A200079431A4A51188968214208D000247D1C44
:101A300015490D614C61042D10D3154906E012497A
:101A40004869401C4861032812D3294900241846DC
:101A5000224601F0FBFF204601B0F0BD6E430B496A
:101A60008A598919496801F097FD204601B0F0BDF7
:101A70000E20009000240A222846214601F0D6FFBD
:101A8000204601B0F0BDC046D49801021C0E0100F2
:101A900018150100F814010064280100B0B50429EC
:101AA0000FD804468068C0467944097949008F44BC
:101AB000020A0E1C1700104910A201F06DFD002053
:101AC000B0BD0120B0BD01F0A1FD0020B0BD0025DA
:101AD0000321284604F034FE064920462A4602E047
:101AE00003490022204601F0B1FF0020B0BDC046EE
:101AF0000815010088150100881300004154453085
:101B00000D0A0000B0B582B001240A2910D88368FC
:101B10007944097949008F440E2905050B0B0B0BFD
:101B20000B0B1A00194909680024224601F08EFFA8
:101B3000204602B0B0BD506814490860144915A28F
:101B4000184601F029FD0024204602B0B0BD002453
:101B5000019403CA09A201AB02F096F80228E7D16A
:101B6000019804F041FE204602B0B0BD184601F0D5
:101B70004DFD0024204602B0B0BDC0462B4353515A
:101B80003A2025642C252A0D0A0000003499010210
:101B90008813000041542B4353510D0A00000000EC
:101BA000B0B582B00546002404F018FE01280DD11E
:101BB00008498C60E86B426853684B60009401925E
:101BC0006A4601F043FF204602B0B0BDE443204620
:101BD00002B0B0BDBC930102B0B50546881E022814
:101BE0000AD3A868012913D0002915D10C490DA2E8
:101BF00001F0D2FC0020B0BD0220014604F0A0FD9F
:101C0000064900242846224601F020FF2046B0BDA8
:101C100001F0FCFC0020B0BD0120B0BDD8140100D3
:101C20008813000041542B4346554E3D300D0A00A9
:101C3000B0B5E0B00324E1016D4628460EF0EEFB9E
:101C4000204621462A460DF023F9002060B0B0BDA1
:101C5000F0B597B008201490642013902548109098
:101C600002200E904B20C0011690234D28461430C0
:101C7000129001270F97B802119003200EA905F0CA
:101C80004BFC0026F443002802D0204617B0F0BDDC
:101C90000C35284601F038FF0028F6D180200C9042
:101CA00016490B910A901648099016480890164854
:101CB000079016480690392005901548049015485D
:101CC00003900D95144D03A9284601F0CFFC002880
:101CD000DBD1009501970F4C104911A2124B204601
:101CE00001F068FE1149204601F098FE3446204676
:101CF00017B0F0BDF0BD010290960102F0C10102E3
:101D000070C20102E52D0000352E0000B52D000047
:101D1000981601000499010200C70102781401001D
:101D2000414952373830450098150100311C0000F8
:101D300010B50748002404700EF00AF8204610BDC4
:101D400080B50348012101700EF002F8002080BD2B
:101D50004C9D0102F0B58DB00E4600270C970B97F5
:101D60000A97099708970797069705970290806842
:101D70000490406B0068019004F0CCFC04465BA129
:101D800005220392FEF712FA5A4D00281ED05AA1DE
:101D900005222046FEF70AFA002817D058A105228E
:101DA0002046FEF703FA00280FD059A1052220464D
:101DB000FEF7FCF9002809D057A105222046FEF7BE
:101DC000F5F9002807D156A500E04FA505A8202168
:101DD0002A4602F02BF801203F2E00D936E0C046FB
:101DE0007E4436797600B7443340474A5731313123
:101DF00031313131313165303131313131313131A0
:101E000031313131313131313131313131313131C2
:101E100031313131313131313131313131311F1FD6
:101E20001F1F1F1F1F1F1F1FBE48416A04290CD1FF
:101E3000039A426287620C2050433D490A580818B1
:101E4000416805AB049801F0A7FB38460DB0F0BD22
:101E5000B44C00206062A062CD49364A049801F07B
:101E60009BFBA06A401CA062EFE7049801F0CEFB48
:101E7000019801F03BFEE8E7AA48406A05E0A9495D
:101E8000486A01220243032A1CD1A649421C4A6225
:101E90008F62062ACFD30BE0A2494A6A012013467B
:101EA0000343052BD2D1501C48628F62062803D30E
:101EB0001E490DE09B48406A0C2141431C48425892
:101EC0004018BDE7886A401C8862032805D316497C
:101ED0000022029801F0BAFDB7E70E200090002121
:101EE0000A220198029B01F0A1FDAEE734363030A2
:101EF000300000008C280100343630303200000001
:101F00003436303031000000554E494E4554000003
:101F100034363030360000003436303033000000C4
:101F200043544E455400000078140100C8140100C9
:101F30004C0E01000C28010070B5022956D30F2960
:101F400007D1784C217A012905D1002222728F49CC
:101F50004AE0012070BD866801F0FCFD002004F01D
:101F6000E7FB012803D10020032104F0E9FB002551
:101F7000284604F0D5FB012804D130346A490022F8
:101F8000204631E0304600F0EBFD00282ED03046F0
:101F9000FFF706FE002829D004F0DCFB012807D15A
:101FA0005F498D60F06B4268E26252684A601AE0F5
:101FB000022004F0B5FB012808D159498D61F06B6E
:101FC0004268E26252684A6110310CE0022004F07B
:101FD000AFFB01280AD152498D62F06B4268E26280
:101FE00052684A6220312A4601F030FD002070BD5F
:101FF00010B582B003460120272931D879440979E8
:1020000049008F442C132D2D162D2D2D2D2D2D2DCA
:102010002D2D2D2C2D2D2D2D2D2D2D2D2D2D1C2D02
:102020002D2D2D2D2D2D2D2D2D2D2D2904F0BEFDE9
:1020300015E0DF490022184601F008FD0FE00020FE
:10204000019003CA08A201AB01F01EFE012806D1CF
:10205000019804F0C7FE02E002480121017200204D
:1020600002B010BDD49801022B51495552433A2079
:1020700022636C6F736564222C25640D0A000000D6
:10208000B0B502294AD30F2914D18568002004F085
:102090004FFB012803D10020032104F051FB002451
:1020A000204604F03DFB012806D1D94830301E49B6
:1020B000002231E00120B0BD2846FFF771FD002865
:1020C0002CD004F047FB012808D115498C60E86B3F
:1020D0004268CF4BDA6252684A601CE0022004F08A
:1020E0001FFB012809D10E498C61E86B4268C84B7F
:1020F000DA6252684A6110310DE0022004F018FBE8
:1021000001280BD106498C62E86B4268C04BDA6249
:1021100052684A622031224601F098FC0020B0BD8E
:1021200044900102D4980102F814010080B50229FC
:1021300005D3042905D19E49002201F087FC002027
:1021400080BD012080BDC046B0B50546881E02286E
:102150000AD3A868012913D0002915D10C490DA272
:1021600001F01AFA0020B0BD0220032104F0E8FAC1
:10217000064900242846224601F068FC2046B0BDEE
:1021800001F044FA0020B0BD0120B0BD18150100D7
:102190008813000041542B4346554E3D310D0A0033
:1021A00010B50F290BD001291DD000291DD1FFF733
:1021B000BFFD0020022104F0C3FA002010BD044638
:1021C000002004F0ADFA012803D10020022104F020
:1021D000B7FA002004F0ACFA012804D10449002227
:1021E000204601F033FC002010BD012010BDC04688
:1021F00008150100F0B581B00124322928D8054620
:102200008768786B0668C0467944097949008F442D
:102210002F3F1919191F1F1F1F1F1F1F1F1F221FAD
:102220001F1F1F1F1F1F1F1F1F1F1F1F1F1F1F1FBE
:102230001F1F1F1F1F1F1F1F1F1F1F1F1F1F1F1FAE
:102240001F1F26001E4900242846224601F0FEFBDF
:10225000204601B0F0BD1B48017800291FD0184965
:1022600000242846224601F0F1FB204601B0F0BDD3
:102270000024FC623969384688470028FAD01148A2
:102280000470FC62FFF754FD0E20009001220EE066
:10229000304601F02BFC0024204601B0F0BD0121A6
:1022A0000170FFF74DFD0E200090002405223046FE
:1022B00021462B4601F0BAFB204601B0F0BDC046D6
:1022C000981401003899010210B586B00346012028
:1022D0003B2900D956E0C0467944097949008F442A
:1022E00050505151335151515151515151515151FE
:1022F00051515151515151515151515151515151CE
:1023000051515151515151515151515151515151BD
:102310005151515151391D1D1D1D1D1D002005908C
:1023200003CA02AA009218A205AB01F0ADFC022874
:1023300027D1039A029817A1FDF738FF002820D172
:10234000059804F04FFD1CE0B5490022184601F045
:102350007DFB16E0002002900590049003CA05AAB8
:10236000019204AA00920DA202AB01F08DFC032899
:1023700007D1049A0599029804F000FE029804F02F
:102380009FFD002006B010BD25642C2025700D0A8D
:1023900000000000434C4F53454400002B5245437E
:1023A000454956452C25642C25643A0D0A256500BF
:1023B000E8140100012901D800207047012070476E
:1023C000B0B50546881E03280BD2104604F0CAF9A2
:1023D0000F48C16A00242846224601F037FB2046F8
:1023E000B0BDAC6801290BD000290ED104F094F9DE
:1023F0000346084908A2204601F0CEF80020B0BDEF
:10240000204601F003F90020B0BD0120B0BDC04658
:10241000D49801028813000025730D0A0000000003
:1024200070B582B001240F293DD803468568686BDA
:102430000668C0467944097949008F4407141E3460
:102440003434342F373434343434434E6648002423
:1024500004708461C461012101716649664A28469D
:1024600001F09AF81FE0284601F0D0F8304601F05C
:102470003DFB0024204602B070BD5B48002404717F
:102480008269042111430278002A2ED0052958D1EF
:10249000016A491C016259D2624961E0524B1878C5
:1024A0000024002831D0204602B070BD4E4B187871
:1024B000012816D103CA183351A201F0E5FB002010
:1024C00002B070BD48480024846101210171007888
:1024D0004849002812D1484A11E0434E307900287B
:1024E0001BD00024204602B070BD052932D1002443
:1024F000012101708461C46101713E493F4A28464F
:1025000001F04AF8204602B070BD03CA183340A259
:1025100001F0BAFB204602B070BD002004F008F9BB
:10252000012803D10020032104F00AF900242046E9
:1025300004F0F6F8012816D130362D490024304633
:102540004BE000210162C169491CC1610E2000906D
:1025500000241CE0C169491CC161652915D33049BB
:102560000024184639E02846FFF71AFB00289AD0C5
:1025700004F0F0F8012812D11C4900248C60E86BAB
:102580004268F26252684A6027E00E200090022200
:102590003046214601F04AFA204602B070BD0220C2
:1025A00004F0BEF8012809D1104900248C61E86BC1
:1025B0004268F26252684A6110310EE0022004F073
:1025C000B7F8012800D06EE7084900248C62E86B58
:1025D0004268F26252684A622031224601F036FABD
:1025E000204602B070BDC046D4980102449001025A
:1025F000F814010088130000282801003328010086
:102600002B43475245473A20252A2C2564000000D9
:102610002B435245473A20252A2C25640000000010
:10262000E8140100A8140100B0B584B001243B29CE
:1026300000D937E0134605468068C04679440979D9
:1026400049008F444B5532322F2F2F2F2F2F2F2FF2
:102650002F2F2F2F2F2F2F2F2F2F2F2F2F2F2F2F8A
:102660002F2F2F2F2F2F2F2F2F2F2F2F2F2F2F2F7A
:102670002F2F2F2F2F2F2F2F2F2F1D1D1D1D1D1DD6
:102680000024039403CB01AA00921C4A03AB01F07F
:10269000FBFA022806D1029A019819A1FDF786FDDE
:1026A00000280FD0204604B0B0BD1848006804F0E0
:1026B00099FB174900242846224601F0C7F9204615
:1026C00004B0B0BD1148006804F08CFB1049002232
:1026D000284601F0BBF9204604B0B0BD0B490B60A1
:1026E0001E210CA200F058FF0024204604B0B0BD0B
:1026F00000F08CFF0024204604B0B0BD8C290100FE
:10270000434C4F5345204F4B000000003C990102C1
:10271000B814010041542B434950434C4F53453D9D
:1027200025640D0A00000000F0B589B004460120C0
:102730003B2900D9AAE01646A7687A6B1568C046FF
:102740007944097949008F44536AA071A1A1A1A1DC
:10275000A1A1A1A1A1A18AA1A1A1A1A1A1A1A1A180
:10276000A1A1A1A1A1A1A1A1A1A1A1A1A1A1A1A159
:10277000A1A1A1A1A1A1A1A1A1A1A1A1A1A11D1D51
:102780001D1D1D1D0027089703CE06AA0092414A71
:1027900008AB01F079FA022877D13F48056808981C
:1027A000854272D1079A069E3CA130460592FDF7FC
:1027B000FDFC002847D03DA13046059AFDF7F6FC08
:1027C000002840D03CA13046059AFDF7EFFC0028D8
:1027D000314E5AD1284604F01FFB7068401C7060CF
:1027E00003283CD303207060306804F09DFA36E083
:1027F00029480660304604F0EBFA05902648006848
:1028000004F0BAFA04902448006804F0C1FA04996C
:10281000019102900598012827D02EA026E0384685
:1028200000F0F4FE284601F061F92EE01A4D286808
:1028300004F0F2FA6868401C686003280FD3002295
:102840006A6022490DE0144E7760284604F0FAFAD7
:10285000306804F039FC002801D01B4900E00C4925
:102860000022204601F0F2F80FE019A000901A496A
:102870001AA23846334600F08FFE0E200090002149
:10288000B4222846234601F0D1F8002009B0F0BD5B
:10289000B81401008C29010008970102414C5245EF
:1028A00041445920434F4E4E45435400434F4E4EF2
:1028B000454354204F4B0000434F4E4E4543542058
:1028C0004641494C000000005815010078140100F1
:1028D00054435000554450008813000041542B438A
:1028E000495053544152543D25642C222573222CC7
:1028F000222573222C25750D0A000000B0B582B088
:1029000014468A1E022A12D38568012917D000298D
:102910001CD1204604F022FA00901E210EA2284667
:10292000234600F039FE0024204602B0B0BD09491C
:102930000024224601F08AF8204602B0B0BD2846A5
:1029400000F064FE0024204602B0B0BD0124204601
:1029500002B0B0BD6815010041545E484541525473
:10296000434F4E4649473D312C25642C25750D0AB1
:1029700000000000F0B583B014468A1E022A1CD362
:102980008568012921D0002926D1164F3C602046B8
:1029900004F0D6F9FDF7F6FB0646386804F0D0F9E6
:1029A0007108009101901E210FA22846234600F0D5
:1029B000F3FD0024204603B0F0BD0949002422465F
:1029C00001F044F8204603B0F0BD284600F01EFE9A
:1029D0000024204603B0F0BD0124204603B0F0BD22
:1029E000B81401004099010241545E4845415254D7
:1029F000424541544845583D25642C25752C257386
:102A00000D0A0000F0B585B0044601203B2900D92D
:102A100085E0A5687944097949008F443F547F5B7C
:102A200080808080808080808080808060808080C6
:102A30008080808080808080808080808080808096
:102A40008080808080808080808080808080808086
:102A500080801D1D1D1D1D1D0020049003CA02AA9B
:102A60000092304A04AB01F00FF9022856D12E48EB
:102A700085680498854251D1039E029F2BA1384658
:102A80003246FDF793FB00283AD02AA13846324659
:102A9000FDF78CFB002841D128461DE0224CA260A6
:102AA000104604F081F9002838D001F01CFAE060EB
:102AB000002833D0A36840680090234923A2284609
:102AC00000F06AFD2AE018480021C160284600F0A5
:102AD0009DFD23E01448806804F084F919E000F0BB
:102AE00005FE012804D11048C16803C900F006FFA3
:102AF0000D48C0680CC81349284600F08DFD0DE054
:102B0000284604F051F90028074907D0C96801F0A8
:102B1000C0F90B490022204600F098FF002005B0C4
:102B2000F0BDC0468C2901000897010253454E4470
:102B3000204F4B0053454E44204641494C00000075
:102B4000B8140100204E00008813000041542B43AC
:102B5000495053454E443D25642C25750D0A00000F
:102B6000F0B583B0074600F0F5FF0026304604F0CC
:102B700025F9032835460BD10421284604F094FAA0
:102B8000F86B51492A4600F061FF304603B0F0BDB2
:102B900002970024204604F011F90428254609D1A3
:102BA0000298C06B49492A4600F050FF264630463D
:102BB00003B0F0BD0027384604F000F905283D4673
:102BC00009D10298C06B40492A4600F03FFF3E46BB
:102BD000304603B0F0BD01970125284604F0EEF819
:102BE0000328029FC8D00125284604F0E7F80428EE
:102BF000D6D00125284604F0E1F80528019FE0D051
:102C00000225284604F0DAF80328029FB4D00225F2
:102C1000284604F0D3F80428C2D00225284604F040
:102C2000CDF80528019FCCD0254C2068401C0321FD
:102C3000FDF766FA0D46084604F0C0F80628029F24
:102C400008D1284604F0B0F8002803D001F04BF971
:102C500000282AD1681C0321FDF752FA0D460846C8
:102C600004F0ACF8062808D1284604F09DF80028A6
:102C700003D001F038F9002817D1681C0321FDF7B3
:102C80003FFA0D46084604F099F80021CE43062885
:102C900000D07AE7284604F087F8002800D174E7CE
:102CA00001F021F9002800D16FE72560F86B054994
:102CB0002A4600F0CBFE0026304603B0F0BDC046E9
:102CC00044990102781501003815010048150100EA
:102CD00080B58AB00620042107F092FF4B20C00186
:102CE00009900820079064200690B448143005909D
:102CF0000648039002200190012002908002049077
:102D0000032001A904F008FC0AB080BDF0BD010257
:102D1000B0B582B001220F293ED803468068446BCB
:102D20002468C0467944097949008F44071F252744
:102D3000343535353535353535350A1527490022D1
:102D400004E02649CA68092A20D8521CCA601649DC
:102D5000164A00F021FC1EE0002003F0E1FC0128EF
:102D600019D11E4830300E49002212E000F04EFC0E
:102D7000204600F0BBFE0EE00D4908E00E2000905A
:102D800000210122204600F051FE04E00549002206
:102D9000184600F05BFE0022104602B0B0BDC046EF
:102DA000F8140100D8140100881300003F28010026
:102DB0008814010080B5032004F096FB80BD00005C
:102DC0000648416B0020002905D0054A914203D0F6
:102DD00049680029FAD1704701207047D498010250
:102DE000C8140100B0B514460D460846114600F05F
:102DF00032FF012816D1285D002813D1002C0BD0FA
:102E00006019401E00780A2806D10320084A0146AE
:102E10002B460CF03DF805E00320054A01462B4601
:102E20000CF036F803202946224604F049FCB0BDD8
:102E3000D5270100F0B585B0054604A8002404702C
:102E4000E743002D12D0EA68002A0FD0686A0028F4
:102E50000CD0A86A002809D0401EE96A814200D33C
:102E60008EE004A928469047002803D03C4620461F
:102E700005B0F0BD514EE86A411CE962696A049AE6
:102E80000A54E86A696A002202920A54E86A092828
:102E900006D1696A09224848FDF77BF900283ED02F
:102EA0003078411E022908D800F054FEB168401A5B
:102EB0004349884264D8414E30780A2820D00128FE
:102EC00023D16E6A3A213046FDF752F9002847D0E7
:102ED000019002980390E96A03AB304639A200F0F2
:102EE000D3FE02284CD10398002849D00A21334A46
:102EF000117001990818696A401AC01C50602FE0CF
:102F00007068E96A81422BD13AE004A800780A2867
:102F10000FD00D2814D101202863E86A1AE001209F
:102F2000307000F017FEB0603078411E0229BBD926
:102F3000C3E7296B012904D102202863E86A03E072
:102F4000296BE86A022905D1022817D10298E862A4
:102F5000286305E0012803D1686A00783E280FD075
:102F6000A86AE96A401E81420AD2EA6804A9284692
:102F700090470028114E00D17DE777E7029828633B
:102F8000E96A686A00F067FE01280FD16B6AE86A97
:102F9000002806D0C018401E00780A2801D10DA2D2
:102FA00000E010A2032001460BF072FF03480470FA
:102FB000204605B0F0BDC0461821010090960102E0
:102FC000DC0500002B524543454956452C252A2C4B
:102FD00025643A005B415420526563765D20257379
:102FE000000000005B415420526563765D2025732C
:102FF0000D0A0000B0B50F2001F040FB194D6870BC
:10300000287033282AD120243721204601F082FB62
:103010002120032101F07EFB2220402101F07AFBD8
:103020002320082101F076FB3020AA2101F072FB59
:103030000D4802210187322001F06CFB3320012171
:1030400001F068FB5F21204601F064FB0F2001F0D6
:1030500015FB28700A2005F037FEB0BD024800219C
:10306000C187B0BDC4950102D6A60102F0B583B0F8
:1030700001903B4C2120029060723A4800886070B9
:10308000394FB98861717A6A7A61384A1278227048
:10309000000AA070080AA0717D78C320060209F01A
:1030A00045FF01998D420DD17D21C900FDF712F830
:1030B0000D46F98009F03AFF28182E494118787812
:1030C000464303E04E432A49711806468D19BD62F6
:1030D00009F0C2FE40190AF01BFB06460D462648C1
:1030E000007B0AF0A1F9254909882222A15482B265
:1030F000D20B801802B2D0175210B2186841130ECA
:10310000029D6355130C202563553B6DA3761D0A64
:10311000E5761D0C25771B0E637723462233090ABB
:103120005970A277BA64F864BA65F865100AE07756
:1031300009F0FCFEB861BB6A2821012220460DF08F
:10314000F1F8F86209F0F2FE386108F017F900288A
:10315000FBD1042007F0D0FC002003B0F0BDC04636
:10316000B2D00102EC97010208960102CA9701024F
:10317000609E010060DB0000BA900102D697010258
:1031800070477047B0B582B0194C2068056801A936
:103190000020087007E090470198401C01A90870C2
:1031A000C0B2082822D2012211048140294209D04C
:1031B0002268516080002018826A002AECD001A8A1
:1031C0000121E8E7130283402B4201D0022104E0F1
:1031D00082402A42E0D003211346226853608000D7
:1031E00020188268002AD7D001A8D4E702B0B0BD69
:1031F000C8920102FEE7000010B509480168CA69DB
:1032000020231343CB610269032A08D101229305CD
:103210000C689C430C605102C26E0A43C26610BD2A
:103220003C93010281B010B581B00393002807D010
:10323000C16A002904D003AB0093C46A0021A047EF
:1032400001B010BC01BC01B00047000080B50246CF
:1032500008480068002807D091B2120C03889A42EF
:1032600003D040690028F9D180BD002200F04AFB5C
:1032700080BDC046FCC60102F0B581B05C4C206840
:10328000856BE80707D0E168002904D00020884753
:10329000206801218163A80707D52169002904D08E
:1032A00001208847206802218163680707D561698A
:1032B000002904D002208847206804218163280760
:1032C00007D5A169002904D0032088472068082178
:1032D0008163E80607D5E169002904D00420884706
:1032E000206810218163A80607D5216A002904D02F
:1032F00005208847206820218163680607D5616A18
:10330000002904D0062088472068402181632806D0
:1033100007D5A16A002904D00720884720688021AA
:1033200081630126E80507D5E16A002904D0370248
:103330000820884720688763A80507D5216B0029E6
:1033400004D077020920884720688763680507D57D
:10335000616B002904D0B7020A2088472068876380
:10336000280507D5A16B002904D0F7020B20884758
:1033700020688763E80407D5E16B002904D0370390
:103380000C20884720688763A80407D5216C002992
:1033900004D077030D20884720688763680407D529
:1033A000616C002904D0B7030E208847206887632A
:1033B000280407D5A16C002904D0F7030F20884703
:1033C00020688763E80307D5E16C002904D037043F
:1033D0001020884720688763A80307D5216D00293E
:1033E00004D07504112088472068856301B0F0BDC2
:1033F000CC930102B0B52B4802782B490B781343CC
:1034000012D02A4A13885B1C138044784D78002D13
:1034100012D0002C1BD09BB2F02B0CD30023437096
:10342000012048701380B0BD204A002313808B70A8
:103430004B7001214170B0BD002C0FD09BB2F02B1E
:10344000F9D30023138001224A704370B0BD0024D9
:103450008C709BB2064DAB42EDD304E000248C701F
:103460009BB2792BE7D3012343708B701480B0BDDE
:10347000B1040000B0B50B4A1378002B0CD1002921
:103480000AD0094B1C78002C06D1064C012565702A
:10349000064C002525805D70002800D1024A11707D
:1034A000B0BDC046409001026C97010242AB0102E0
:1034B000F0B58DB0002862D00446406800285ED088
:1034C000A06840285BD8E56A002D58D00746204602
:1034D00040300026039003E0019E4AE0039848E054
:1034E000402101220691FCF731FEAE4202963ED207
:1034F00000203146019009900398069B3E46002E1D
:10350000EAD0606A0491405C07900998401C0590DD
:103510000021042708916518EA5C012A17D10A9650
:103520006268D3191B1F1B68099E9E5D079886421F
:1035300008D1059D5B5D002B0A9E22D00898401C97
:10354000089003E0403500222A70A668069B0837E1
:10355000491CB142DFD308980028BFD00499491C08
:10356000E06A8142059809900398C8D301E0039866
:103570003E463746E56A029E761CAE42B0D30DB099
:10358000F0BD616A0B91E16A0C91D1590BAA2046FA
:1035900000F09CF80DB0F0BD81B0B0B583B00D4621
:1035A0000446079307AB02938069E1690CF036FF8C
:1035B000206265480078002803D1216AA06900F0E4
:1035C0009FF96369A169226A204698470146A06B6A
:1035D000002905D069460C600021224B0A460CE008
:1035E00000F084FA7D2081002846FCF773FD024636
:1035F000A06B69460C6000211B4B00F0D3FA002041
:1036000003B0B0BC02BC01B00847C04680B5806BB7
:1036100000F06CFA002080BD70B582B00D46044603
:10362000466911461A46B0470146A06B002907D0EB
:1036300069460C6000210B4B0A4600F0B3FA0EE01D
:1036400000F054FA7D2081002846FCF743FD024635
:10365000A06B69460C600021034B00F0A3FA002028
:1036600002B070BD513700006737000070B50D46DD
:103670000446802100F0C0FA2868E0636868606052
:10368000A868A060E868E0602869206168696061F6
:10369000A869A061E86900262662E061286A606284
:1036A000686A2663E662A062A86A606320463830D2
:1036B00000F02AFA002802D0F643304670BD2148B7
:1036C000016821600460304670BDC04670B5144684
:1036D0000D460646881E032802D8B06B00F006FA95
:1036E000F06B2946224600F00DF970BD16480178AE
:1036F000012048407047C04670B512480468002C4D
:103700001FD0114E11A5216920468847002815D1E8
:10371000307800280DD1E16A606A00F09CFA014619
:10372000606A012903D0E16A00F0E8F8284600F059
:10373000E3F82046FFF7BCFE0020E0622468002C7E
:10374000E1D170BDF8C60102F0C601020D0A000009
:1037500010B50446806B00F0C9F9E06B052100222A
:1037600000F0D0F810BD10B50446806B00F0BEF933
:10377000E06B0421002200F0C5F810BDF0B581B067
:1037800000910646C7680468A01C3946FCF7A2FCF5
:1037900000257068814201D1ED430BE0601C394681
:1037A000FCF798FC316032695143B0680818009901
:1037B000FCF7BAFC284601B0F0BDB0B501240025E5
:1037C0000560446008300EC0B0BD70B50E460446BA
:1037D000C1680068401CFCF77DFC002560688142E0
:1037E00002D1ED43284670BD22695043A1684118BB
:1037F0003046FCF799FCE1686068401CFCF76AFC05
:103800006160284670BDB0B5002400280DD0054683
:1038100000688842FDD3401A286068684018E9684B
:10382000FCF758FC69602046B0BDE4432046B0BDBB
:10383000B0B5002400280ED0054600684018286066
:10384000EA689042FDD8A86840181146FCF742FC8F
:10385000A9602046B0BDE4432046B0BDF0B583B0BA
:10386000164602460027F843002E22D01C46002BA5
:103870001FD00D46D168136899421AD9CB1AAB42B2
:1038800017D39268019252198A423A4607D9019A8F
:103890008A1A0292029A52199342029A09D3029208
:1038A00001981018FCF716FC31600298401920604E
:1038B000384603B0F0BD40687047806870470246E4
:1038C0000020002A04D0106050609060D1607047E2
:1038D000C0437047002803D0016848424841704700
:1038E00001207047002805D00168C068411A48428D
:1038F0004841704701207047002070470020704702
:1039000000207047F0B583B014460D460646408847
:10391000012818D1306900280CD0A900405801783E
:103920002D2910D0F368716809686A4611605060EB
:1039300010A205E0F36870680068694621C115A20D
:103940003046FFF76FFC7768FB6830462946224611
:103950009847012808D00AE0C36830462946224625
:1039600098477F68012802D178680028F4D103B015
:10397000F0BDC04646534D3A252D3873205354416F
:1039800054453A252D323873204556454E543A2534
:10399000730D0A0046534D3A252D38732053544178
:1039A00054453A252D323873204556454E543A2514
:1039B000750D0A00F0B581B0002828D01E460C46CF
:1039C0000546079B0698009000206862A862E8629E
:1039D000104909886B8029800F4B1F686C60009B21
:1039E000AB602B460C33C4C3A861E8612862481C55
:1039F0000849088008480560002C08D06C60002148
:103A000028460A46FFF77EFFA468002CF6D101B0D5
:103A1000F0BDC04680CA0102FCC601020246002079
:103A2000002A01D0D1627047C043704710B582B000
:103A300004AC24881B881B041B196C462360024BB2
:103A400000F0B0F802B010BD4D320000F0B597B0F4
:103A50001646029105464268002A30D001966A60F7
:103A600001210024284616462246FFF74BFF304628
:103A7000029FBE4232D003A85021FCF76EFB3246B3
:103A80007268002F0CD003AF029811C74068083F3E
:103A9000824209D0394608313C4600280F46F4D10D
:103AA000002A019EDBD10AE0019E3868686000218F
:103AB00028463246FFF726FF7F68002FF5D102988F
:103AC0008468002C08D06C60002128463246FFF73D
:103AD00019FFA468002CF6D117B0F0BD00212846CC
:103AE000019E3246FFF70EFFE9E700000146002085
:103AF0001F2901D9C043704718224A433449012382
:103B00008B5089188860704710B50021CC4300287D
:103B10000BD00A4A1368002B09D01832491C2029FF
:103B2000F8D306D106A0FFF7E7FE204610BD01231B
:103B3000136001600024204610BDC04680C701020A
:103B400074696D65722049442069732066756C6CD8
:103B50000D0A0000264800687047C04670B5202452
:103B60001B4D234E2868022817D13068A968EA68DF
:103B7000401A904211D96969002907D02879002894
:103B800007D0022028603068A86004E00120286087
:103B900003E001202860286988471835641EE1D1B8
:103BA00070BDC046F0B5044600201F2C01D9C043AB
:103BB000F0BD059D18266643054C0227A751A419A0
:103BC00021710B4909682646083626C66361F0BD97
:103BD00080C7010206480168491C01600548416828
:103BE00002680023521C02604B4143607047C0468C
:103BF00030AB010238AB010280B5FCF7AEFA80BDF4
:103C0000B0B50278002A24D0441C0021084601E007
:103C1000573A08E023460001D5B2302D0C4611D3A7
:103C2000392D02D8303A14460CE0412D0C4609D308
:103C3000462D01D8373AF6E71446613CE4B2062C2B
:103C4000E6D30024E2B280185C1C1A78002AE1D185
:103C5000B0BD0020B0BD10B50246012000290DD036
:103C60000023D45C202C02D37F2C04D307E00D2C3E
:103C700001D00A2C05D15B1C8B42F2D310BD002071
:103C800010BD002010BD000081B0F0B584B00993D4
:103C900000230393002800D1C2E0002A00D1BFE036
:103CA00009AB03931678002E00D1A8E05623DB431E
:103CB000009300231D46002900D1A2E0252E3FD10C
:103CC000971C52781446643C0023142C43D8C046F9
:103CD0007C4424796400A7440A99A3A3A3A3A3A3C3
:103CE000A3A3A3A34CA3A3A3A3A3A3A35F0002978F
:103CF000039A131D039312680192012200231746B1
:103D00001E460478FF0703D02D2C01D1164607E08C
:103D10002746303F092F09D80A275F433B19303B1C
:103D2000491E401C00270029EBD13946029A019C0C
:103D3000002C03D0012E00D15B4223606B1C06E0F7
:103D40000378B3425BD1491E521C401C2B461678A7
:103D5000002EAFD164E02A2A62D13A7803789342E8
:103D600004D0491E401C0029F8D100216B1C3A46A2
:103D7000EDE7039A131D03933E7812680023C45C99
:103D8000B44233D0491E5B1C0029F8D13C46C71809
:103D90000021002A2ED12EE00297039A131D0393CF
:103DA00012680023009E0778302F18D33A2F02D2D2
:103DB000344627340BE0612F03D3672F344606D3F4
:103DC0000DE03C46413C052C09D8344620341B010B
:103DD0001B19DB19491E401C0029E4D10021029C5B
:103DE000002A00D013606B1C2246B0E73C46C7187F
:103DF000002A00D009C26B1C22463846A7E70023E0
:103E00000EE0252E0BD15178652908D103990A1DA2
:103E100003920968002900D008606B1C00E02B4663
:103E2000184604B0F0BC02BC01B0084781B010B520
:103E300081B00C46039303AB00930CF0EFFAA04261
:103E400000D3601E01B010BC02BC01B0084770B5C1
:103E500004460020002A1BD0002C19D0002B17D0BC
:103E600014600120022B13D32578002D10D0641C80
:103E700001208D4205D1651E00262E70850054510B
:103E8000401C984204D2661C2578002D3446F0D19F
:103E900070BD70B504460026F043002C0DD00D46D1
:103EA00000290AD0204610300121FFF7ACFCA96898
:103EB00020342046FFF7A7FC304670BD70B504469D
:103EC0000026F043002C0DD00D4600290AD02046D4
:103ED00010300121FFF7ACFCA96820342046FFF721
:103EE000A7FC304670BD70B50024002814D00546EC
:103EF000064610363046FFF7EDFC01280CD0284668
:103F00002030FFF7E7FC012806D02C683046FFF789
:103F1000D2FC0C2141436418204670BDF0B583B03B
:103F200000250295019500281FD00C46064607463D
:103F300010373846FFF7D6FC002816D1304620301F
:103F400002AA01AB2146FFF789FC00280DD1356894
:103F50003846FFF7B2FC0C214143B068029A1018B2
:103F600068506D186C600198A860284603B0F0BDD9
:103F700070B505460C2058430024904211D2121A05
:103F8000461829606860AE60EA602846103019461D
:103F9000FFF795FCE96820352846FFF790FC20469E
:103FA00070BDE443204670BD04217046084204D031
:103FB000EFF30983EFF3088203E0EFF30883EFF3F5
:103FC00009829BB004A8F0C044464D4656465F4661
:103FD00008A8F0C01846F0C86846F0C018690C90F0
:103FE000202018440D9058690E9098690F90D86958
:103FF0001090EFF310801190EFF3148012900949A4
:1040000008681390084908681490084908681590D2
:1040100007490868169017931892704619906846D9
:104020000AF0F4F804ED00E00CED00E010ED00E023
:1040300014ED00E0F0B581B003260024304621469F
:1040400006F0DEFD04252846214606F0D9FD0127AD
:10405000304639463A4606F067FD3046214632463C
:1040600006F0F6FD284639463A4606F05DFD022187
:104070002846224606F0ECFD01B0F0BDF0B589B04F
:1040800008900425284606F037FD0A27384604F034
:104090001BFE284606F040FD0324204606F034FDB2
:1040A00007900526304604F00FFE284606F024FD52
:1040B000384604F009FE284606F02EFD204606F09C
:1040C00023FD0690304604F0FFFD284606F014FD5F
:1040D000384604F0F9FD284606F01EFD204606F09D
:1040E00013FD0590304604F0EFFD284606F004FD70
:1040F000384604F0E9FD284606F00EFD204606F09D
:1041000003FD0490304604F0DFFD284606F0F4FC81
:10411000384604F0D9FD284606F0FEFC204606F09D
:10412000F3FC0390304604F0CFFD284606F0E4FC93
:104130003846019704F0C8FD284606F0EDFC2046FD
:1041400006F0E2FC0290304604F0BEFD284606F080
:10415000D3FC384604F0B8FD284606F0DDFC2046C6
:1041600006F0D2FC0746304604F0AEFD284606F0C5
:10417000C3FC019804F0A8FD284606F0CDFC2046BB
:1041800006F0C2FC0446304604F09EFD284606F0C8
:10419000B3FC0699481E81410A460799481E814191
:1041A000480080188000059A511E8A41510040182D
:1041B000049A511E8A4180188000039A511E8A4138
:1041C00051004018029A511E8A4180188000791EC1
:1041D0008F4179004018611E8C410619089800280B
:1041E00003D0032006F088FC02E0032006F094FCD4
:1041F0000A24204604F068FD0425284606F08CFCBD
:10420000204604F061FD284606F076FCF0B209B0C5
:10421000F0BD70B50446042006F06EFC60B20028C4
:1042200003D4032006F068FC02E0032006F074FCCF
:104230000A25284604F048FD0426304606F06CFCAA
:10424000284604F041FD304606F056FC284604F0AE
:104250003BFD600603D4032006F04EFC02E0032081
:1042600006F05AFC0A25284604F02EFD04263046A6
:1042700006F052FC284604F027FD304606F03CFCD0
:10428000284604F021FDA00603D4032006F034FCE8
:1042900002E0032006F040FC0A25284604F014FD45
:1042A0000426304606F038FC284604F00DFD304662
:1042B00006F022FC284604F007FDE00603D40320A4
:1042C00006F01AFC02E0032006F026FC0A25284628
:1042D00004F0FAFC0426304606F01EFC284604F0E2
:1042E000F3FC304606F008FC284604F0EDFC2007FD
:1042F00003D4032006F000FC02E0032006F00CFCCF
:104300000A25284604F0E0FC0426304606F004FCAA
:10431000284604F0D9FC304606F0EEFB284604F0AF
:10432000D3FC600703D4032006F0E6FB02E0032081
:1043300006F0F2FB0A25284604F0C6FC04263046A7
:1043400006F0EAFB284604F0BFFC304606F0D4FB3A
:10435000284604F0B9FCA00703D4032006F0CCFBE8
:1043600002E0032006F0D8FB0A25284604F0ACFC46
:104370000426304606F0D0FB284604F0A5FC304663
:1043800006F0BAFB284604F09FFCE00703D10320A7
:1043900006F0B2FB02E0032006F0BEFB0A24204632
:1043A00004F092FC0425284606F0B6FB204604F0F3
:1043B0008BFC284606F0A0FB204604F085FC70BD6F
:1043C000F0B581B003260025012430462946224657
:1043D00006F0AAFB304606F09FFB0626304604F0A6
:1043E00073FC042006F098FB304604F06DFC0320BB
:1043F00006F08AFB00281BD0681CFA2D0546F6D370
:104400000425284606F078FB0326304606F074FBA8
:104410000A27384604F058FC284606F07DFB304653
:1044200006F07AFB384604F04FFC204601B0F0BDA0
:10443000032001210A4606F077FB042006F05CFB0E
:104440000024204601B0F0BDB0B50446C00703D13A
:10445000032006F051FB02E0032006F05DFB082577
:10446000284606F059FB284606F046FBA00703D471
:10447000032006F041FB02E0032006F04DFB082577
:10448000284606F049FB284606F036FB600703D4B1
:10449000032006F031FB02E0032006F03DFB082577
:1044A000284606F039FB284606F026FB200703D4F1
:1044B000032006F021FB02E0032006F02DFB082577
:1044C000284606F029FB284606F016FBE00603D432
:1044D000032006F011FB02E0032006F01DFB082577
:1044E000284606F019FB284606F006FBA00603D472
:1044F000032006F001FB02E0032006F00DFB082577
:10450000284606F009FB284606F0F6FA600603D4B2
:10451000032006F0F1FA02E0032006F0FDFA082578
:10452000284606F0F9FA284606F0E6FA60B20028B6
:1045300003D4032006F0E0FA02E0032006F0ECFAD0
:104540000824204606F0E8FA204606F0D5FA0724AB
:10455000204606F0E1FA204606F0CEFAB0BDF0B5EE
:1045600081B0032700243846214606F039FB38463F
:10457000214606F045FB012538462946224606F02D
:10458000D3FA052638462946324606F061FB08274D
:104590003846214606F034FB38462946224606F0C6
:1045A000C3FA38462946324606F052FB07273846FA
:1045B000214606F025FB38462946224606F0B4FA85
:1045C00038462946324606F043FB01B0F0BD0000F4
:1045D00010B50B2006F098FA13490A7800280BD082
:1045E000002A1DD11148012404700C7010480021CC
:1045F00001700AF085FD0AE0012A11D10B48002262
:1046000002700A700A48012404700AF05DFDA202DB
:104610000849094B20460BF08FF802F0E3FE10BD6D
:1046200002F0E0FE10BDC04620D1010298980102C0
:104630001890010288CB010271F9000002488068DD
:10464000811E484248417047E095010280B5FDF760
:10465000FFFA002801D00020C04380BD80B5FEF7DE
:10466000AFFB80BD10B504480F2100242246FFF7A0
:1046700049F9204610BDC04604990102F0B581B049
:1046800007460324204606F047FA0425284606F08C
:1046900043FA204606F030FA0A26304604F014FBAE
:1046A000284606F029FA3220FFF7B3FDFFF788FE0F
:1046B000F8B2FFF7AEFDFFF783FE204606F02CFAB6
:1046C000284606F029FA204606F016FA304604F08D
:1046D000FBFA284606F010FA3320FFF79AFDFFF7A1
:1046E0006FFE0020FFF7CAFC0746284606F004FAD2
:1046F000204606F001FA304604F0E6FA284606F0B5
:104700000BFA204606F008FA304604F0DDFA384687
:1047100001B0F0BDF0B581B00091074603242046FA
:1047200006F0FAF90426304606F0F6F9204606F0BF
:10473000E3F90A25284604F0C7FA304606F0DCF90A
:104740003220FFF766FDFFF73BFEF8B2FFF761FD91
:10475000FFF736FE0098FFF75CFDFFF731FE3046AD
:1047600006F0CAF9204606F0C7F9284604F0ACFA6C
:10477000304606F0D1F9204606F0CEF9284604F07E
:10478000A3FA284604F0A0FA01B0F0BD80B50748AE
:1047900001210170064802680A4302600548026868
:1047A000002A02D000200146904780BD86CA01023F
:1047B0001C10005088CA0102F0B599B0F548017B81
:1047C000C67A427B0E92F44C221F1368F34A126899
:1047D000069242780C9202790592C76A04931F40B0
:1047E00001200F907A0200D5BCE03A0200D5BFE06C
:1047F000FA0102D50F9802062260502508968A1900
:104800001826BB0102D50F98430623604123079564
:1048100069430A96354655431426FC0210D50F9875
:10482000040538463746DC4E3460DA4CA469B4647B
:10483000D84CE4697464DA4C241D34603E46074663
:1048400090000B90D8040D90681809900E9B73434C
:104850000F988203B902D04D22D50F9841052960E7
:10486000CC480E961646024681692965C16969657C
:1048700009990D9801430898000108180B994018F0
:10488000C018C849098892794A4380180A301C46E2
:1048900004F0FAFC234632460E9EC04988672A601F
:1048A0000F98C404380300D52C60F80302D50F9884
:1048B000000428600F984104B80300D5296038042B
:1048C00000D4E4E1039402910E9308920D980B99A1
:1048D0000C180A980C9941430C910F98C0030B9047
:1048E000286007F0C7FA002801D004F0AFFC0C984C
:1048F000005B410B43D1099800190E9940180599A6
:10490000090140180E90E74D287B079B4343E97A45
:104910000A010D9C2243D21841188B00D2180A9B21
:104920004B43D1186A7B564389190E9E2A79101879
:10493000DF4A12884243881816903068C000800D04
:1049400010A9C882002511957079C0077ED110A8E2
:104950000F998182069C00940020E8A2049B0AF033
:1049600097FA78E00F98820522603A0200D43FE778
:104970000F98C2052260FA0100D53BE73DE7072109
:1049800049030840032149038842089A00D07EE188
:10499000069706F01BFF0020169009901590C14C59
:1049A000E07A217B08180A99414380000D9A104350
:1049B0004118627B0E9672438A186178A379079E2C
:1049C0007343D718FA683F26324063789A420C97AF
:1049D0006ED105960A9A4A4380580F210A07024071
:1049E0000398401EC04B1B68DB09034098181090C9
:1049F0000F98C0020B90B868800767D42C46283CFB
:104A000009F0BCF905462068000609D5C3208401D9
:104A1000786A400704D409F0B1F9401BA042F7D9E5
:104A200005980002B96849080140B34803688268E4
:104A3000B868C40C20202040DB0700D095E000239C
:104A400010221D461C460E9E0B9FB1E010A88582C9
:104A5000B0681190069C701D924B1979E20707D13E
:104A6000491C1971D97A1A798A4202D31D7100E062
:104A7000D97001784278120251188278120489188C
:104A800003229143017035715878401C5870D87AD0
:104A9000197B08185978884200D85D70D879401E73
:104AA000D871596B002901D010A888477E4DEDE0E0
:104AB00010A80B998182F86830406378009000203C
:104AC0007CA20F990AF0E4F90E9E94E0388A874A96
:104AD000024010A8C2822022BA5C9307DB0F3C6818
:104AE000C3720F9B1A4082726205D20C0D9B1A434F
:104AF0001692FA68130E0372BB69FC697C4D2D682F
:104B00002D0C05745204920F427211931394654C4C
:104B1000A07B002809980E9E0B9F5FD07548006807
:104B2000007A0328099859D00C98007D084009287C
:104B3000099853D1C320840109F020F905460C9847
:104B4000406A41070BD4594909680906890F06D103
:104B500009F014F9401BA042F1D90C98406A4103B6
:104B60000898884310A9888237E0D2070E9E0B9FD1
:104B700003D108230022154619E00C9B9A68029C79
:104B8000224211D19A68520C022494430022134607
:104B900015460DE08CCF010228A000503CA100502A
:104BA000FC1F000088CF0102042500221346144692
:104BB0000843104318432843204310A988823842F1
:104BC0000BD10C9B198A494A0A4010A9CA8219685C
:104BD0004905C90C0D9A11431691324C2921615C8B
:104BE000002908D03037B84205D010A90846113046
:104BF000123108F02FFCE77A2A48047BE51929488E
:104C000000790E9027484078401C2946FBF762FA4D
:104C100088000D9A1043189007996143380110439A
:104C200040182049497B4E4380191C216943401894
:104C30000E9909191B4B1E4A12884A438018179077
:104C4000099A0C998A60987B002800D04A6298796A
:104C5000401C9871187B99798142069F00D39A7104
:104C60005978491C5970D97A0818597888420E4DDC
:104C700000D85A70187A401E18722820185C002834
:104C800004D0996B002901D010A88847089A1742D0
:104C900002D00F98000328601C480449486019B0EE
:104CA000F0BDC0468CCF010228A000503CA10050AE
:104CB00088CF010248572045542069647820256434
:104CC00020616E6420455420696478202564206941
:104CD0006E2052582064657363206D69736D617432
:104CE00063680D0A0000000038200040FF03000048
:104CF0009430004038940102604000404D41432010
:104D00004556542025782025780D0A00FFFFFF0323
:104D1000F0B5A5B01E460C9208910024239422A958
:104D20000C8016A90C8024A909250D80598C0D91A1
:104D3000FBF7D0F92A99012900D0DFE03189012958
:104D400000D0DBE0318C012900D0D7E00D9900299B
:104D500000D1D3E0224607962C990B912B9906910E
:104D600080B205900F9415A8058090000E900C99C4
:104D70000C582E460025204629461746FBF72CFDE9
:104D80000028119636D12C200A97784308990818E4
:104D900017A90A4668C868C2E8C8E8C2E8C8E8C2F5
:104DA000079F119880B280000E5822AD019523A86C
:104DB000009020463946059A069B03F093FF0F9812
:104DC000401C0F90288800282DD03B8A239913ACD3
:104DD000039416A8029014A8019015AE009617A887
:104DE00024AA04F059F92588308811900120149ED6
:104DF0000A9A05E013A8058014952E4628463A46DF
:104E00000E9F51000B9B119C5C52591808830D8416
:104E1000D81986600F981885521C0D9882426DD063
:104E200024A805889FE7099616A8002505801495F3
:104E300024A80688239812902F46109503E06D1C35
:104E4000A8B2B04213D8A8B2800017A90C582046C7
:104E50001299FBF7CFFC0028F1D1002FEFD115A854
:104E6000058016A80127078014941094E7E715A879
:104E70000288B01A012805D115A80680099F149749
:104E8000119628E010200799095E0129119221DB73
:104E9000551CA8B20C18109F0E9B099403E06D1CC2
:104EA000A8B2844218DDAAB2B242F8D8800017AA8C
:104EB00010581090394634461E46FBF78DFC334699
:104EC0002646099C0028EAD115A80580109F149752
:104ED0001195E4E7109F0E9B1C463E4638461299FA
:104EE000FBF7A9FAFBF7DEFC0546052800D30525EC
:104EF00013A8058001200A9A274682E725B0F0BD55
:104F0000F0B58BB00243159A149C139E2BD0054626
:104F100001A856C0129CD869196A09900A911E46C8
:104F20009F6B0123009309A807AA0146059305F08A
:104F3000B5FE716C3846FBF77EFA0746E06A616B96
:104F4000FBF779FA002D069613D0044611980199C3
:104F5000012924D10921081A0421069A515E8842A8
:104F600029D16425B1E000203080207010700BB092
:104F7000F0BDB08800226425002829D00592694937
:104F80003846FBF753FC0028049C039E6FD166490A
:104F90003846FBF74BFC00281DD05A2567E03C251E
:104FA000082800D191E05F492046FBF73FFC00282C
:104FB00019D0502589E00A291DDB1D293BDC594900
:104FC0003846FBF733FC0022002854D05A253AE03B
:104FD0003346049C39E055493846FBF727FC002846
:104FE00021D0502543E050492046FBF71FFC002804
:104FF0002ED0462569E03C25012866D04949204647
:10500000FBF714FC0028D4D147492046FBF70EFCDF
:105010000028EED145492046FBF708FC002854D172
:10502000434920466EE042493846FBF7FFFB002823
:105030001CD128251BE03B493846FBF7F7FB002233
:10504000002832D05025049C069B0299039E41E023
:1050500036492046FBF7EAFB002836D13449204682
:10506000FBF7E4FB00282FD114252EE03725029909
:10507000059A069B2EE005922B493846FBF7D6FB96
:10508000002896D129493846FBF7D0FB0028B0D13B
:1050900027493846FBF7CAFB0028049C069B029967
:1050A000039E059A3BD11E2514E005921E49384601
:1050B000FBF7BCFB00289CD11C493846FBF7B6FB2C
:1050C00000281DD03C2500E02325049C069B029966
:1050D000039E059A258032700020087030780028E1
:1050E0000CD118681349FBF793FB002806D12088E0
:1050F000102803D30F3820800BB0F0BD0BB0F0BDEB
:105100000B493846FBF792FB0028049C069B02994A
:10511000039E059A01D11425DCE72325DAE72D2526
:10512000D8E7C046CDCCCC3DCDCC4C3DCDCCCC3C55
:105130000AD7233C0000204070B588B00C460646D4
:105140004088002820D0FBF798FB059005A804A90B
:1051500001252A4606F00CF83088B188081AFBF7BA
:1051600081FB0390049903A807AA2B4605F0C0FF12
:105170005249079D2846FBF759FB002808D0BF205D
:105180000006206008B070BD0020206008B070BD2F
:105190004B492846FBF72EFB002804D03F20000691
:1051A000206008B070BD47492846FBF73FFB002848
:1051B00001D0002010E000212846FBF737FB002833
:1051C00001D0022008E040492846FBF72FFB0028C9
:1051D00001D0042000E0062001957F21C90502913D
:1051E00080003A49091801A806AA022305F034FFF5
:1051F0000698206008B070BDF0B587B00C46054633
:105200004768002638463146FBF71EFB002802D0CF
:10521000266007B0F0BD049704A803A90126324612
:1052200005F0A6FFA8682968FBF7C0F8029003996B
:1052300002A806AA334605F05BFF2049069D2846D2
:10524000FBF7F4FA002804D0BF200606266007B05A
:10525000F0BD1B492846FBF7CDFA002804D03F20BB
:105260000606266007B0F0BD16492846FBF7DEFAB1
:10527000002801D0002010E000212846FBF7D6FAD4
:10528000002801D0022008E00F492846FBF7CEFA9B
:10529000002801D0042000E0062000957F21C905E8
:1052A0000191800009490918684605AA022305F002
:1052B000D3FE059E266007B0F0BDC046CDCC0C3FA6
:1052C000295C0FBFCDCC4C3ECDCC4CBE40940102EE
:1052D000F0B587B00C4606467F270088002801D02D
:1052E000FD0503E0B08800282ED0334DFBF7C5FA4A
:1052F00003907088FBF7C1FA049003A802A9012665
:10530000324605F035FF029904A806AA334605F097
:10531000EFFE2A49069E3046FBF788FA002802D0A5
:105320003F20010641E026493046FBF763FA00289A
:1053300002D0BF20010638E022493046FBF776FA5A
:10534000002805D0002024E00020206007B0F0BD38
:105350001D493046FBF76AFA002801D0022018E008
:105360001A493046FBF762FA002801D0042010E009
:1053700017493046FBF75AFA002801D0062008E00A
:1053800014493046FBF752FA002801D0082000E00B
:105390000A200096F905019180000F490918684616
:1053A00005AA022305F058FE05992846FBF706F8E2
:1053B000206007B0F0BDC046000080BF0000384349
:1053C0003333733F0000C8420000704200002042A7
:1053D0000000A0410000C04060940102F0B59DB003
:1053E00015460B917F210391C9051C9102911B91D8
:1053F00019A900248C80199418941794598C06913B
:10540000198C0F91DE8B998B0791997805911F88E4
:105410002B21CA432799914201DB7F0015E04022EE
:10542000D243914211DC4922D243914202DB7908F6
:10543000CF190AE05322D2439142EEDA5D22D243E1
:10544000914201DBBF0000E0FF000A971396269E01
:10545000597E00290BD0002132460F46D170917041
:1054600051701170121D7F1C5C7EA742F6D30C9305
:1054700011952599149122990D91159041088C420E
:1054800011D2FD4A2346A00084583454270A451CF3
:105490007755250C871CF555240EC01C34545B1C15
:1054A0009CB2A142EFD8239810900120099000905F
:1054B00030463146149A159F3B4605F0FDFB0D988A
:1054C00000060890400E139D00D186E0680004900D
:1054D000002F3FD0002210461146144606E01C461D
:1054E0001146159F401C82B2BA420ED283B2AB4223
:1054F000F8D09200149B9A5E0FB2BA42034600DCC9
:105500002346BA42EBDC0A46E9E7002F25D0002209
:1055100010461146129206E012931146159F401C48
:1055200082B2BA4214D283B2AB42F8D0A5B2AB4237
:105530000CD09200149B9A5E0FB2BA42034600DC74
:10554000129BBA42139DE7DC0A46E5E7139DE6E7A6
:10555000129903E00024214600E0002112911098E6
:105560000183C4828582049FF057FBF77BF9792180
:10557000C9050E91FAF722FF1099C86109980743EF
:10558000F057FBF76FF90E99FAF718FF109F386282
:105590002004C40B3057FBF765F90E99FAF70EFF9C
:1055A0007862601C3056FBF75DF90E9C2146FAF7D5
:1055B00005FFB86212980004C70BF057FBF752F9C9
:1055C0002146FAF7FBFE109CE062781C3056FBF790
:1055D00049F90E99FAF7F2FE2063119805800C98AC
:1055E000407E410000278D4228463A46149E1ED335
:1055F0000A9880B28AB29300F45E84420BDA491CA6
:105600008AB2AA42F6D9002728463A4681B2691AD8
:10561000012910D01BE0F018119B1980078808049D
:105620000FD0500040008019001F0288084681B248
:10563000691A01290BD1A800301811990D8007882B
:1056400026E00020024681B2691A0129F3D00A99A6
:1056500089B2079B4B43BB421AD306998A4217D89B
:105660000599002914D0401C82B2891803E0401C1F
:1056700082B291420CD983B2AB42F8D89200B35EA9
:10568000BCB2A342F3DDB218119B18801788EEE775
:1056900012970B980580119800882B1A002B16DDA5
:1056A00002210F9A1143032942D10E93411C421E3D
:1056B00010B281420EDA0E98032824DB0C98808CFD
:1056C000012820D019A818A9FFF736FD1FE00020F7
:1056D00018902BE00026F443374608E0B8B24000AB
:1056E00019AD2B527F1C521C10B28142E3DB13B266
:1056F000A3423346F2DD159B98423346EEDA800032
:10570000149B1B5AEAE719A818A9FFF7E1FD149E9C
:10571000139D0F9A012A13D0032A11D0022A04D113
:1057200011980088281A02280ADA0020179034E01D
:10573000022A01D1022BB8DA00201890012AEBD1FD
:10574000681C691E0FB2B84208DA0C98808C0128D8
:105750001DD119A817A9FFF7BBFD1CE00022D343F8
:10576000144608E0A5B26D0019AF7E53641C491CB5
:105770000FB2B842E9DB0DB29D421646F2DD159D2F
:10578000AF421646EEDABD00149E765BEAE719A832
:1057900017A9FFF7D1FC149E139D249F189C1799FD
:1057A0002046FAF703FE0F99012900D820463860F9
:1057B0000D98002800D1CBE011990888109FB88679
:1057C0000888281AB880129880B2FBF756F8792119
:1057D000CC052146FAF7F2FD2146FAF7EFFDB86352
:1057E000119F3888002849D081008919091F09882C
:1057F000129C0C191599884203D280008019808868
:10580000041915984300534916AA304605F032FC96
:10581000169810994864FBF75EF8A4B2A04201D133
:105820004D480FE0001BFBF728F81C901CA81BA993
:10583000012205F09DFC2046FBF71FF801461B984E
:10584000FAF7BCFD109908603988491B4A1C92B2CE
:10585000032A02D20021159F17E009B20229159FE1
:1058600012DB3F210906FAF7E1FF002802990CD16B
:105870000998810709E0C046402100400020129CA1
:1058800015998842B9D3BCE734491098016108984A
:10589000800E5DD0002F1CD0002211461446104609
:1058A0004B1B1DB2ED135B196B40139D1BB2920095
:1058B000B25E53431818A418491C8AB2BA42EFD3F7
:1058C000FAF7DBFF06462046FAF7D7FF002C03D194
:1058D00000E000260398C0051C901CA81BA9012508
:1058E0002A4605F045FC1B9C20463146FAF766FD2A
:1058F000014610988160002F119422D00024274681
:10590000264613951291B8B2FAF7B7FF1299FAF733
:105910004DFD0546A0001499085EFAF7A3FF014665
:105920001398C00785432846FAF748FD01463046DC
:10593000FAF7EBFC06467F1CBCB215988442E2D312
:1059400000E0002611983146FAF738FD1099C8603A
:105950001DB0F0BDD4A40102000020410000404071
:10596000F0B58FB00692F74A09AF70CA70C770CA17
:1059700070C70328079320D88800F3A10858F64978
:10598000FAF7C3FC0446F549FAF7BFFC0D90F44959
:105990002046FAF7BAFC0C90F2492046FAF7B5FC1B
:1059A0000B90F1492046FAF7B0FC0A90EF492046E7
:1059B000FAF7ABFC0990EE4969E0042822D00628EA
:1059C00020D88800EBA10858EE49FAF79EFC04465F
:1059D000ED49FAF79AFC0D90EC492046FAF795FC50
:1059E0000C90EB492046FAF790FC0B90E9492046D1
:1059F000FAF78BFC0A90E8492046FAF786FC0990F2
:105A0000FD4944E00838022821D88800FBA1085845
:105A1000D149FAF77AFC0446FC49FAF776FC0D9076
:105A2000FB492046FAF771FC0C90FF2081052046C7
:105A3000FAF76BFC0B90F7492046FAF766FC0A90E0
:105A4000CA492046FAF761FC0990FE491FE0880028
:105A5000F1A10858F449FAF758FC0446F349FAF75B
:105A600054FC0D90F2492046FAF74FFC0C90F14996
:105A70002046FAF74AFC0B90EF492046FAF745FC1E
:105A80000A90EE492046FAF740FC0990EC49009450
:105A90002046FAF73AFCEC4909680E90EB48046896
:105AA000EB4801684808EB4F05463D400022002DB9
:105AB00008922DD0CA01120E07D0280CE90D12D180
:105AC0004000E649085AE6490AE0C903090E0CD02D
:105AD000280AE90B10D14000E049085A8F218900BB
:105AE0004018E4300DE0DC490AE081B27F2905D896
:105AF0004800DA49085A04E0D94901E08F218900B9
:105B0000401800B2FAF7AEFED649FAF757FC024643
:105B10000292039507252606D34B1A68002A089897
:105B200040D0791C8A420BD21102090E13D0110CFD
:105B30001F46D00D1FD14800C849085AC84907E080
:105B40001F46110E002A13D44800C449085AC249FE
:105B50004018E4301FE011041F46090E0ED0110A50
:105B6000D00B12D14800BD49085A8F218900EFE7B8
:105B7000BE4808180FE0B84808180CE091B27F2919
:105B800006D84800B549085A05E0B548081802E0AB
:105B90008F218900501800B2FAF764FEB149FAF774
:105BA0000DFC3B460590159F2C40F50E5B69B049F6
:105BB0001940089810D0DA02D20E34D0C80B3E211A
:105BC0000140A648405AA6494018E43000B2FAF70E
:105BD00049FEA449FAF7F2FB0490149E6800A5A1BF
:105BE000085EFAF73FFE0146A00009AA1058FAF72E
:105BF0008CFB0146B8B20128089F019102D1022C0A
:105C00000AD9A74F052C24D1189808900C2D20D81C
:105C10000B2D16D3A44918E00027022C089718D0A2
:105C20008120C70515E01A04120E00D1CAE0080A47
:105C3000C90B00D0CDE040008849085A8F21890067
:105C4000C2E7092D00D2C7E096490898FAF75DFB34
:105C5000089001200021B542034600D30B46052CD5
:105C600000D308461799169A1A9C199D1843069B4B
:105C7000012B12D1079B402B22D1002840D038465F
:105C8000FAF743FB01460198FAF73FFB01460098FB
:105C9000FAF78CFB059A04998AE0079B402B1FD1E9
:105CA000002838D03846FAF730FB01460198FAF759
:105CB0002CFB01460098FAF779FB059A049977E0E6
:105CC000002833D03846FAF720FB01460198FAF74E
:105CD0001CFB01460098FAF769FB059A049967E0F6
:105CE00000285BD03846FAF710FB01460198FAF716
:105CF0000CFB01460098FAF759FB059A049957E006
:105D000002981146FAF752FB0399002900D167481F
:105D1000059A04994CE002981146FAF747FB03995B
:105D2000002900D16148059A049941E00298114682
:105D3000FAF73CFB0399002900D15C48059A0499C5
:105D400036E0C046940E0100000068C1000088C122
:105D500066665EC1000084C1000084410000B44159
:105D600000004841000020400000F0C0000084C155
:105D70000000F841333323C1000050C19A9929C172
:105D80009A9949C19A9949413333CB416666764124
:105D9000CDCCAC40333393C09A9949C10298114697
:105DA000FAF704FB0399002900D14048059A0499A9
:105DB00028601046FAF7FAFA0899FAF7F7FA20601D
:105DC0000FB0F0BD99B27F2911D848002349085A75
:105DD000FCE623494018F9E6C12001060898FAF7C5
:105DE00094FA0890062D00D933E7002030E78F2180
:105DF00089005818EAE6C0463333F341000058C121
:105E00009A9961C19A9969C1000084C10000AC41AE
:105E100000003841000008C1CDCC80C1CDCC88C184
:105E200033338FC1333397C133339741CDCC8C415A
:105E30003333F3409A9919C0666646C1333397C12C
:105E4000CDCCB4410000D4410C00004050300040A3
:105E500068400040FFFFFF007C0800009C1201002A
:105E60005C050000919AF63C642000409C0B000009
:105E7000FFFF1F00FAFFFCFFFEFF0000020004000E
:105E8000060008000A000C000E00100012001400AA
:105E9000160018001A001C001E002000220024001A
:105EA000000080BF0000A0C0000040C00000DCC2B5
:105EB000F0B5FFB0ECB017460E460D900021E99109
:105EC000E891DC9199919891979196911491139101
:105ED00012919AA8F49DF39CF29A002E00D1E6E16B
:105EE0000B938030F09B1180099529602546DBAC2F
:105EF000218095AC21800C952980DA917F24E405DE
:105F0000B994B894B794B694B594B494B394B29445
:105F1000B194B094AF94AE94AD94AC94AB94AA9475
:105F2000A994A894A794A694A594A494A394A294A5
:105F3000A194A0949F949E949D949C949B949A94D5
:105F4000046644668466C466046744678467C467FD
:105F5000046444648464C464046544658465C465FD
:105F6000046244628462C462046344638463C463FD
:105F7000046044608460C460046144618461C461FD
:105F8000B0090B250B2800D3AE011095012B0B9DFA
:105F900000D070E12B89012B00D06CE1298C002905
:105FA0000E9200D18BE16B8C002B00D1FAE1AA8C10
:105FB0003021695C002900D188E10892109F5F437D
:105FC0001196304639460F93FAF784F80590FAF7A0
:105FD00049FC01462046FAF72EFA8321C905FAF753
:105FE000EDF9064696A8021D119887420A9200D83C
:105FF00079E155A811909AA9069196AF15463A46AF
:10600000059C234605F028F815A80F9006992A4606
:10601000234605F021F802230D93384631463A46CF
:1060200005F066F8012308930093E8AA1092384619
:10603000394604F033FEE898DD901198069D294614
:106040003A46234605F008F80F9829460A9A23464F
:1060500005F002F8384631463A460D9B05F048F8FF
:10606000089B009338463946109A04F017FEE898CA
:10607000DE9011982C4629463A46059D2B4604F0A1
:10608000EBFF0F9821460A9A2C462B4604F0E4FFBA
:10609000384631463A460D9B05F02AF8089B009396
:1060A00038463946109A04F0F9FDE898DF901198C7
:1060B000069D29463A46234604F0CEFF0F9829460E
:1060C0000A9A2346254604F0C7FF384631463A4629
:1060D0000D9B05F00DF8089B009338463946109A41
:1060E00004F0DCFDE898E0901198069C21463A46C1
:1060F0002B4604F0B1FF0F9821460A9A2C462B46F6
:1061000004F0AAFF384631463A460D9B04F0F0FFF2
:10611000089B009338463946109A04F0BFFDE89872
:10612000E1901198069D29463A46234604F094FFD3
:106130000F9829460A9A2346254604F08DFF3846D3
:1061400031463A460D9B04F0D3FF089B0093384636
:106150003946109A04F0A2FDE898E2901198069C46
:1061600021463A462B4604F077FF0F9821460A9ABB
:106170002B4604F071FF384631463A460D9B04F039
:10618000B7FF089B009338463946109A04F086FD05
:10619000E898E390119821463A462B4604F05CFFBC
:1061A0000F9821460A9A2B462C4604F055FF384694
:1061B00031463A460D9B04F09BFF089B00933846FE
:1061C0003946109A04F06AFDE898E4901198069D0B
:1061D00029463A46234604F03FFF0F9829460A9A7B
:1061E0002546234604F038FF384631463A460D9B93
:1061F00004F07EFF089B009338463946109A04F05D
:106200004DFDE898E5901198069C21463A462B46AC
:1062100004F022FF0F9821460A9A2B4604F01CFF37
:10622000384631463A460D9B04F062FF089B0093C6
:1062300038463946109A04F031FDE898E6901198F6
:1062400021463A462B4604F007FF0F9821460A9A4A
:106250002B4604F001FF384631463A460D9B04F0C8
:1062600047FF089B009338463946109A04F016FD04
:10627000E898E7907AE010880C9A108099919891AC
:10628000DA9E08460F46099DF59CFAF78FF82860BC
:10629000DC9827606060A6600C34DDA80EC80EC4D0
:1062A0002EC82EC42EC82EC47FB06CB0F0BDFF2007
:1062B00010800021296020807FB06CB0F0BD0022EA
:1062C00001233021695C002900D076E6DDAA1ACFCF
:1062D0001AC23ACF3AC23ACF3AC20B213046F9F746
:1062E000F9FE054642E000200690059D0796089FAE
:1062F0001190069801460D9C0F9A4A43D219109BA3
:106300005A43119BD218D200A35889002E4655AD8E
:106310006B503546121DA25815AB5A50401C01B2A5
:106320008E42E9DC55A89AAE96AC314622462B4601
:1063300004F092FE15A831460A9A2B4604F08CFE12
:10634000022320460799224604F0D2FE012300933F
:10635000E8AA2046214604F0A1FC119B9800DDA983
:10636000E89A0A505B1C0B2B1846C1D1F19EDDA8A0
:106370009AA9DCAA0B2304F06FFE09210E980F9155
:1063800001800B98C168DC9C2046FAF717F801469B
:10639000A8B2E69F0F281BD808280DD30846F9F7A6
:1063A000B4FF14E0FF2010800021099A11600C99BD
:1063B00008807FB06CB0F0BD042803D3812208466A
:1063C000D10502E0412208461106F9F7F7FF014620
:1063D0002B20C04386420D9704DB0846F9F795FF52
:1063E000014603E04020C043864244DD0E9A0C9CE7
:1063F0000B98408A002811D00B98038A95A8039027
:10640000DBA80290DAA801900094DDA80D4602F006
:1064100043FE29462488DA9E099D68E011910F9871
:10642000208000273D46109705E00E9804887F1CC9
:10643000B8B2A04211D8B8B28000DDA90C582046ED
:106440001199FAF7D7F90028EFD1002DEDD10C986A
:10645000078001250F971094E7E7DBA805800F9AC6
:1064600090B2201A012811D10C9804800D9FDA9760
:106470003E46099D3AE04920C043864200DA8BE05F
:10648000FF2208469105F9F799FFA9E710200B991B
:106490000E5E012E00DA90E0551CABB21846A1B298
:1064A000AAB28A4217D805E00E990C88A1B2AAB206
:1064B0008A4210D88000DDA90C58204610991F464A
:1064C000FAF78AF93B46002805D10C9805800B980D
:1064D000068A0F95109430B2C1186D1CA8B2814283
:1064E000E2DC109EDA960F9C099D0D9F11993046B3
:1064F000F9F7A1FFFAF7D6F9052800D3052095A9E9
:106500000880A0B20E990988814218D9401C611EEA
:106510000CB2A04218DA12A898A9FEF76DFE0E98E8
:106520000188481C491E0CB2A04221DA12A899A980
:10653000FEF762FE99999898099D0D9FA4E60021A7
:106540009891999108469FE60022134608E09CB274
:10655000A40012AF3D515B1C491C0CB2A042DADB17
:106560008DB20A2D1546F2D8A400DDAD2D59EEE707
:106570000022134608E09CB2A40012AF3D515B1C00
:10658000491C0CB2A042D1DB8DB20A2D1546F2D8BF
:10659000A400DDAD2D59EEE75320C043864200DB59
:1065A0001BE70E460B9881692046FAF715F900287B
:1065B0000C9C08D10B98808B07E01446099D0D9F19
:1065C0001199109E93E70B98C08BFAF756F9014684
:1065D0003046F9F7F3FE119021E70000F0B58BB0DB
:1065E0001C4609930E46034600200A904048008846
:1065F000224F05970AA9049103940292109C0194DA
:10660000012500950B21414389B230331C4A3046A5
:10661000FFF74EFC3868079078680890B8680690D5
:1066200033480088334F009501940297324E30363C
:106630003249334A3346FEF76BFB0698F8620798F7
:10664000386308987863099800882E4905912E4987
:1066500004912E4903910297019000962C4B2846F5
:1066600029462A46FEF74CFC432001060A98F9F712
:10667000A5FEFAF717F90BB0F0BDC0469CA40102C5
:1066800060DC0102F0B589B00F9F0E9C002815D088
:106690001098079016480088164E01250095019124
:1066A00002960893144B30331449154AFEF730FB19
:1066B000089BF76207983063746303E00D484763F3
:1066C000C462002518880F4905910F4904910F49AC
:1066D0000391084902910190074830300090012150
:1066E0000B4B28460A46FEF70BFC09B0F0BDC0462E
:1066F00044AB010224D10102009E0102509D01021F
:10670000C8CF0102CCA1010240AB0102DCAA010208
:10671000E4AA0102304870470048704784AB010288
:10672000800037490918C86B0022CA637047C04609
:10673000800033490918886C00228A647047C0467B
:1067400080B52F4AD369002B01D0126A98470020E8
:1067500080BDC0460249087800220A707047C046D2
:10676000F4C601020020704780B5182905D80346F9
:106770008A1E03481946F9F7D7FC002080BDC046A1
:1067800048AB0102B0B502460020022901D2C04345
:10679000B0BD8C1E0F2C07D8044D2846114622464A
:1067A000F9F7C2FC00202855B0BDC04664AB010219
:1067B000B0B502460020022901D2C043B0BD8C1EF4
:1067C0000F2C07D8044D284611462246F9F7ACFC99
:1067D00000202855B0BDC04674AB010208490878B6
:1067E00000220A707047C046B0B50446044DAA683E
:1067F000002A02D0E968204690472C610020B0BDF5
:106800001897010280B5124801681F220A400260F1
:1068100003200840022812D10E480268D30D02D08E
:10682000FF231B06D2180C4B1A600C4A12680C4B43
:106830001A6080680B4A1080000C0B4A10801A48BE
:106840008268002A02D082680020904780BDC0463E
:106850007420004064400040DCCF010278300040EA
:10686000E0CF0102649E010216D1010280B50D48FD
:10687000016889070FD5052101600B48C1780029FF
:1068800008D00021C170C168002903D0C2684168E6
:106890000020904780BD054805A10B4A0BA307F0D7
:1068A0009BFAC0462C040040289401027E2B010074
:1068B0005048595F54494D45525F49525148616EA5
:1068C000646C6572000000008D0A0000556E6578EA
:1068D00070656374656420696E7465727275707436
:1068E0000000000070B50446401E012814D80320A3
:1068F000084011D13F2040030818050B28198028B3
:106900000AD8164E317801204840294603F01EFB74
:10691000641E6D1C002CF5D170BDC04680B50020F2
:10692000014603F05BF8002800D080BD0B48012130
:10693000017080BD70B516460C460546FF22F9F77A
:1069400005FC0548311805480278012050402A46C8
:10695000234603F0A3F970BD00E00704D4A60102AA
:10696000012000037047012040037047F0B583B059
:1069700030480068C16B0901890F01D003B0F0BD38
:10698000C16BC06B2C4D05404800400F0826029695
:1069900086400227384602F0C7F801907043C10BC9
:1069A0004A1B26485043F9F7ABFB044607F056F95B
:1069B000032123A238461F4F0091234608F068FAAE
:1069C000F88A002817D0019840012946F9F782FB80
:1069D00046431822324001200F2A014600D80021E8
:1069E00073095B181B4CA3420DD8194DED1A6D05A8
:1069F0000F2A0CD80CE038680021C160112002F089
:106A000083F803B0F0BD5D1C6D050F2A00D9564216
:106A10002A0C029D2E4009018919A34202D8009830
:106A2000000400E04004081880183968086303B0C7
:106A3000F0BDC046B8940102FFFF1F0040420F00A6
:106A400052434F33324B2070706D2025640D0A0085
:106A5000FF070000FE7F0000B0B582B0154908684E
:106A60008269D2070CD00122C2610D69002D07D0C6
:106A700000686C46214606F0E3FE00212046A84748
:106A800002B0B0BDB0B582B00A490868026C920786
:106A90000ED5026C012313430364CD68002D07D08B
:106AA00000686C46214606F0CBFE00212046A84730
:106AB00002B0B0BDB89401020648016803229143B8
:106AC0000160016801220A43026000F01BFB07F02D
:106AD000E7F8C0462800004080B50D490868002846
:106AE00010D5224802680423032A01D01A4300E08B
:106AF0001A460A601E490A68002A02D0416800202E
:106B0000904780BD03A00CA19E2211A307F064F959
:106B10002C100140696E636C7564652F6472697630
:106B20006572732F6D6B5F736C6565705F74696DF3
:106B300065722E6300000000534C4545505F544978
:106B40004D45525F49525148616E646C6572000058
:106B5000556E657870656374656420736C656570E7
:106B600020696E7465727275707400000C90010279
:106B70001CD10102B0B582B004460078002811D0C3
:106B8000094D01A908702868416A0029FCD101A9B2
:106B900001220020034608F011FF611C60780028E4
:106BA0000C46EED102B0B0BDD494010210B5CE4C6B
:106BB000216806290FD8012002468A4058210A423E
:106BC00009D020600020A0602369002B03D06269F7
:106BD000002002219847C3482258062A12D80121D2
:106BE0000B469340582213420CD02150201800210C
:106BF00081600369002B05D0AD20C0002258012020
:106C00000221984747482258062A11D801210B46ED
:106C10009340582213420BD021502018002181604C
:106C20000369002B04D003482258022001469847EC
:106C3000002010BDBC0A0000F0B581B0002402287D
:106C400003D9E443204601B0F0BD17460B46094E78
:106C5000464309488519284618302A2107A2FDF71E
:106C6000E5F842202F52032003498851204601B005
:106C7000F0BDC0465405000004AC010225730000BD
:106C8000F0B585B0E04D2C68002C0CD0DD4FDE4C0B
:106C9000E659002E0CD0234FE659002E0DD00020CF
:106CA000C04305B0F0BD01AC0FC400272E4608E07C
:106CB00001AE0FC6E619012703E001AE0FC6E619C3
:106CC0000227D04C30462146FCF796FF0220306068
:106CD0007C432919029D4D60CF6003980861049898
:106CE000486108464430CC31012256021023324616
:106CF000FDF73EF9E4480019B32189004118012D40
:106D000005D1B83001233246FCF757FD04E074305A
:106D100010233246FDF72CF901980760002005B0DA
:106D2000F0BDC046A80A000001460020022901D992
:106D3000C0437047E24A4A43E24988507047C04620
:106D4000022806D8E6494143E6484018024940185F
:106D500070474B2080007047D4040000022802D9FD
:106D60004B2080007047DE494143DE4840184D21EA
:106D7000090140587047C046032801DB03487047AB
:106D8000D7494143D7484018183070478B29010034
:106D9000022806DCD2494143D24840184221405AD9
:106DA000704700207047C046032801DB0020704771
:106DB000CB494143CB48401844307047022804DC9B
:106DC000C7494143C7484058704700207047C046F4
:106DD000022805DCC2494143C24840184068704758
:106DE00000207047B0B50024E14302280FD8BC4A08
:106DF0004243BC4B9D58042D09D0991801220A60CA
:106E00000B69002B05D04A690221984721460846A4
:106E1000B0BD2046B0BDC04610B50024022801D93F
:106E2000E04310BDAE494143AE4A072353505118C9
:106E30000B69002B03D04A6900242146984720465D
:106E400010BDC046F0B581B00024022803D9E44348
:106E5000204601B0F0BD0546A1486843A14906227D
:106E60000A500F18384644303946CC3101225602B8
:106E700010233246FDF77CF8786801280CD1B32046
:106E8000800039183846B83001233246FCF795FCAB
:106E90003B69002B0CD1DBE7B32080003918384662
:106EA000743010233246FDF763F83B69002BCFD0D6
:106EB0007A69012128469847204601B0F0BDC046B6
:106EC00010B50024022801D9E04310BD8449414394
:106ED000844A51180B69002B02D04A690321984754
:106EE000204610BD5405000004AC0102F0B583B08B
:106EF00017460024E24302281AD8002B18D00D466A
:106F0000774941437748461870680128029312D1A7
:106F1000002F0AD0B836002429193046FCF755FC5A
:106F2000002825D1641CA742F6D1029807600022F0
:106F3000104603B0F0BD019274363046FCF7D3FF23
:106F4000002811D003464268BA4209D2196828467F
:106F50001D46F9F7E9F82B46686802990860019424
:106F600030461946FCF795FF019A104603B0F0BD74
:106F7000029804600022104603B0F0BDF0B581B065
:106F800004460020C343022C02D9184601B0F0BDCC
:106F900015460E461B4A62431B498F187968012922
:106FA00010D1002D28D01C460090B8373846314605
:106FB000FCF7E4FB002821D1761C6D1EF6D1009869
:106FC00001B0F0BD0090743738462946FCF7A6FFA3
:106FD00000280CD00446006831462A46F9F7A4F888
:106FE00038462146FCF76AFF009801B0F0BD07A0C3
:106FF0002146FCF781FC009801B0F0BD204601B0AD
:10700000F0BDC0465405000004AC0102536F636B31
:1070100065745B25755D20526563762042756666F2
:1070200065722046756C6C0D0A000000F0B583B0E7
:10703000154607460022D043022F19D8002D17D03D
:1070400000AB07C30F4878430F490E18443630464B
:107050002946FCF763FF00280CD00446006801991C
:107060002A46F9F761F830462146FCF727FF0298D7
:1070700003B0F0BD05A03946FCF73EFC009803B014
:10708000F0BDC0465405000004AC0102736F636B91
:1070900065745B25645D2073656E6420627566208F
:1070A00066756C6C0D0A000002460020022A04DCA2
:1070B0000B4B53430B4AD1507047C0437047C046F7
:1070C0005405000004AC0102022801D900207047D9
:1070D0000349414303484018034940587047C0469C
:1070E0005405000004AC0102CC04000080B5044843
:1070F0000168491C01600069002800D0804780BDFC
:107100008CDC010201480249016070477490010261
:107110000026B80310B57B4800248460001D0121BF
:10712000024A2346FFF7ACFD204610BD1D72000049
:1071300070B5A0B0FDF792FA012814D1FCF70AFD52
:10714000224DA968022914D0002909D129780029E3
:107150002AD0E968411A062902D300212970E86083
:10716000002020B070BD194800218160002020B0AF
:1071700070BD2969421A16490E2A02D80A78002AD7
:10718000EED0286100200870124883886C46802168
:1071900011A2204609F026F9024668682146FFF749
:1071A00045FF002020B070BD0126AE60B102154C35
:1071B00015A22046FCF73AFE6868174A2146FFF7F9
:1071C0003BFD2E70002020B070BDC046E09501024E
:1071D00038930102D6A60102246D65737361676559
:1071E0002068656172742C253034782C3030303052
:1071F000312C312C35302C35302C35302C2C2C2C9E
:107200000D0A0000F0C201023131312E3139382E21
:1072100036302E3600000000D204000070B58EB06B
:10722000032925D87944097949008F4401091116A9
:107230003448816801291BD1002181600EB070BDE6
:1072400030488168012913D1022181600EB070BDE0
:107250002C48002181600EB070BD00250195294C9D
:1072600060682949294A01ABFFF740FE002801D098
:107270000EB070BD032026A2014607F009FE224889
:1072800026A10A22F8F785FF0028F1D11E482C21FB
:1072900002AA0C23FCF7DBFD0598FCF7B1FC608328
:1072A00080B2214EB1888142E2D10398FCF7A8FC5C
:1072B00060610528DCD8C0467844007940008744E6
:1072C0000213181C1C1C83480560A08B7083208C43
:1072D000F0822220215C7D20C000F8F7FBFEB08305
:1072E00006F04CFC0EB070BD7A480560758306F060
:1072F00045FC01200146FCF7BDF82220205CB0834C
:107300000EB070BDE0950102F0C20102FF03000063
:10731000CAD5B5BDCAFDBEDD0D0A000024696E7375
:1073200074727563742C0000D6A6010280B582B019
:107330000E4908680022C2600192CA68002A02D081
:10734000016801A8904702B080BDC04680B582B0F8
:10735000064908690022C26001220192CA69002A16
:1073600002D0016801A8904702B080BD10930102CD
:10737000F0B582B0144C2078009000281DD0134B3B
:1073800024330025019504E09B1C6D1C0098854268
:1073900015D262196026905D471C97550428F3D8D2
:1073A0000199C8B222181C8897554000074A101846
:1073B0008484054C491C0191E6E700200190019866
:1073C000207002B0F0BDC04608960102709701021D
:1073D00080B5002007F0AAFF80BD80B5012007F02E
:1073E000A5FF80BDF0B581B003F00EFB164CE06048
:1073F000A178002901D001B0F0BD21790029FAD18E
:107400000121217100281BD08D02281AA168814218
:1074100016D00E4E2F46A068305C21698847A068C0
:10742000401CA060681EA168814201DD0020A060B0
:10743000E168A068022F03D3691A7F1E8842EAD14F
:107440000020207101B0F0BDB095010288CB01028F
:10745000B0B5204C2068002807D0022810D00128A1
:1074600037D108F0CFFE00F087FB08F0A9FE2068B6
:1074700002281DD001282CD11A4800210180B0BD5E
:1074800015480078002817D014480021018008F022
:10749000B9FE00F039FC124D287008F091FE2878F2
:1074A0000028E4D0012020600E4800210180B0BDFA
:1074B0000948007800280AD10A4801884A1C02803D
:1074C000792904D3044901220A700021018008F0BF
:1074D0003FFCB0BDE4970102D0940102DC970102A9
:1074E000CB970102BCE4010280B5032810D8002923
:1074F0000ED07C224243BF488018C268012A07D1BF
:107500002030FCF762F9002801D00020C04380BD84
:107510000020C04380BDC046F0B589B00022D543ED
:10752000032800D9ABE00C46002900D1A7E0009564
:10753000216A0727534DA9420EDC574DA9421ADD97
:10754000564A91422FDC4B22D501A9423ED012026D
:1075500091424BD1042246E04B4A914217DD4B4AFF
:1075600091422ADCE1221203914231D0494A9142F0
:107570003CD10C2237E04B252E01B14233D06A01B9
:10758000914227D0AA01914230D102222BE0E12280
:107590005502A94220D09502A9421FD0D2029142A1
:1075A00024D109221FE04B225202914218D0E1223D
:1075B000120291421AD1062215E0E12252039142B1
:1075C00010D0334A914211D10D220CE003220AE07F
:1075D0000A2208E0012206E0072204E0082202E075
:1075E000052200E00B22D1002D4A57587C2141434F
:1075F000804A505056182068B0606068F060A168FA
:107600003161E268726100250595032304930395B7
:10761000029501970695079501231B0208930128FF
:1076200007D000280AD18818009A8018B161F0614B
:1076300004E0304620300123FCF7BFF82069706376
:107640006069B063E069B067A069F063706801A920
:1076500007F09EFF2068012806D8304640302346B8
:1076600010330ECBFCF784FC6068012807D1301D75
:107670007036006801220B4B314608F05DF8284651
:1076800009B0F0BDFFC10100FF0F0E00FF1F1C007D
:1076900080841E0040420F007F250000FF950000FF
:1076A000D80E010089F90000B0B50C467C21484392
:1076B000504A15182846FCF79FFA6C600020B0BDB0
:1076C000F0B583B00024E743032800D98EE00E46CE
:1076D000002900D18AE01546002A00D186E07C21ED
:1076E0004143444841188868022832D001283AD0E2
:1076F00000282BD1EFF31080C00702D1EFF31080E8
:1077000072B602910846403001902946FCF706FC0B
:10771000002863D0014601980F46FCF7CFFB38687C
:1077200031462A46F8F700FD0198FCF7DCFBEFF341
:107730001081C90703D1EFF3108172B662B60299C6
:107740004D6806C82C4B284608F038F9204603B08F
:10775000F0BD4868002431462A46234608F02EF939
:10776000204603B0F0BDEFF31080C00702D1EFF365
:10777000108072B602910846403001902946FCF70D
:10778000CDFB00281ED0014601980F46FCF796FB62
:10779000386831462A46F8F7C7FC0198FCF7A3FB86
:1077A000EFF31081C90703D1EFF3108172B662B60F
:1077B00002994D6806C8104B284608F0FFF820468D
:1077C00003B0F0BDEFF31080C0070FD1EFF31080CE
:1077D00072B662B63C46204603B0F0BDEFF31080AF
:1077E000C00703D1EFF3108072B662B63C46204664
:1077F00003B0F0BD00BC01028DFC0000B0B582B04A
:10780000602833D0622843D0642854D101A82F497E
:107810000180EFF3108072B600242046214602F06A
:10782000DDF82B4D002805D1012002030020294658
:1078300002F02EF8103501AA02232046294602F054
:1078400005FD62B623A0FFF795F964201B490C5291
:1078500006F094F91A4801F037FABFF34F8F194830
:1078600019490160BFF34F8F00BFFDE76020134946
:1078700000220A5206F082F9114801F025FABFF3FE
:107880004F8F104810490160BFF34F8F00BFFDE7D5
:1078900062200A4900220A520A8006F06FF908485D
:1078A00001F012FABFF34F8F064807490160BFF39A
:1078B0004F8F00BFFDE702B0B0BDC046D6A60102A3
:1078C000A08601000CED00E00400FA05AAAA000061
:1078D00000D00204BDF8C8EBC9FDBCB6C4A3CABD44
:1078E0000D0A0000F0B5D1B0944F3978002920D0AE
:1078F000F96808294AD88A0001A39A589746C046D1
:10790000257900008D7900008D7900009D790000B7
:10791000C7790000D3790000DD790000AB79000061
:10792000E7790000552800D0A6E00120F86051B0AA
:10793000F0BD83490978002900D191E0BA798649E0
:107940008854F979F8713972521CBA710A2800D03A
:1079500086E00D2900D083E003A8019037A80090AD
:107960003C4628347C487D491DAB2246F8F72EFC66
:1079700038617BA105222046F8F70BFC002840D097
:107980000020B861F861386278624BE0AA2869D1BA
:10799000012967D10220F86051B0F0BD0421F960DF
:1079A0000021F970B87051B0F0BD7979654A505432
:1079B000481C7871B978491FC0B2814250D1082063
:1079C000F86051B0F0BD0521F9605D49487051B0D3
:1079D000F0BD0621F960F87051B0F0BD0721F960E3
:1079E000787051B0F0BDB97806294AD34A1F0024F7
:1079F000544D23462E5D9B199BB2641C9442F9DBC7
:107A000040E01DA80024214609F0B5F9B861F961EC
:107A100037A8214609F0AFF93862796203A8F8F770
:107A200067FC7861504800F0BDFD7869002807D0F8
:107A30004E48002101704E48012202704D480180DD
:107A40001DA864242146F8F788FB37A82146F8F7DB
:107A500084FB03A82146F8F780FB00203872F880E9
:107A600051B0F0BD032807D1022905D1012038719A
:107A70000320F86051B0F0BD0020F860788051B06C
:107A8000F0BD0023181841182D4840780918FE78D9
:107A900089197C7809193A79002A00D0C91CC9B221
:107AA000FF2945D1012819D0022841D12748801942
:107AB000244D29462246F8F737FB2878012802D1C1
:107AC0003046FFF79BFE06F059F8BFF34F8F204872
:107AD00020490160BFF34F8F00BFFDE71A4DAC7125
:107AE00003202871A870AA2068705520287070089B
:107AF0006871661DEE70400014490918E81D2246A1
:107B0000F8F712FB281DE11CF2B2D21C037892B2E6
:107B1000D218401C491EF9D16019D143C171090A1C
:107B200001720934012000232946224607F046FF4E
:107B30000020F8607871788051B0F0BD989801020B
:107B40001890010224CB010248990102D6A6010235
:107B50000CED00E00400FA058CCA0102752001005A
:107B6000474E47474100000041AB010241900102EE
:107B70006D97010242AB0102F0B583B008F076FBCD
:107B8000E248E34903F088FCE24F0025BD7005F0B0
:107B9000CDF9B861042002F0BFFF584A28462946B3
:107BA00008F096FB03F0EAFB0028FBD105F0BEF9D4
:107BB0007861B878012870D1DA4C2078DA490978F0
:107BC000814200D091E0607A202800D08DE0607979
:107BD000A17909020818D549498B884200D084E070
:107BE00005F0A4F97861A07A787002460190607976
:107BF000A17909020E18BE800B3452000292CC48C3
:107C00002146F8F791FA029AC64811180B31C84874
:107C10003230F8F789FA0198002863D00094C548FB
:107C2000006802900022019DC1490EE029186023DE
:107C30000027CF542F464000BF49081886842C6285
:107C4000019DBB49521CAA4232D050000B5A029CE3
:107C50009C42F7D108183223C45E3D463B78002B86
:107C60000ED0B54F243700203988B1420DD0BF1C4B
:107C7000401C8342F8D11F461846172B08D9D5E778
:107C800000273846172B03D9D0E7C7B2172BCDD81A
:107C90009F42CBD1591C2970C8E7194801784A1C6A
:107CA0000270152921D3174902220A6005701CE0D1
:107CB000002D0ED09F4801680020009C2278637838
:107CC0001B029A18914206D0A41C401C8542F5D193
:107CD00008E0002506E0C4B22046FBF7C7F97D782E
:107CE000A54202D12846FBF7C1F9944805F0BAFF36
:107CF000042002F001FF03B0F0BDC046881300006D
:107D00001AD00102E4970102F0B585B008F0AEFA8E
:107D10007B4C607808F050F87A498A8803A8828002
:107D20000A88498809048918039104F079F8607871
:107D3000052804D002227449092804D104E0012254
:107D40007149092800D0891849792078621C08F007
:107D5000F7F8607A05F07AFB6C486D4903F09CFBFC
:107D60006C4F0025BD7005F0E1F8B861042002F009
:107D7000D3FE694E28462946324608F0A9FA05F096
:107D8000D5F86649386379634118481C00D0084625
:107D9000B863F96B814204D3614A8018814200D8EC
:107DA0009FE0604C00E0F86303F0E8FA054605F058
:107DB000BDF8002DF7D17861B87801280FD120786F
:107DC0005949097881420AD1607A202807D160791F
:107DD000A179090208185549498B88420ED000251F
:107DE00028462946324608F073FAB96BF86B884288
:107DF000DAD34B4A89188842D6D872E005F096F853
:107E00007861A07A7870024601906079A1790902C0
:107E10000E18BE8025460B35520002924448294672
:107E2000F8F782F9029A1119019C0B31404832305F
:107E3000F8F77AF9002C4CD000953E480068029083
:107E400000223B4B0DE0391860230024CC54400045
:107E50003949081886843D62019C354B521CA24268
:107E600026D05000195A029D8D42F7D118183221A0
:107E7000455E3B78002B0ED02F49243100200C8822
:107E8000B4420DD0891C401C8342F8D119461846D3
:107E9000172B08D9D7E700210846172B03D9D2E7BB
:107EA000C1B2172BCFD89942CDD1591C3970CAE72E
:107EB000002C0ED01F4801680020009D2A786B78A6
:107EC0001B029A18914212D0AD1C401C8442F5D17D
:107ED00000E000242046FBF7C9F8184805F0C2FE70
:107EE0000125042002F008FE284605B0F0BDC5B209
:107EF0002846FBF7BBF87C78AC42EED1EAE7C046F7
:107F0000BA900102AC0E0100689E0102A1F00000CF
:107F1000DDDA00000896010280841E000098E00E61
:107F20000026B8031CD00102CA970102D6A601029E
:107F300030980102EC970102709701027C3F00002B
:107F400080B582B0002001900448C268002A02D0A7
:107F500001A80021904702B080BDC046649501028F
:107F6000F0B583B000242046FEF7D8FCFEF7FBFCFA
:107F7000274EB060FEF7F4FC7060264F0BE001A8BE
:107F8000C1888088084319D101A840882418083482
:107F9000B068844235D201AD082128462246FEF75A
:107FA000C9FC28880028EAD0B8422AD001AD0421B3
:107FB000284600F073FEA9888842E5D03460B06896
:107FC00084420CD201AD022128462246FEF7B2FCC3
:107FD0002888B84203D0A41CB0688442F2D37068E9
:107FE0002118491E4042084030600DD0002425462B
:107FF00001202946FEF776FC03CE4D19083E854246
:10800000F6D3346003B0F0BD0024346003B0F0BD9B
:1080100084960102FFFF0000F0B585B01F46049270
:108020000646C8170C1844400A2C039114D30125A6
:108030000A212046F8F74EF86D1C632C0446F7D849
:1080400004998D4200D329460A9C002F09D0039839
:10805000002808D4002207E0012504998D42F2D2BD
:10806000F2E7002205E00122042323409B0813438A
:10807000FA1A0223234004980028029412D1002BFC
:1080800010D0F468002C62D40398002825D40298FC
:10809000400734D57068B5686F1C87422FD83068A8
:1080A0002B2423E0E407ECD1002A0AD1E9E7376862
:1080B00020203855B560F068441CF460521E002C36
:1080C000DFD49142DDD27768B468651CBD42EED939
:1080D000F468521E002CF4D5D3E740420390706838
:1080E000B5686F1C87420AD830682D244455B760A4
:1080F000F068441CF4600025ED43A84227DB002B08
:108100001CD00120029B1840049B184316D1002A62
:1081100003D113E0521E002C0ED491420CD2706891
:10812000B3685D1C8542F5D830683024C454B5600E
:10813000F068441CF460EDE7002C08D4009202982B
:1081400001900A2230460399049B00F003F805B021
:10815000F0BD0000F0B587B01F461546029001241F
:1081600006919142009407D3012406982946F7F717
:10817000B1FF641CA842F9D20D980C9ABC42039737
:1081800000D3039400990140002A009109D00029EE
:10819000029C25D12021800705D40846002F11D04C
:1081A00004E0029C1CE03020002F0BD0084609E0C0
:1081B00023685854A260E168491CE1603246721E8F
:1081C00000290DD4039991420AD216466368A1682A
:1081D0004A1C9A42ECD9E1683246721E0029F1D558
:1081E000E068002859D40590012401E07F1E6C430B
:1081F000022FFBD2069821461646F7F76BFF324650
:10820000A842F4D2029880680490069F01950697D0
:1082100038462146F7F75EFF049D691C029F7A6885
:10822000914206D9069F059A019D0592002A0ED516
:1082300016E01B4A125C3B685A55B960FA68521C3A
:10824000FA600491069F019D0592002A08D46043BC
:108250003F1A20462946F7F73DFFAC420446D6D2E6
:1082600000980028029C059B049D16D0002E14D077
:10827000701C01E0002B10D4401E039981420CD2E7
:10828000691C62689142F5D8226820235355A16089
:10829000E268531CE3600D46ECE707B0F0BDC04652
:1082A000B4110100F0B583B001900291002923D0F0
:1082B0000025164F2E460AE017480818410F4018AF
:1082C000C010B871761CB1B2029A914216D20198D0
:1082D00000884B24210100B200F02CF8400061011D
:1082E0004018F88201B20A4881422846E9DB094871
:1082F0008142E1DD6420E4E704488079C3B20320D1
:1083000006A2014606F0C4FD03B0F0BDC897010205
:10831000E40C0000041000001CF3FFFF546865200B
:10832000766F6C746167652069732025252564204C
:108330000D0A0000074A904201DD054A801800B28C
:108340004143C817400D0818C00A00B27047C04624
:1083500000F0FFFFFF07000010B50078012819D1D9
:1083600061480269012A04D1624A13680124A343C7
:108370001360032905D080214161C269002A05D11B
:1083800007E001214161C269002A02D001898069A8
:10839000904710BDFF222E32024803A107A305F02B
:1083A0001BFDC046681D01006164635F646D615F11
:1083B00063616C6C6261636B00000000556E6578F0
:1083C00070656374656420646D61206368616E6EBE
:1083D000656C0D0A00000000F0B58DB00D4601245B
:1083E000EFF31081214002D1EFF3108372B63E4EBD
:1083F00073690F2B06DD102B37D0402B2FD0802B2D
:108400002DD005E0002B2AD0012B01D11023736160
:10841000B5813581B061F261002900D162B6317950
:10842000002929D00294314C05A90A4604950390ED
:10843000E8CCE8C2E8CCE8C2029C204600F0B4FCDC
:108440002B4800902B4D294608312046039A049B67
:1084500000F01AFD2C60002420460DB0F0BD00296C
:10846000FAD162B620460DB0F0BD02240029F3D146
:1084700062B620460DB0F0BD3178002907D01D4806
:10848000072181610460002420460DB0F0BD3269EF
:10849000B3891849002B15D0B5693089012A02D05B
:1084A000002A03D003E09FB2874200D10C604F68DE
:1084B000FF07FCD08F6880C55B1E1F04EED1002330
:1084C000B381B561012A02D10A68A2430A607461CE
:1084D000F2690024002ABFD0B36931898800181AD4
:1084E000904720460DB0F0BD78950102F4110100CF
:1084F0005983000008D0014070B5002801D0012048
:1085000070BD0C461625284600F006FB284605F0EF
:1085100089F9002C05D01B48183014222146F7F7A2
:1085200003FE28211748415C002915D04168002925
:1085300016D403220B469343144A9C588D07ED0E24
:10854000FF26AE40B4439C501F220A4001219140B7
:108550000F4A11600F4A116001210161002070BDB6
:108560008A07D20EFF2393400F220A40083A0321C4
:108570008A43054954589C4354500121016100200D
:1085800070BDC046789001021CED00E000E400E000
:1085900080E200E000E100E05A21014A50527047B9
:1085A000009E0102F0B581B004460078414241418D
:1085B000217024480078C0012349097889010143CA
:1085C0002248007840010843214909780901014304
:1085D00020480078C00008431F4F397889000143C4
:1085E0001E4D2878400008431D4E31780143C8B223
:1085F000FBF72AFF642000F067FB207841424141ED
:10860000217010480078C0010F49097889010143A1
:108610000E480078400108430D49097809010143DB
:108620000C480078C0000843397889000143287855
:108630004000084331780143C8B2FBF705FF01B0A1
:10864000F0BDC0464C9D01026E97010220940102CC
:10865000BEE4010241AB01024D9D0102C8A001022E
:10866000C9A00102B0B5504D68600B24002120461E
:108670000A4602F059FA01210522204602F0E8FAE2
:108680006A680321204602F0C7F9B0BDB0B5094DB4
:1086900028600224002120460A4602F045FA012102
:1086A0000522204602F0D4FA2A680321204602F06F
:1086B000B3F9B0BD489D01025C21AA480022425294
:1086C00082847A2141840284C2830283C28202822C
:1086D000114941608260C2603D2149044183418269
:1086E000090C8183818270475C219E48002242529E
:1086F00082847A2141840284C2830283C2820282FC
:10870000054941608260C2603D2149044183418244
:10871000090C8183818270474C37373770B5924896
:108720004C21016001252C02601C00F075F93220FB
:1087300000F0CAFA00F05EF9284600F065F9284614
:1087400000F074F800F050F90C4800F065F90026CC
:108750003046314600F070FA2846314600F06CFA97
:10876000204600F059F9022000F056F9483420461E
:1087700005F0AAFA05F008FB70BDC0460102000032
:1087800010B50446072106F0E1F907480460032408
:1087900006A22046214606F07BFB0AA20F4B20468C
:1087A000214606F075FB10BDD895010248656C6C3A
:1087B0006F2066726F6D204D4B53454D49210D0A58
:1087C000000000004275696C6420696E666F726D0E
:1087D0006174696F6E2025730D0A0000483D010029
:1087E00010B505200424214602F00AFA062021468D
:1087F00002F006FA0E20214602F002FA0D20214670
:1088000002F0FEF900240121204602F0F9F90221CC
:108810002046224602F01CFA10BD00000248016802
:1088200001229143016070475800004002490A68E4
:1088300002408242FBD1704704600040B0B5494D10
:1088400028688107484C0ED528797F210840226886
:108850008A431018206023680B4002200321434AFA
:1088600006F016FB286880040ED55E20285C7F2168
:10887000084062688A431018606063680B400220F9
:1088800003213B4A06F004FB172000F045F9394864
:10889000016802220A4301218A43026036483749AF
:1088A000016037480021C17181791F2529408171FC
:1088B000817A427C837C1B029A18C37C1B04D218E9
:1088C000037D1B06D2182F4B9A4218D1427B837B23
:1088D0001B029A18C37B1B04D218037C1B06D218F8
:1088E000294B9A420BD1C27A037B491E122906D822
:1088F00019028918254A914201D12021017201787B
:10890000CA0602D11022114301701C3C20682021AC
:10891000884320601E481F49016041680029FCD53A
:1089200003F0EAF90446022003211BA2234606F0C5
:10893000AFFA0A20C441032C05D8022003211DA24E
:1089400006F0A6FAFEE71848C1680F229143C160FD
:108950000168164A0A400260192000011449486063
:108960000D60B0BD689E010248000040B01D0100CE
:108970009A1D0100040200400C060040AF6B100A73
:108980006B0001404D383650312E3236073400002E
:1089900000600040FE1C0080436869702049443A32
:1089A00020253038780D0A00C8600040FEFFC3FF64
:1089B0000C0400404F6C642063686970206D6F6424
:1089C000656C206973206E6F7420737570706F72A0
:1089D00074656420627920746869732053444B2164
:1089E00021210D0A0000000080B5172000F08CF84E
:1089F000002080BD10B51724204600F08DF82046D9
:108A000004F010FF002010BD0121C90701430148F7
:108A1000016070470060004010B5C1B2000AC2B2E8
:108A200002290CD0012913D0002930D1911E7F4892
:108A300002291BD20121032A2AD0490429E07B48BC
:108A40004168002A1FD00246203A1143416010BD00
:108A500076480168D31E022B10D3012A29D0002AA0
:108A600041D1012292079143016010BD002A16D125
:108A70000121490702688A43026010BD0123042ACC
:108A80001FD05A041EE0012292079143416010BD9D
:108A90000904194A7F32C36A13405918C162174941
:108AA0008A699207FCD50121490702680A430260DE
:108AB00010BD0522120791430246203A0A43026084
:108AC00010BD1A04836A0C4C1C40A21882620B4A27
:108AD000131F00241C600A4B0A4C1C600D235B0210
:108AE00014681C431460054A93695B06FCD5052293
:108AF00012071143016010BD80FFFCFF140200400B
:108B000004010040FF0F0000012181404748026836
:108B10008A4302607047C046012181404348026891
:108B20000A4302607047C04610B5052811D8C046F8
:108B30007844007940008744020E192434393B49B7
:108B40000A680868C0003CD53A4820390A425DD01E
:108B50003BE0002010BD35490A680868C00035D5E3
:108B600034480B46203B1A4237D134E02F490A687B
:108B70000868C00036D52F480B46203B1A424CD11E
:108B800035E02A494C680120C0030A680B46203BA7
:108B90001C421AD00C68E4003BD5264C1A423CD04B
:108BA0003AE0224800680120C00310BD1F490A684E
:108BB0000868C0001ED51F480B46203B1A4220D132
:108BC0001DE01B4820390A4220D010BD18480B4632
:108BD000203B1A4201D10120C00349688900890F56
:108BE000C84010BD12480B46203B1A4215D1012047
:108BF000C00312E00E480B46203B1A4201D101206F
:108C0000C00349680903890FC84010BD0120C00393
:108C100010BD074C1A4200D020464A689200920FBD
:108C2000D04049680901890FC84010BD20000040AC
:108C3000006CDC020026B80304282CD8164AC04673
:108C40007844007940008744020A121A2100032068
:108C50000007136883438807800818181AE0032068
:108C600080061368834388070009181812E0032060
:108C70008004136883438807000B18180AE0FF205C
:108C80000002136883430802181803E01068FF23EA
:108C9000984340181060704724000040B0B500228F
:108CA00000290CD0074B047895B22D0A65406C0062
:108CB0001C5B12026240491E401C0029F3D190B295
:108CC000B0BDC046B40F010000280AD030B407255B
:108CD0002C02CD256419604340091238001FFDD8CD
:108CE00030BC7047F0B583B01F4616460D460146AE
:108CF000E8680291F7F762FB04460F2E11D8082EA0
:108D000004D320462146F7F700FB09E0042E02D3E6
:108D10008120C10501E0412001062046F7F74EFB06
:108D200004460999089E2B20C043874205DB204654
:108D30000F462146F7F7E9FA0DE03F20C04387428E
:108D40000BDA4920C04387420CDBFF200F46810528
:108D50002046F7F733FB39460446688A08803460BA
:108D600003B0F0BD01915320C043874206DB20468B
:108D70002146F7F7CAFA0446688A10E0A869029902
:108D8000F7F746FD002801D1A88B00E0E88BF7F744
:108D900074FD01462046F7F711FB044600200199B7
:108DA0000880346003B0F0BDF0B581B00546012005
:108DB000072D66D80C46002963D04A4F38680169F0
:108DC000C90736D105263046FFF7A6FE304604F027
:108DD00029FD03CF0369012213430361002918D43D
:108DE00003200B4683438E481E588807C00EFF277A
:108DF0008740BE4340278740374389481F501F2084
:108E00000840824087480260874802603548006811
:108E10000FE08A07D20EFF2696400F230B40083B37
:108E200003218B437D495F58B743402696403E431C
:108E30005E5069014018012109024218E369DB060E
:108E40009B0CA569ED00EDB2EB1853606268520708
:108E5000520B23685B075B099A18A3685B079B0C9E
:108E6000D218E3685B075B0DD21823695B01DBB2A4
:108E7000D21863699B07DB0ED2188023134343503B
:108E8000002001B0F0BDC046F0B581B0002A23D06B
:108E900005460835134C2668F668EE40F50702D003
:108EA000022001B0F0BD069D8600A619B560400104
:108EB00024682018009301231D02461977680724AF
:108EC000A7437760F16032610099B160415919435D
:108ED0004151002001B0F0BD03A00AA174220DA3EE
:108EE00004F07AFFC8920102696E636C7564652FA5
:108EF000647269766572732F6D6B5F646D612E634A
:108F000000000000646D615F7472616E736665726B
:108F100000000000496E76616C6964207472616EB5
:108F2000736665722064737420616464720000006B
:108F300000015849085840687047C046F0B581B0F4
:108F400005460120012D4CD80C46002949D0002DA2
:108F500003D0012D04D10F2000E00E20FFF7DCFD2F
:108F6000A668012E04D0002E4FD1E08900284CD1F4
:108F70002901294843580020D860F507AD0F27681C
:108F80006668B607360F76192569EA07920EB61895
:108F9000022F04D0012F03D10122164300E04036F6
:108FA0001D4F9E60E2681A6079188D606269CA6020
:108FB0004968002917D403220B469343184A9C584A
:108FC0008D07ED0EFF26AE40B4438026AE4026430B
:108FD0009E501F220A4001219140124A1160124AFC
:108FE000116001B0F0BD8A07D20EFF2494400F2318
:108FF0000B40083B03218B4308495D58A54380245F
:1090000094402C435C5001B0F0BD08A00FA1492250
:1090100012A304F0E1FEC046109301021CED00E033
:1090200000E400E080E200E000E100E0696E636CD3
:109030007564652F647269766572732F6D6B5F64FA
:1090400075616C5F74696D65722E63006475616C27
:109050005F74696D65725F6F70656E00636F6E66D9
:10906000696720697320696E76616C69640000002D
:109070000001084A10580160816880220A4382601A
:109080007047C04600010349085881688022914317
:109090008160704710930102F0B58DB001931546C1
:1090A0000E460A901298002408900480149F3C8079
:1090B000139809900460159804900480FF2081059E
:1090C0003046F7F77BF90290304603963146F7F7C2
:1090D0001CF92B463D460690274607950B9311E059
:1090E0001180188880002858099908600120079D80
:1090F00028800520049908807F1CBCB2188884420F
:1091000000D9A0E028880028F6D1A0000A9D2E589A
:1091100030460699F7F76EFB002817D030460399C2
:10912000F7F768FB00280B9B079DE5D1089A17808D
:10913000099D2E601888011B012934D110801988DF
:1091400089000A9A51582960059035E0089A1780DD
:10915000099806600B9B1988081B0128C0D00C9643
:10916000019825187E1CB0B28542BFD389B2B2B235
:109170008A420ED880000A990C5820460C99F7F7BD
:109180002BFB0B9B002804D10998046008980680EB
:109190000C94761CB0B28542A8D3198889B2B2B2B9
:1091A0008A42E7D9F5E70C96019962187D1CA9B2AD
:1091B00016468A4205972CD2059884B2A5000A9ECD
:1091C0007259002C104609D0A819001F01681046DA
:1091D0000C92F7F79AF80C9A062C07D80446A819AF
:1091E00041681046F7F791F80C902046079D0299C8
:1091F000F7F70EFB00280B9B07D10C980299F7F7A5
:10920000F9FA0B9B002800D076E701202880032084
:1092100070E780B2AAB282420FD888000A990C582F
:1092200020460C99F7F7D8FA0B9B002805D109982E
:1092300004600898058005950C946D1CA9B28E42B7
:10924000BAD31888E5E70DB0F0BD00000A490A68F6
:109250000A4802400A60FD214900094A1268515C2F
:10926000002908D007490A6C02400A640120000660
:109270000A6882430A60704700040040FFFFFF7FD6
:10928000389401022000004000207047F0B583B000
:109290000D4604467C26464350488719F869396ACA
:1092A000F6F718FFA84200D892E001950294012138
:1092B000EFF31080084002D1EFF3108272B63C4603
:1092C00010343B690025062B0CD80A469A40D30679
:1092D0005B0F06D161231A4275D00D46002803D0DA
:1092E00003E00225002800D162B6002D02D02846F6
:1092F00003B0F0BD00943C4620343848805910211A
:10930000C1613E46143604F039FD05463868C0692F
:10931000C00605D504F032FD401B31888842F5D9DE
:109320000621029D284600F00BFF20680199414369
:10933000B869091838688160172179563C46173496
:10934000002909D5C16920220A43C2610121F966B9
:10935000890502680A4302600521284600F0F0FEF4
:10936000207840B200250028C1D42B4800687D2415
:10937000E100F6F7AFFE61014143029800F0B2FE52
:1093800004F0FCFC04463868C069C00705D004F04E
:10939000F5FC001B31888842F5D904F0EFFC044647
:1093A0003868C169890706D504F0E8FC001B3188DC
:1093B0008842F5D938680121009A116053498161CA
:1093C000284603B0F0BD0321216000288CD08CE733
:1093D000034804A1084A09A304F0FEFC3C930102DF
:1093E000E01D0100666C6173685F626C6F636B5FA8
:1093F00065726173650000005D020000626C6F635E
:109400006B20696478206973206F766572207261C1
:109410006E67650D0A000000A0DC0102F0B583B0A4
:1094200002907C214143934A5418E56EEAB2511EE2
:1094300002291FD229040126090E18D00196009294
:10944000022100F07DFE2746143704F097FC064603
:109450002068C169890606D404F090FC801B398815
:109460008842F5D92068007DC007019E08D03046AB
:1094700003B0F0BD032A36D100922804000E36D086
:1094800020466C302D0C00210191016027461437D5
:1094900004F074FC06462068C069C00705D004F0DB
:1094A0006DFC801B39888842F5D904F067FC0646BC
:1094B0002068C169890706D504F060FC801B3988E3
:1094C0008842F5D9206811498161E9B2012000295B
:1094D00011D003290099019E00D006202061226F3F
:1094E000002A0ED1C3E70026304603B0F0BD0126A6
:1094F000304603B0F0BD0099019E2061226F002A22
:10950000B5D002A89047304603B0F0BD000093EB01
:1095100070B5002801D0012070BD7825CD4E705D5A
:1095200000280ED000240921204600F009FE0F205B
:10953000FFF7CAFB1520FFF7E7FA745534612046A0
:1095400070BD042070BDC046F0B581B00C460078F7
:10955000484EF16881422CD1032C54D1706EB16E0B
:10956000884261D900240621204600F0E9FD3068D8
:10957000F16D81602046214600F0E2FD3546603500
:109580002CCDF0683168B48C414F00975B1BA3422F
:1095900000D81C46A3081431FFF776FCB06E001902
:1095A000B066306E00193066F06D0019F06501B0DC
:1095B000F0BDB168814255D1032C45D1F08CF16DDD
:1095C0000918F165316E09183166B16E0818B06678
:1095D000716E814238D900240621204600F0B0FD8A
:1095E0003068F16D81600121204600F0A9FD316EE7
:1095F000B068F38C3268264C009414329B08FFF755
:1096000043FC01B0F0BD30681021C16104F0B6FB2D
:1096100005463068C069C00616D504F0AFFB401B94
:10962000B18A8842F5D90FE030681021C16104F099
:10963000A5FB05463068C069C00605D504F09EFB51
:10964000401BB18A8842F5D90120C10732681368EE
:109650008B431360F16E22040A4300021043F0664C
:1096600001B0F0BD4D200201034804A1844B04F079
:10967000B3FBC0463C930102E01D0100666C6173C0
:10968000685F646D615F63616C6C6261636B000055
:1096900049950000F0B581B000786E4DAA6882420D
:1096A00000D0D0E001263002032942D16A6DAA66BB
:1096B000AB6DAC6AA418EB652C66AB6C5B1CAB6441
:1096C0006B6E934235D95E30FFF7FEFA686CA96C79
:1096D00002293AD3814238D1E88C696D081868654F
:1096E0000020062100F02CFD2868E96D81602F6DB7
:1096F00004F044FB04462868C069C00705D004F0A4
:109700003DFB001BA98A8842F5D904F037FB0446CB
:109710002A68D069800706D504F030FB001BA98AAF
:109720008842F5D92A687420285C012841D0F104C8
:1097300040E0F2072B681C6894431C60EA6E090441
:1097400011430143E96601B0F0BD0229FBD3814218
:10975000F9D2E88C696D09186965A96D0818A865C2
:109760000020062100F0ECFC2868E96D8160EF8C98
:1097700004F004FB04462868C069C00705D004F063
:10978000FDFA001BA98A8842F5D904F0F7FA0446CD
:109790002A68D069800706D504F0F0FA001BA98A70
:1097A0008842F5D92A687420285C012822D0F10467
:1097B00021E03105334B3B405918012802D01920D4
:1097C000400601E00720C00608182F4940185060E5
:1097D000002F0DD004F0D2FA04462A68D069800721
:1097E00006D404F0CBFA001BA98A8842F5D92A686E
:1097F0002B6D1FE03105234B3B40C918012802D0D7
:109800001920400601E00720C00608181E4940182C
:109810005060002F0DD004F0B1FA04462A68D069D8
:10982000800706D404F0AAFA001BA98A8842F5D959
:109830002A68EB8C296EA868144C00941432FFF748
:1098400023FB01B0F0BD044804A10C4A0C4B04F00A
:10985000C3FAC0463C930102E01D0100666C6173CF
:10986000685F646D615F77726974655F6E62797459
:1098700065735F63616C6C6261636B00720400000E
:10988000C71D0100FF3F000000808000959600008A
:10989000F0B587B004460126880E14D01546002A7C
:1098A00011D00F468120C004401B88420BD37C207E
:1098B0006043F04908180590818C38460691F6F708
:1098C00009FC002902D0304607B0F0BD28460699B1
:1098D000F6F700FC0029F6D1059880693E1A30465B
:1098E0000699F6F7F7FB0746039670190190069E56
:1098F0003146F6F7EFFB0546C01B04900598006A59
:1099000002903146F6F7E6FB049981420FD2002619
:10991000BD42D8D92046394600F018FB2046FFF753
:109920007DFD0028FAD17F1CAF42F3D3CBE7009036
:109930000398029D2946F6F7CDFB0646284670435C
:109940000399081A019800D0761C2946009D75439A
:10995000F6F7C0FB0590029941430198401A039025
:109960000699F6F7B7FB0490AF420BD22046394672
:1099700000F0ECFA2046FFF751FD0028FAD17F1CD9
:10998000AF42F3D305988642069D009F0CD2204635
:109990003146FFF77BFC2046FFF740FD0028FAD157
:1099A000761C05988642F2D30398A84203D200267B
:1099B000304607B0F0BD059847430025E919204619
:1099C00000F0C4FA2046FFF729FD0028FAD16D1CEB
:1099D000002604988542F1D375E7C046F0B585B0FE
:1099E000002803D00124204605B0F0BD7822A14F05
:1099F000B85C002803D00024204605B0F0BD0492D6
:109A0000002905D0384614300CC90CC01CC91CC034
:109A10000020F86615242046FFF77EF8204603F064
:109A200001FF38681021C16104F0A8F904463868C4
:109A3000C169C90607D504F0A1F9001BB98A88429B
:109A4000F5D9386800E0B98ABA7D1207120B5218AE
:109A5000F97DCB07DB08D2188B07DB0F5B05D2182B
:109A6000CB06DB0FDB05D2184B07DB0FDB06D2186A
:109A70008B06DB0F5B07D2180907C90F8907114353
:109A8000016000240A21204600F05AFB3220FFF733
:109A90001BF90821204600F053FB04F06FF905463E
:109AA0003868C169890606D404F068F9401BB98A90
:109AB0008842F5D93868017D0A46C23A534253417B
:109AC00074257B550904027D12025118007D0B1884
:109AD0000220032668A2314605F0DAF9785D0128F4
:109AE000039619D1F87D029000260621304600F039
:109AF00027FB0721304600F023FB01210298814318
:109B0000785D012847D1386889010175067575218E
:109B1000795C012938D048E00020032100F010FBD7
:109B200004F02CF906463868C169890606D404F0A9
:109B300025F9801BB98A8842F5D93868007D460826
:109B40000122F87D014631431640C90701D030405B
:109B500036D00295002506212846019200F0F0FA41
:109B600007210095284600F0EBFA0198464002983C
:109B7000385C012813D13868B1010175009901756D
:109B80007521795C012910D114307621795C4A4223
:109B90004A41510008E038680675490003E038681A
:109BA00000990175710014300170374800687D21FB
:109BB000C900F6F78FFA28214143002000F092FAFD
:109BC0007720385C012803D102200021FFF734F808
:109BD00004F0D4F806463868C069C00705D004F020
:109BE000CDF8801BB98A8842F5D904F0C7F806463B
:109BF0003868C169890706D504F0C0F8801BB98AA6
:109C00008842F5D93868D049816117203856002834
:109C100029D57868002816D40146039A91431C4A36
:109C20008B588507ED0EFF26AE40B3438026AE402D
:109C30001E438E501F2101400120884015490860B5
:109C4000154908600FE08107C90EFF228A400F23E3
:109C50000340083B039883430C481D5895438022DA
:109C60008A402A431A5001200499785438612046CA
:109C700005B0F0BD3C9301026A656465635F696489
:109C80002025780D0A000000A0DC01021CED00E098
:109C900000E400E080E200E000E100E0F0B593B015
:109CA0007C270A9047439348C619980704D0F07D53
:109CB0004024044000D017E10125880E2ED0002B4F
:109CC0002CD08120C004C01A884227D309920122D7
:109CD000EFF31084144002D1EFF3108072B63046D7
:109CE000103005903069002506280891069310D899
:109CF000079414468440E106490F04D161210C42C7
:109D000003D0154604E0022502E00221059B1960FC
:109D1000079C002C00D162B6002D02D0284613B05B
:109D2000F0BD344617347348C05910210491C16105
:109D30003746143704F022F805463068C069C0067B
:109D400005D504F01BF8401B39888842F5D92078E6
:109D5000400665D40297B78C069C20463946F6F734
:109D6000B9F9079039464143601A039035462435C6
:109D7000A74200D894E0039800281CD006210A9C32
:109D8000204600F0DDF928880799484308994018D3
:109D90003168886000272046039C394600F0D0F9DE
:109DA000079B099A28885843C0193168097D1154C6
:109DB0007F1CA742F6D330680499C16103F0DEFF2F
:109DC0000446029D3068C069C00605D503F0D6FF81
:109DD000001B29888842F5D903F0D0FF044630687B
:109DE000C069C00705D003F0C9FF001B298888425D
:109DF000F5D903F0C3FF04463068C169890706D569
:109E000003F0BCFF001B29888842F5D93068012186
:109E1000059A1160B24981610025284613B0F0BD52
:109E200003200025089FF765099931660699716638
:109E3000B566F0660120C00731680A6802430A600F
:109E400006210A9C204600F07BF930688760204696
:109E5000294600F075F93A4F0BAA0A921BCF1BC294
:109E60001BCF1BC2B48CF0680A99FEF79DFFF06807
:109E70003168344A0092069A944200D31446A308EB
:109E80001431099AFFF700F8B06E0019B066306E11
:109E900000193066F06D0019F065284613B0F0BD6A
:109EA000002404E0641C0798844200D363E7062181
:109EB0000A9800F045F928886043089940183168ED
:109EC000886000270A98394600F03AF92888002867
:109ED000099AE7D0604310183168097DC1557F1C8D
:109EE00028888742F6D3DDE7034804A1064A07A382
:109EF00003F072FF3C930102E01D0100666C617388
:109F0000685F726561640000C603000054686520E4
:109F1000444D412072656164206C656E67746820F1
:109F200073686F756C6420626520746865206D7558
:109F30006C7469706C65206F6620340D0A00000037
:109F40005412010049950000000093EBF0B583B076
:109F50000D4604467C26464351488719F869B98C5A
:109F6000F6F7B8F8A84200D894E0019502940121D0
:109F7000EFF31080084002D1EFF3108272B63C4636
:109F800010343B690025062B0CD80A469A40D306AC
:109F90005B0F06D161231A4277D00D46002803D00B
:109FA00003E00225002800D162B6002D02D0284629
:109FB00003B0F0BD00943C46243439488059102148
:109FC000C1613E46143603F0D9FE05463868C069C3
:109FD000C00605D503F0D2FE401B31888842F5D972
:109FE0000621029D284600F0ABF8208801994143E4
:109FF000B869091838688160172179563C461734CA
:10A00000002909D5C16920220A43C2610121F966EC
:10A01000890502680A4302600421284600F090F88E
:10A02000207840B22C4600250028C0D42B48006878
:10A030007D21C900F6F74EF820492D3141432046D5
:10A0400000F050F803F09AFE04463868C069C00773
:10A0500005D003F093FE001B31888842F5D903F048
:10A060008DFE04463868C169890706D503F086FE6F
:10A07000001B31888842F5D938680121009A1160A7
:10A0800017498161284603B0F0BD032121600028F3
:10A090008AD08AE7034804A1084A09A303F09CFE7A
:10A0A0003C930102E01D0100666C6173685F73659B
:10A0B00063746F725F657261736500002B0200004C
:10A0C000736563746F7220696478206973206F769A
:10A0D00065722072616E67650D0A0000A0DC0102E6
:10A0E000000093EBF0B583B001917C2202904243D3
:10A0F00053498C182546143503F040FE06460221CC
:10A10000029800F01DF803F039FE07462068C16987
:10A11000890606D403F032FEC01B29888842F5D98F
:10A120002068007DC00708D06420FEF7CDFD03F055
:10A1300025FE801B01998842E1D903B0F0BDC046DD
:10A14000F0B585B0049104467C2060433C490F186B
:10A150003D46143503F012FE06463868C069C00754
:10A1600005D003F00BFE801B29888842F5D903F047
:10A1700005FE06463868C069800705D503F0FEFD78
:10A18000801B29888842F5D91421049B5943DC207F
:10A1900060432C4A1018039002914018018A82688B
:10A1A000C47C7426BE5D012E0DD10191012B029954
:10A1B0000CD0012B0DD07526BE5D012E0ED0019E58
:10A1C000072B0ED10EE00E4602990BE00222012B66
:10A1D000F1D138247526BE5D012EF0D10326072B60
:10A1E00000D0019E184B334024069207D20A121960
:10A1F000D218039B5958C907490C52184168CB071C
:10A200001B0CD218837C5B075B0BD218C06840071D
:10A21000000A10183A685060002E0ED001290CD1A7
:10A2200003F0ACFD04463868C069800705D403F02C
:10A23000A5FD001B29888842F5D905B0F0BDC046B0
:10A240003C9301029C130100FF3F0000F0B59DB05C
:10A250000D460126890E2FD0002B2DD01192812181
:10A26000C9041093C91AA94226D30121EFF310841F
:10A270000C4002D1EFF3108272B67C220F90424361
:10A28000E74814928718384610303B690026062BA1
:10A290000DD80A469A40D3065B0F07D161231A42B4
:10A2A00000D16FE30E46002C03D003E00226002C01
:10A2B00000D162B6002E02D030461DB0F0BD029033
:10A2C000BD650021139179651098401E12904019C8
:10A2D000B964B9690D916E1A1199B962FD6238635A
:10A2E0007E63F98C0E913046F5F7F4FE0446B863B0
:10A2F000129830180E9E3146F5F7ECFE109B011BAC
:10A300004A1CF86339647A64139A0029194608D004
:10A31000704359190D9BC91A0A1A7443581B8019A6
:10A320000119384648300E90384644300D90384672
:10A3300040300B9038462630059038465830139000
:10A34000384654301290F9643A651498B449085864
:10A350001021C161384614301490384650300490B2
:10A360003D464C3503F00AFD04463868C069C00616
:10A3700006D503F003FD001B149909888842F4D91F
:10A38000F87D40060C9500D574E201230E98036019
:10A390000D98016800290F9800D1CDE23A46743239
:10A3A0000A92DA0407921A050992192252060692B5
:10A3B0000722D206089216E09A4800687D21C9005B
:10A3C000F5F788FE109941430F9C2046FFF78AFE5F
:10A3D00020460C9D0E9A11684B1C13600D9909685C
:10A3E0008B4200D9A8E20B9A1268012A55D0002AA4
:10A3F00000D0A8E02E6812990C6813990D68062108
:10A400001091FFF79DFE386885601198051903F0DB
:10A41000B5FC04463868C069C00706D003F0AEFC3E
:10A42000001B149909888842F4D903F0A7FC04465C
:10A430003868C169890707D503F0A0FC001B14998F
:10A4400009888842F4D938680A990A78012A089953
:10A4500000D00699012A099A00D0079A3346724C17
:10A46000234013430B4371490B434360002EA3D099
:10A4700003F084FC04463868C069800706D403F002
:10A480007DFC001B149909888842F4D93868297822
:10A4900001756D1C761EFAD18EE7012B00D0C7E046
:10A4A0002E6812990C6813990D6806211091FFF718
:10A4B00047FE386885601198051903F05FFC044673
:10A4C0003868C069C00706D003F058FC001B149917
:10A4D00009888842F4D903F051FC04463868C16900
:10A4E000890707D503F04AFC001B149909888842A4
:10A4F000F4D938680A990A78012A089900D006998F
:10A50000012A099A00D0079A3346474C2340134347
:10A510000B4346490B434360002E69D003F02EFCE9
:10A5200004463868C069800706D403F027FC001B86
:10A53000149909888842F4D93868297801756D1C06
:10A54000761EFAD154E0012B00D0C9E02E68129992
:10A550000C6813990D6806211091FFF7F1FD38681A
:10A5600085601198051903F009FC04463868C06934
:10A57000C00706D003F002FC001B1499098888422A
:10A58000F4D903F0FBFB04463868C169890707D595
:10A5900003F0F4FB001B149909888842F4D9386849
:10A5A0000A990A78012A089900D00699012A099A7D
:10A5B00000D0079A33461C4C234013430B431B49DE
:10A5C0000B434360002E13D003F0D8FB04463868D9
:10A5D000C069800706D403F0D1FB001B14990988D9
:10A5E0008842F4D93868297801756D1C761EFAD135
:10A5F0000C4800687D21C900F5F76CFD10994143B6
:10A600000F9C2046FFF76EFD20460C9D2A68139B89
:10A61000196889181960129B196889181960D9E698
:10A620003C930102A0DC0102FF3F0000008080009B
:10A630008B4200D0CEE604990E6812990C681399EB
:10A640000D6806211091FFF77BFD38688560119831
:10A65000051903F093FB04463868C069C00706D0AB
:10A6600003F08CFB001B149909888842F4D903F08D
:10A6700085FB04463868C169890707D503F07EFB6E
:10A68000001B149909888842F4D938680A990A7815
:10A69000012A089900D00699012A099A00D0079A40
:10A6A0003346D44C234013430B43D3490B434360FD
:10A6B000002E00D180E603F061FB04463868C069D3
:10A6C000800706D403F05AFB001B149909888842BE
:10A6D000F4D93868297801756D1C761EFAD16BE6BD
:10A6E000129A1268119CA618139A15688B425FD1B2
:10A6F00004990C6806210391FFF722FD38688560F4
:10A7000003F03CFB05463868C069C00706D003F07B
:10A7100035FB401B149909888842F4D903F02EFBBD
:10A7200010900C9D3868C169890708D503F026FB95
:10A730001099401A149909888842F3D938680A99FF
:10A740000A78012A089900D006991091012A099ADD
:10A7500000D0079A2346A7490B40134310990B4397
:10A76000A5490B434360002C14D003F007FB109065
:10A770003868C069800707D403F000FB1099401ABD
:10A78000149909888842F3D9386831780175761CA4
:10A79000641EFAD19A4800687D21C900F5F79AFC39
:10A7A000039941430F9C2046FFF79CFC204611E68D
:10A7B00005990C8806210391FFF7C2FC3868856073
:10A7C00003F0DCFA05463868C069C00706D003F01C
:10A7D000D5FA401B149909888842F4D903F0CEFABF
:10A7E00010900C9D3868C169890708D503F0C6FA36
:10A7F0001099401A149909888842F3D938680A993F
:10A800000A78012A089900D006991091012A099A1C
:10A8100000D0079A234677490B40134310990B4306
:10A8200075490B434360002C14D003F0A7FA109035
:10A830003868C069800707D403F0A0FA1099401A5D
:10A84000149909888842F3D9386831780175761CE3
:10A85000641EFAD16A4800687D21C900F5F73AFC08
:10A86000039941430F9C2046FFF73CFC2046059985
:10A870000A88CCE65E4815A90A4678C878C278C826
:10A8800078C20125E8073A68136803431360B86883
:10A89000FEF78AFA02200026139C2168BA6AF9653D
:10A8A0003A6610997966BE66F8660C980068129A46
:10A8B0001168091811600E9B19684A1C1A602268F9
:10A8C00010182060002900D0F6E41095384660305A
:10A8D00013903C465C3438460830129006210F989D
:10A8E000FFF72EFC3868216881600C980068119091
:10A8F00003F044FA04463868C069C00706D003F084
:10A900003DFA001B149909888842F4D903F036FAFD
:10A910000446109D3A68D069800707D503F02EFAE7
:10A92000001B149909888842F4D93A687420385C6D
:10A9300001282DD0E9042CE003F020FA0446386801
:10A94000C069C00706D003F019FA001B14990988E2
:10A950008842F4D903F012FA04463868C1698907BD
:10A9600007D503F00BFA001B149909888842F4D923
:10A9700038680121029A116022498161002630461F
:10A980001DB0F0BD04210160002C00D191E491E4E0
:10A990002905119C174B2340591801280C9D02D002
:10A9A0001920400601E00720C00608181249401887
:10A9B0005060002C0ED003F0E1F904463A68D069EB
:10A9C000800707D403F0DAF9001B1499098888423C
:10A9D000F4D93A682B681398016812980068074CFC
:10A9E00000941432FEF750FA30461DB0F0BDC04658
:10A9F00014120100FF3F00000080800095960000C7
:10AA0000A0DC0102000093EB3920C0000149096875
:10AA100008587047C8920102F0B5032920D8C046F3
:10AA20007944097949008F4401080F1501218140BB
:10AA30004F4B1B685963D96212E0012181404C4B96
:10AA40001B681963D9620BE001218140484B1B68E8
:10AA5000596304E001218140454B1B6819639962E9
:10AA600083004349CB18DA608A68002A29D14A68F2
:10AA7000002A16D4032314469C43174BE558960727
:10AA8000F60EFF27B740BD438027B7402F43E7505E
:10AA90001F23134001229A40104B1A60104B1A607A
:10AAA0000FE09307DB0EFF259D400F241440083C68
:10AAB00003229443074AA658AE4380259D40354360
:10AAC000A5500122824008680262886810438860AD
:10AAD000F0BDC0461CED00E000E400E080E200E0D4
:10AAE00000E100E010B501242046FEF715F82046ED
:10AAF00002F098FE002010BD012181401C48006832
:10AB000042688A4342607047194909680968C14030
:10AB1000012008407047C046012181401448006868
:10AB200042680A4342607047012907D0002910D1CA
:10AB3000012181400F4802680A430FE00121814052
:10AB40000B4800684368002A0DD00B434360016145
:10AB5000704701218140074802688A430260044827
:10AB60000068416170478B43436001617047C04694
:10AB7000CC9301020801004080B5114A1170114ABE
:10AB800010708001C90101430F480078400108435B
:10AB90000E490978090101430D480078C0000843B7
:10ABA0000C490978890001430B48007840000843AC
:10ABB0000A4909780143C8B2F9F746FC80BDC0468E
:10ABC0004C9D01026E97010220940102BEE4010235
:10ABD00041AB01024D9D0102C8A00102C9A00102C2
:10ABE000012282400548002903D001681143016019
:10ABF00070470168914301607047C0460001004002
:10AC0000124A072809D880000F2383408140194049
:10AC1000106898430843106070470F280AD88000D6
:10AC200020380F23834081401940506898430843DF
:10AC300050607047800040380F23834081401940A6
:10AC400090689843084390607047C04634000040C5
:10AC5000F0B54307DC0E0726A640C3089D000E4B47
:10AC6000EF187D68B5433E1D002908D035600122EC
:10AC7000824001290CD1186810431860F0BD0121F1
:10AC80008140186888431860A24015433560F0BDC4
:10AC9000186890431860F0BD0C01004010B582B0F8
:10ACA00014460A4601460498009301900820234662
:10ACB00000F092F802B010BDB0B584B014460A4658
:10ACC000014608980225009501930290072023462B
:10ACD00000F052F904B0B0BD70B500285BD0314926
:10ACE0000A783149002A03D14A68012313434B6093
:10ACF000428803881B049A180B46183B1A60828806
:10AD000083891B049B180C460C3C23600B46083BB4
:10AD100084681C60446903232340057CAD00EB1864
:10AD20008569AD072D0D5B19457C2D035B19C56940
:10AD3000AE07B60A9B19867CB6059B190E1F3360B9
:10AD4000036A122B04D107240C60541EA2410AE0AE
:10AD5000032C05D1012D03D807220A60012202E04D
:10AD600006220A600122114C002525700F2464017F
:10AD70002034C57C6D0225401B069B0BD218C3797D
:10AD80001B07DB0ED21880790007C00D1018401980
:10AD90001439086070BD064806A1862209A303F095
:10ADA0001BF8C04684CA01021810005086CA01026E
:10ADB0003B2A01006C73705F656E67696E655F7238
:10ADC000756E0000506172616D6574657220697303
:10ADD000206E756C6C000000F0B58BB0109E3404D2
:10ADE0003ED00D46D64C2140012701977F06B9423F
:10ADF0003CD111462140B9423FD11C40BC4243D115
:10AE0000119902AC0027E781E780668027802782BE
:10AE1000A774E1749908A181A908A1800A900997F3
:10AE200008970797900880B204902046FFF754FFD8
:10AE3000AA480078002801D00BB0F0BDAB480168EB
:10AE4000C90708D10168C90705D10168C90702D13E
:10AE50000168C907F3D07F48019901700BB0F0BDBC
:10AE6000B8480D49AF22C14B02F0B6FF0095B54876
:10AE70000949B022754B02F0AFFF0092B148064974
:10AE8000B122724B02F0A8FF0093AE480249B222F1
:10AE90006E4B02F0A1FFC046112A0100F0B58DB043
:10AEA0000392139E340446D00A46A54C2140012546
:10AEB00002956F06B94244D103992140B94247D166
:10AEC0001C40BC424CD11499129D04ACE174294938
:10AED00021820027E781E780668027809908A18189
:10AEE0009108A1800B95012D01D16121CF43A77459
:10AEF0000C9002200A9009900398800880B2069076
:10AF00002046FFF7E9FE75480078002801D00DB013
:10AF1000F0BD76480168C90708D10168C90705D1A5
:10AF20000168C90702D10168C907F3D049480299ED
:10AF300001700DB0F0BD83480D49FB228B4B02F030
:10AF40004BFF00927F480A49FC22404B02F044FF2D
:10AF5000039800907B480649FD223C4B02F03CFFE1
:10AF6000009378480249FE22384B02F035FFC04674
:10AF70001E2A01008E8E0000F0B58BB0119E3404A5
:10AF800047D00D466E4C2140012701977F06B942FC
:10AF900045D111462140B94248D11C40BC424CD158
:10AFA0001299109F02ACE174294921820021E181AC
:10AFB000E180668021809908A181A908A180099774
:10AFC000012F01D0712100E06121C943A1740A90D1
:10AFD000032008900790900880B204902046FFF765
:10AFE0007BFE3E480078002801D00BB0F0BD3F4802
:10AFF0000168C90708D10168C90705D10168C907F7
:10B0000002D10168C907F3D01248019901700BB051
:10B01000F0BD4C480C49D522544B02F0DDFE0095A2
:10B0200048480949D622094B02F0D6FE009245480D
:10B030000549D722054B02F0CFFE00934148024953
:10B04000D822024B02F0C8FE2D2A01005B2A010023
:10B050008686000086CA010210B582B014460A46F0
:10B06000014600200093019004202346FFF7B4FE20
:10B0700002B010BD10B584B014460A460146002047
:10B0800000900193029004202346FFF707FF04B0CD
:10B0900010BD000070B50D46064604242046FDF79D
:10B0A0003BFD204602F0BEFB0B4805600B480670D6
:10B0B000002E0ED00A48016880220A437F218A436D
:10B0C000026001200003074908600749086007483B
:10B0D0000460002070BDC04688CA010284CA010213
:10B0E0000CE400E080E200E000E100E01C10005011
:10B0F000B0B582B0144602461148204001256D06C5
:10B10000A8420DD1180413D0174801600020009305
:10B110000190062011462346FFF75EFE02B0B0BD47
:10B120000094FF228C320748074908A302F054FE1E
:10B13000FF208C30421C034803490C4B02F04CFEAC
:10B140000300FCFF3B2A0100032A01004473742022
:10B150006164647265737320257820697320696E59
:10B1600076616C696400000008100050792A0100C3
:10B1700080B582B00B46014600200092019003206A
:10B180000A46FFF729FE02B080BD0000002801D06A
:10B19000042100E00221C24A5172411E884180010F
:10B1A00003490A6840239A43101808607047C04654
:10B1B00050A00050F0B583B002912E49CD7A0E7B9D
:10B1C000771987424FD9089901911825454341269F
:10B1D000F604BF00BE19745B34490C4057033C1998
:10B1E0009B07D90C6418324B1B681B7A7453751972
:10B1F0006C880326B60326409B079B0C9B193F24B3
:10B2000004401819029CA3061B0DC0186880012A6F
:10B21000184E13D8707B14224243307B5023434393
:10B2200024011B199A18F37AC0181C234343D01821
:10B2300080081E4A104007430F432F800198686022
:10B2400001F074FEA860E8681A4908403030E860F0
:10B25000286908402721715C4018286100F006FE2B
:10B26000686103B0F0BDFF228832034803A108A340
:10B2700002F0B2FD8CCF0102CA2A01006D61635F4A
:10B2800063735F636F6E73747275637400000000A4
:10B29000435320696E646578206973206F76657208
:10B2A0002072616E67650D0A00000000FF07000054
:10B2B000389401020000F0FFF0B581B0009314460D
:10B2C0000D46074606263046FDF726FC304602F0BE
:10B2D000A9FA26211D48475400210170417081714F
:10B2E000017181704171C170C17102224272C162EB
:10B2F00001634163816304734273C572009A561CF3
:10B30000134A168001724120C00401214903F4F759
:10B3100024FF502060432901081861198A00801811
:10B3200018224A438018B2B24A438018094940188B
:10B330000949884204D200F0B5F8002001B0F0BD00
:10B34000064807A19A2209A302F046FD8CCF01020C
:10B3500088CF01022800080201200802CA2A010041
:10B360006D61635F696E697400000000454D206F78
:10B37000766572666C6F770D0A000000A448C1798B
:10B38000002901D001207047007A411E8841704792
:10B39000F0B583B002912A494B7B834248D9CB7ADE
:10B3A0000C7BE31818245C439B00E3184124E4045D
:10B3B0001A1914240190054665430026565100923F
:10B3C0005519EE882E4F0B467A1C3240F54E3688C2
:10B3D000497A711A2B4E0E40B618EE803740997B91
:10B3E000EF80AA88284F17404A424A4191007918B5
:10B3F000264A8918A980264F0F402D1D0298012842
:10B400000AD124490E400921C9027118698001211D
:10B41000C9037918298000E02F80019844430098DF
:10B420000019074A918C4182118C018203B0F0BD52
:10B430003520C200034804A109A302F0CDFCC04698
:10B440008CCF0102CA2A01006D61635F6C696E6B6B
:10B450005F646573635F636F6E73747275637400AA
:10B460004C696E6B206465736320696E6465782037
:10B470006973206F7665722072616E67650D0A00D0
:10B48000FFFBFFFFFF03000003D0FFFFE80F0000FA
:10B49000EF1F0000FF830000BE4A506391637047B6
:10B4A0008CCF0102F0B581B04348CC21016003216B
:10B4B0004160B8490A7BD304404C1B19CC7AA218CE
:10B4C000541E1C431823534392009A184B7B142597
:10B4D0005D435219920122430124630613434361E1
:10B4E00000228262C262026342638263C263426577
:10B4F0000267334B1A605A609A60324B1A601A61C5
:10B500009A61DC61304C1C62304C251D1D63254660
:10B510000C3D5D632546283D9D632D4EDE631C6416
:10B520005C642C4D2F461C379F642746143FDF6414
:10B53000103C1C65284C5C65284C9C650C369E674D
:10B54000274CA5634035E563DA651A665A669A6644
:10B55000DA661A67234DDD6702258561224DC561D4
:10B56000C325AD03CD620A63D2435A601F4A1368F4
:10B57000FF25AB4326254D5DAD072D0EEB1813605F
:10B580001B4A102313601B4A1360272260238B542D
:10B5900019498160C160016121607D210901016655
:10B5A00041661649C164164941641649016400F0B8
:10B5B0004DFC01B0F0BDC04604A000500000F8FFF3
:10B5C00094A0005034A10050FF185A0030040040ED
:10B5D000041000401C2000405430004060400040F7
:10B5E000B8A1005014001400FF3F3FFF04E400E046
:10B5F00080E200E000E100E0DC05DC053F027002D3
:10B600000133D007D007D0072921C64A50547047CC
:10B610008CCF0102F0B58BB0079208910146C14F63
:10B62000B8780991FFF7B4FE78793A7B7979069179
:10B63000824200D89FE0FB7A9A1818235343920065
:10B640004124E10404915218D2187B7B14214B430E
:10B65000D21850246043155801230A93DB022E466A
:10B660009E4316504E4B2B4005937D7B03914D43DB
:10B670003E7B7443F97A0B011B195B1971181C246A
:10B68000029461435918A84B1B88069C5C43091916
:10B69000C904490D059BC91811501018079941603C
:10B6A00038787979089A00920322099BFFF782FD86
:10B6B000F87A397B09183878814263D98300099375
:10B6C000049AD45C0894F7212140D154D1184D78C4
:10B6D0008E7836027619CB781B04F31807900A98F7
:10B6E00086051E43330CCB70FB7A387BBC784D70DB
:10B6F0009F4D3540039E6643C018029B43439819F3
:10B7000040029C4B03405C19200A8870200CC870D2
:10B71000F023089D2B401B1D3D7B0895FE7A099D5B
:10B720005355C8700620079A50438019089A80180C
:10B7300048701F22D20222400243100A8870787992
:10B74000401C7871387B7979814201D3002179716D
:10B750003978491C3970F97A08183978884201D843
:10B760000020387028200A993954387A401C3872E1
:10B77000387A0BB0F0BDA7204200D2480649074BEB
:10B7800002F02AFBA72042007A32CE487349744B5C
:10B7900002F022FB8CCF0102EA2A0100932A010069
:10B7A00000F0FFFF88CF01020320000605490A6868
:10B7B00082430A600A6802430A600348012101606B
:10B7C0007047C0461C0000401CA0005080B50120FE
:10B7D000FDF758FC80BD0000F0B587B00693064623
:10B7E000504C607A504B1B88181A0C9DA84200DC04
:10B7F00089E00F460592012E06D156480021C1620C
:10B800000169554A89180160A0783146FFF7C0FDEB
:10B81000E078E178069A2B4600F0AEF82078E178DF
:10B820000097002206923346FFF7C4FCE07A217BA2
:10B830000818217888426ED94120C20404918800FA
:10B84000815C0391F7250D40029285544549455C82
:10B850004549465C360276194449475C3F04F6196F
:10B860000127BF0537433E0C4654E67A217BA37877
:10B870003C4A85543E4D3D4014275F4389191C23A3
:10B880004B43D91949023B4B0B405D19290A364BF2
:10B89000C1542E0C35494654F02703990F400599A1
:10B8A000002900D13F1D217BE37A029A87542F4A59
:10B8B00086540622049E7243D2185118294A815494
:10B8C0001F22D20215400D43290A274A8154E078ED
:10B8D000401CE070E07AE178814201D30699E17082
:10B8E0002178491C2170217B08182178884201D8D1
:10B8F00006982070E079401CE071A07A401CA0728C
:10B90000E07907B0F0BD3920C2001632074808A11F
:10B9100009A302F061FA3920C20004480F49104B14
:10B9200002F05AFA8CCF010288CF0102CA2A010024
:10B930006D61635F747800004D4143205458206C62
:10B94000656E206973206F7665722072616E67651F
:10B950000D0A00000804004090D00300002B0100F5
:10B96000B12A0100010008020200080203000802D7
:10B97000FF07C0FF00F83F00F0B589B008930192BF
:10B9800004914F4DEF7A874200D891E0297B5026F1
:10B9900032464A434124E3040693D218CC19A1004D
:10B9A00051181822059254430A19697B14230793EE
:10B9B0005943531802900001195804460390504A05
:10B9C0000A40A97AC902511808988205D2088A1833
:10B9D0001A514C4911402A7B00965643384CE57A5F
:10B9E0002C0106982418A719354E5419A5007D1965
:10B9F000059844432819747B079D6C430519049FDF
:10BA0000D2194148048854432A19089CD204520D83
:10BA100051181D460398195000F032FA0146707A09
:10BA2000001902043E460CD080B2C000002900D1AB
:10BA3000801E029FA5214900F4F74CFB1F21014005
:10BA400001E00021029F38012818427983791B0206
:10BA50009A18C3791B04D2182C4B13404371090464
:10BA60005918090CC171002C20D0154835460646DE
:10BA7000007B009B4343F17A0A01069F3A43D218A8
:10BA800041188B00D218059B4B43D118727B079B42
:10BA90005343C91840191C4A128842438818019917
:10BAA000884203D001992246F4F73EFB09B0F0BD6D
:10BAB000FF225C32034804A109A302F08DF9C046BD
:10BAC0008CCF0102CA2A01006D61635F74785F64E4
:10BAD0006573635F636F6E737472756374000000E7
:10BAE0005458204445534320696E64657820697337
:10BAF000206F7665722072616E67650D0A00000026
:10BB0000FF0700E000F8FFFF88CF0102EFFFE00031
:10BB100082B0FCF703FEFCF763FE0020FCF730FE6A
:10BB200001F000FE01F0F8FD60480168604800681F
:10BB3000890309D403210907084001210907884224
:10BB400002D0FCF7B9FD06E0FCF70AFAFCF7CCFDE1
:10BB50000020FDF7DDFCFCF771FE0024204604F018
:10BB60000DFC032000902146FBF79EFDF8F76EFDCB
:10BB7000FBF7D0FAFEF7B6FFF8F75CFAF7F73AFAF8
:10BB8000F8F7EDFC042738462146FFF739F8012580
:10BB9000384629462246FEF7C7FF05223846294681
:10BBA000FFF756F8284629460195FEF7E5FF414F75
:10BBB00038462830404A2946FCF70EFC3F4E311DDE
:10BBC000284603F0E5FC3E483E49016000F0AEF82F
:10BBD0003D4B2825DD823D48B86438610220F8617C
:10BBE00098887862997AB9709989F981598B384A1D
:10BBF0005A833987B8867D20C000D988F4F76AFA5D
:10BC0000B881019882023349334B03F095FD01F06E
:10BC100067FB324A0198014601F0F4FF304802F018
:10BC200021F83048FCF71EFD2F48FCF72FFD2FA20E
:10BC30000098014603F02CF90CE03170401C78703C
:10BC4000F7F7C8FF7F20C105B869F4F75EFBB8615C
:10BC5000F8F7BEFC3078002803D1F8F7EFFC002895
:10BC60000DD03879002802D03C71F7F731F8F8F799
:10BC7000F9FCF7F741FDF7F771FFFBF759FA78790F
:10BC80000028E5D07C71FBF773FBF7F7B3FB0E4898
:10BC9000C582F8F7D3FC002802D034707C70CFE75F
:10BCA00078781E280199C8D32146C6E718000040BD
:10BCB00030000140C8970102A58200001C900102DB
:10BCC000C0950102E5780000D6A6010228002800F0
:10BCD0003412000088CB010271F90000C9DB0000BA
:10BCE0007C3F00007903010021BD0000B2E2CAD40C
:10BCF000BDF8C8EB61707000014800687047C0462D
:10BD00000C00004081B080B581B0039303AB009379
:10BD100002F038FD01B080BC02BC01B00847000051
:10BD20000148002181617047C8970102F0B581B0D8
:10BD3000002630463146FDF751FE0125AC0222496E
:10BD4000224F30463A462346FDF7A8FF398820485F
:10BD5000814236D064217E5262217E5260217E5221
:10BD600050217E5244217E52FD87BD8778217987FC
:10BD7000022139874321F986BE83FE811549B981A5
:10BD80007E810A2139811449B9803880FE837D2063
:10BD90008000F880EFF3108072B630463146FDF730
:10BDA0001DFE00280CD12A0300263046064D2946E8
:10BDB000FDF76EFD054A304629462346FEF746FA52
:10BDC00062B601B0F0BDC04600E00204D6A6010292
:10BDD000AA550000E1FF0000341200000020704767
:10BDE00010B50024002809D0002905D003464A00D8
:10BDF00003481946F4F798F9204610BDE04310BDFA
:10BE000030930102014600200A2901DAC04370473D
:10BE1000014A11807047C046B89301020020704764
:10BE200080B50188064A11808178064A1170C17870
:10BE3000054A11700079FCF7AFFB002080BDC046B9
:10BE40002294010224940102D8CF0102044805493A
:10BE50000160152109044160034981607047C046B3
:10BE60009C3000404100080034000700074800688B
:10BE700040697047FD20400004490968085C70472C
:10BE8000024800686221405C7047C0463894010255
:10BE90000A491A220A600A4948704878FF210902B3
:10BEA000084A13688B43800380B2C01810600648AC
:10BEB000202101600548016000207047702000408B
:10BEC0002894010204E400E080E200E000E100E0E8
:10BED000F0B5A9B016460F460546C648002B0246E7
:10BEE00000D01A463921CC003D21C90051181191CA
:10BEF0008242189206D001204202BE491898F4F7F7
:10BF000013F9189A6120111913910E21119C0A91AD
:10BF1000A170002F0D9501D00A2100E009215923BD
:10BF200017938300E1707842784113990870307854
:10BF300010901070F17AE17471785170B778977041
:10BF4000F178D1703579157174795471B179917135
:10BF5000F179D171317A1172717A5172B17A91722B
:10BF60007E1EF0B200210328169106D870B2800020
:10BF7000A1A210586A00805A16901798820018984B
:10BF8000C0181490F81E022804D3012E084604D8C5
:10BF90009D4800E09D48031918781290189DA81834
:10BFA00017902846303015902C4656346D2080006E
:10BFB0002950974A974B149E33627262B362F262C1
:10BFC0003176F182139B597009229A7028184160CA
:10BFD0008160C1600161109880008F490858F4F7B2
:10BFE000B3FC012F10900F9104D0022F05D17F21B7
:10BFF0007E2004E07C217B2001E05B215A20159DFE
:10C00000A984207003200C90A080012666701F2058
:10C010000B90A8821820A8740A46083A179BDA7673
:10C02000169B129AD2184A439100189A9163B7024C
:10C03000791E8B420E9109D978486080342068843B
:10C040007748288277481399088339E07F2B10DDE1
:10C05000802B18D031028B421BD071028B4227D12A
:10C060006E49618068846F4813990883CF20C000AF
:10C0700025E0202B17D0402B1AD16848608004207F
:10C08000688469481BE065486080062068846748CA
:10C0900015E0624860801020688462481399088324
:10C0A000C520C0000BE0624860800220688404E084
:10C0B00004206884812040006080FF2002302882B4
:10C0C000104600F0D7FE1298102806D0402808D15C
:10C0D00008201499C876072000E00420179988707A
:10C0E00002E017980C9981701898169A8078C11EF2
:10C0F00002290CD3022811D001280CD12672BA4291
:10C1000000D900266672BA4213D8F44812E00D2016
:10C110000002119908800120800201E00C980002C1
:10C120002081BA4201D8EE4800E0FA2017998860D1
:10C130000EE0FA201799886013980078002811996A
:10C1400001D0E8484880E848139A1083E7480880FF
:10C15000A88CF4F799FB0026E54B3246F4F75CFA1D
:10C1600002460B46E3493046F4F7BEFAE24B32464C
:10C17000F4F752FAF4F7C4FB0746E080DF49304693
:10C18000109A0F9BF4F7B0FADD4B3246F4F744FAFD
:10C19000F4F7B6FB78434042800B608116990E9805
:10C1A000814208D90C20149FB872D6481799888309
:10C1B0001220189A0EE0480A189A149F01D00D20F8
:10C1C00003E0080A00D1DBE20A98B872CE4817995A
:10C1D00088831220F872D078052844D878440079F2
:10C1E000400087440227402C3339C848B881C848EA
:10C1F0002FE0C046C8900102C4110100C411010023
:10C20000D4110100D4110100B20E0100B90E0100D9
:10C210003075000010270000740F010005020000B7
:10C22000FF060000040800000A04000036040000B5
:10C2300003020000B748F881B748388013E0B748D8
:10C24000F881B7483882B74838600CE0B448B88104
:10C25000B5481799C88306E0B4487882B448B880D6
:10C260000B9800069064AE483881A748F880B14822
:10C2700002882A84B0480078E874B0480078119F9A
:10C280007875387D139000285ED0AD490A68102378
:10C29000DA413A600A794B79CF8867801B029A1895
:10C2A0006A840A7A4B7A8F7AC87A0D7B65701B0292
:10C2B0009A183B04D21800061018179FF860487BA4
:10C2C0008A7BCB7B3B77120210186081087C7877E1
:10C2D000487C149A9072887CD072C87C159B187424
:10C2E000087D5874487D11909874C87D0A7E1202AA
:10C2F00012181A84887DD87418464B7EC375887EC0
:10C30000CD7E2D022818B880087F4D7F2D02281879
:10C31000F880887FB877C87FF8772020085C149D64
:10C3200028732120085C68732A20085C2A314D7824
:10C330002D0228188D782D044019C9780906401857
:10C3400018998864119801E0EB7DA87C7D498B7079
:10C350000A8080001F38C882C883139800281FD025
:10C3600022227748825C034622335B781B029A18AC
:10C370000A842422825C034624335B781B029A18C9
:10C38000CA842622825C034626335B781B029A18F5
:10C390008A832822825C28304078000280188884B2
:10C3A0006948032569A2294602F072FD189F387872
:10C3B00014907B78B8780F90FA78B8791390F87960
:10C3C0001190387A1090787AB97A08900991009390
:10C3D0000F98019002921698039012980490139867
:10C3E00005901198069010980790FAA2F8482946EF
:10C3F000149B02F04DFD3D46643580212846F3F73D
:10C40000ACFEB878C11E02290ED3012800D18FE1FD
:10C41000022800D0ABE11691149078787F22504327
:10C42000F7494018F74907E01691149078785B2295
:10C430005043F1494018F14941182846F3F774FE7A
:10C440000D9D1898C6870E34324602E0641C0F2AF0
:10C450000ADA21780029F9D0491C8907C90F9140CF
:10C460000E43C687521CF1E71699022907D3149987
:10C47000491E012900D97DE14279D24901E0427982
:10C48000CF4989180C78002D00D177E1C1790E9140
:10C49000032900D94AE14279062A00D979E14921E4
:10C4A000890041181191E43010900E98401E1290AE
:10C4B00019A800190F9000231392149403E0189800
:10C4C000290600D15AE1052A5AD8C0467A44127981
:10C4D00052009744455C728598ABC04688130000B3
:10C4E000E20400000C080000060A0000040F00002F
:10C4F0000000104130C1BD41000070400000F0401C
:10C500000000D041120C0000140B000012120000B9
:10C51000140E00000E160000130D0000121600008D
:10C520000E120000140B0E0A120800001016000074
:10C530000E0B00002294010224940102D8CF0102C4
:10C54000E4CF010290940102010800004361736589
:10C5500020706172616D65746572733A200D0A0016
:10C560001693DFB2002F04D019A801223946F3F741
:10C57000EDFD002C00D191E019A8C019BB498AE05B
:10C58000E8B2022867D00027022867D06BE00E9837
:10C59000022872D1E8B2022800D103461693DFB216
:10C5A000002F04D019A801223946F3F7CFFD002C43
:10C5B00074D019A8C019ACA16DE0E8B2022800D16E
:10C5C00004231693DFB2002F04D019A801223946A4
:10C5D000F3F7BCFD002C61D019A8C0199FA15AE047
:10C5E000E8B2022800D106231693DFB2002F04D050
:10C5F00019A801223946F3F7A9FD002C4ED019A83D
:10C60000C01992A147E0E8B2022800D10C2316938A
:10C61000DFB2002F04D019A801223946F3F796FDA6
:10C62000002C3BD019A8C019874934E0E8B2811E1C
:10C630004A424A419700022804D119A801223946EA
:10C64000F3F784FD002C16D019A8C0197CA122464E
:10C65000F3F76AFD0FE00627022804D119A801228A
:10C660003946F3F773FD002C05D019A8C01980498D
:10C670002246F3F759FD169710E01693DFB2002F0C
:10C6800004D019A801223946F3F760FD002C05D02B
:10C6900019A8C01973492246F3F746FD3C193F2CEF
:10C6A00005D80F98C0194021091BF3F756FD1298C1
:10C6B0000228189801D2002002E0C078411E88416B
:10C6C00015990870611E2E46E8B202280CD1179AFF
:10C6D000517019A9119AB8C9B8C2B8C9B8C2B8C9B5
:10C6E000B8C2B8C9B8C20DE0179A117019A9109A4A
:10C6F000B8C9B8C2B8C9B8C2B8C9B8C2B8C9B8C24E
:10C70000C10709D180073546149C139A169B00D4A3
:10C71000D5E602208543D2E6FE203546054018982E
:10C72000149C139A169B290628D0CCE637A231E038
:10C730001691149078780B994143334808181F38A4
:10C740006F21C9430D9D7A180378D427D3554378B8
:10C75000D827D3558378DC27D355002900D170E63C
:10C76000C378E027D3551031001D189FEBE7012057
:10C77000404A10E00024002D00D087E629B0F0BD2B
:10C7800080290ED30F20B872104817998883102083
:10C7900020E525A20120014602F07AFB189829B075
:10C7A000F0BD1020402904D3B8720849179B998323
:10C7B00010E5B87204481799888314200AE5C0462A
:10C7C000B90E0100B20E0100150F0000140B00009D
:10C7D00001080000256420256420256420256420AC
:10C7E00025642025642025642025642025642025D7
:10C7F000642025640D0A0000863401001DF7FFFF48
:10C800009E2B010089FBFFFF8E3301007472785F5D
:10C810006D6F646520706172616D6574657220650D
:10C8200072726F720D0A00004E736664207061723E
:10C83000616D65746572206572726F720D0A000019
:10C84000FFFFFFFF01FF000074120100FFFFFFFF69
:10C85000FF0101FFFF01FF01FFFF01FFFFFFFF01DC
:10C86000FFFF01FF60180100FFFF01FF94120100AC
:10C87000E41101003C2B0100002800D101480649C9
:10C8800008607047C8900102F0B586B0002805D155
:10C890000148006802E0C046389401023121C90015
:10C8A000049141188A791F231A40CD79ED06AD0D08
:10C8B000AA180D7AED066D0C52194D7AED062D0B66
:10C8C00052198D7AED06ED095219CD7AED06AD08B3
:10C8D00052194D7CED075219BD4C22600A7B1A405B
:10C8E0004E7BF606B60DB2188E7BF606760C9219C4
:10C8F000CE7BF606360B92190E79F606F6099219DA
:10C900004E79F606B608921962604A6AB14D2A401D
:10C91000A2608A6A2A40E2602D22D20087183A7EFD
:10C920001A4003937E7EF606B60DB218BE7EF6065A
:10C93000760C9219FE7EF606360B92193E7FF606AD
:10C94000F60992197E7FF606B60892190E7CF60754
:10C9500092192261BA7F1A400597FE7FF606B60D3E
:10C96000B218049BC35CDB065B0CD2184B78DB0669
:10C970001B0BD2188B78DB06DB09D218CB78DB06D1
:10C980009B08D2186261CA692A40A2610A6A2A40D9
:10C99000E2618A7C01252A40CB7CDB079B0F9A1839
:10C9A0000B7DDB075B0FD2184B7D9B07DB0ED2188C
:10C9B0008B7DDB079B0ED218CB7D1B079B0D9A1836
:10C9C0000B7E1B079B0CD2184B7E5B06DB0A1343C6
:10C9D0008A7E520612091A43CB7E5B075B0813431B
:10C9E0002362CA6A62620A6BA2624A6BE2628A6B63
:10C9F00022633922D200835C1E462E4066635E426B
:10CA00005E41B304AE04744F3C68B443E3183B602A
:10CA100083185A782A409C782407E40EA2188C8F39
:10CA20006401A2186D4C1440C98FC905490A09193F
:10CA3000DA78D207120A89181A79120712098918A6
:10CA40005A79D207D2088918FB4EB1639968F1630D
:10CA5000997904952940DA79D207920F51181A7BF7
:10CA60005207D20E89185A7BD206920D51189A7B22
:10CA70005207D20C8918DA7BD206920B89181A7CDD
:10CA8000D206520A89185A7C520792090A43997CA5
:10CA9000C906490851183164D97C039A11401A7D9E
:10CAA000D206920D51185A7DD206520C89189A7DE1
:10CAB000D206120B8918DA7DD206D2098918716460
:10CAC000197E0F2421405A7E120151189A7E1203BA
:10CAD0008918DA7E1207120A51181A7F12071209F2
:10CAE00089185A7F12078918B164997F01942140EF
:10CAF000DA7F1207120E51183D22D200835C5B07C9
:10CB00005B0D5918841862781207520C8918A278A4
:10CB1000D206120B8918E278D206D2098918F1647C
:10CB2000217907220A406179C9008918A279520641
:10CB3000920B5118E2799207120B8918227AD207C8
:10CB40008A18BF490A60627AA37A1B029A18E37AAC
:10CB50001B04D2184A60E289BA4B13400394228A1C
:10CB6000D2049209D2188A6003463033598CB64AEF
:10CB7000114002939A8CD205D20A51185622825C37
:10CB800012068918B14D2960014656314A788C78D1
:10CB90002402A2188C8864056409A218CC782407A2
:10CBA00012196A60CA880C7AA407A40BA2184C7ADE
:10CBB0006407E40A1219AA604989E96049218900D9
:10CBC0004118FF226632821800921035002207E0D9
:10CBD00000300040FFFFFF0004040040FF3F000062
:10CBE00084186427E65D03273E406523E35C9B07CA
:10CBF0001B0F9B196626A65DB607B60EF3186726AF
:10CC0000A65DB601F318DBB26826A65DB607B60DC1
:10CC1000F3186926A65DB607360DF3186A26A65DD9
:10CC2000B607B60CF3186B26A65DB607360CF318DC
:10CC30006C26A65DB607B60BF3186D26A65DB60783
:10CC4000360BF3186E26A65DB607B60AF3186F26E4
:10CC5000A65DB607360AF3187026A65DB607B609B4
:10CC6000F3187126A65DB6073609F3187226A65D7D
:10CC7000B607B608F3187326A45DA407E31808C521
:10CC80001032802AACD1019AD243704EB4180B787E
:10CC90003B404D78AD072D0FEB188D78AD07AD0EED
:10CCA000EB18CD78AD01EB18DBB20D79AD07AD0D0A
:10CCB000EB184D79AD072D0DEB188D79AD07AD0C47
:10CCC000EB18CD79AD072D0CEB180D7AAD07AD0B38
:10CCD000EB184D7AAD072D0BEB188D7AAD07AD0A29
:10CCE000EB18CD7AAD072D0AEB180D7BAD07AD091A
:10CCF000EB184D7BAD072D09EB188D7BAD07AD080B
:10CD0000EB18CD7BAD07EB18A3641031121DBDD11C
:10CD1000009B19785A785207520D51189A78D20709
:10CD2000120D8918B164059B1968F164D97D5A68A0
:10CD30001202511831659968454A0A40998A490595
:10CD400089187165D9683D4C2140B1651969214048
:10CD5000F165029E3178049D294082785207120FB6
:10CD60005118C2799207920E8918427A9207920D51
:10CD70005118827A9207120D8918C27AD207920C42
:10CD800089189A7DD207520C891872789207D20BB3
:10CD90008918B2781207D20A8918F2781207D209D4
:10CDA0008A182C490A60327C737C1B071B0D9A1869
:10CDB000B37C9B069B0BD218F37C1B079B0AD218F3
:10CDC000337DDB065B09D218737DDB071B09D218A4
:10CDD0004A60B27D2A40C38F5B009A188A60826CD9
:10CDE000CA60C26C22400A61F27D7F231340328CFC
:10CDF0005204520AD2184A6102698A614269CA61C0
:10CE000082690A62C2694A62026A8A62426ACA62C4
:10CE1000826A0A63C26A4A63039A927CD201121D33
:10CE20000A64027A3A40CA65808F074A1040086651
:10CE3000002006B0F0BDC04600300040FFFFFF00FC
:10CE40009C300040FF1F0000FF0300000040004036
:10CE5000FFFF1F000020004004480068806B80082E
:10CE600003490968490040180930704738940102A5
:10CE70001004004010B52D21C9004118027A032A80
:10CE800004D10079002807D0082006E08378DA1E54
:10CE9000022A05D2032412E0142088601C203DE001
:10CEA000012B02D1C8228A6012E00479042C01D33C
:10CEB000462404E0032C01D1322400E014248C60C9
:10CEC0005B1E022B04D3022A10D24279154B01E0DB
:10CED0004279154B9B181B78402B04D0102B06D1A0
:10CEE0001423442405E02A233E2402E0427934231B
:10CEF00048244B800C80022A06D0062A08D0052A36
:10CF000008D118224C2301E0142250230B8000E0AA
:10CF10001C224A80C078042803D114204880642051
:10CF2000088010BDB90E0100B20E01001348006860
:10CF30007047C04610B5104A107091700F49002814
:10CF400013D050680861042048619078FF221202D3
:10CF50000B4B1C689443800380B2001918600120B9
:10CF60004007084A1060084A10600020086007491E
:10CF700001220A6010BDC046289401021804004036
:10CF80001CE400E080E200E000E100E0700000400E
:10CF9000F0B591B0002801D1C04800688778F91E2B
:10CFA000022913D3012F21D0022F3CD11021CA43D3
:10CFB00044782146193991423DD800970125B94A54
:10CFC00028462946234601F063FF53E10821CA435E
:10CFD000447821462139914218D800970125B14A59
:10CFE00028462946234601F053FF43E10821CA435E
:10CFF000447821460939914234D800970125A94A3D
:10D0000028462946234601F043FF33E1032F3CD055
:10D01000042F43D1C3780125042B00D02DE106460F
:10D020002A02042343E00125A6A2284629463B46BE
:10D0300001F02EFF1EE1C3780125052B0AD8064614
:10D040002A02284698401B21084230D10021052B96
:10D0500008462ED002200090914A2846294601F029
:10D0600017FF07E10646C3780021022B1ED3032BCE
:10D070001CD0042B08460A461BD001250095884A7F
:10D080002846294601F004FFF4E0C3780125032B6C
:10D0900000D0FAE006462A02032308E0012583A215
:10D0A000284629463B4601F0F3FEE3E00A4601210B
:10D0B00048020F91592189007518FD214900711806
:10D0C0000291314662313F05D219641E1F27274065
:10D0D0005C013C191443044332795207D20C2243B9
:10D0E0002B789B065B0BD218B379DB071B0B134322
:10D0F0006D4D2B60F279032310931A40737A9B07CE
:10D100009B0E9A18B37A5B07DB0D9A18F37ADB074C
:10D110009B0DD218337BDB075B0DD218737B1B078B
:10D120005B0CD218AA603269EA6072692A61B2693E
:10D130006A61F269AA61326AEA61726A2A62B26A53
:10D140006A620F980870F06AA8623F20C4432C35C9
:10D150003046E4300F903046E5300E903046E630F1
:10D160000D903046E7300C903046E8300B9030465A
:10D17000E9300A903046EA3009903046EB300890AA
:10D180003046EC3007903046ED3006903046EE30B9
:10D1900005903046EF3004903046F030039037462B
:10D1A000F1373046F230F3360F990A194021525CBC
:10D1B000109B1A400E9B1B195B5C9B071B0F9A1858
:10D1C0000D9B1B195B5C9B079B0E9A180C9B1B19F4
:10D1D0005B5C9B019A18D2B20B9B1B195B5C9B0793
:10D1E0009B0D9A180A9B1B195B5C9B071B0D9A18D9
:10D1F000099B1B195B5C9B079B0C9A18089B1B19CE
:10D200005B5C9B071B0C9A18079B1B195B5C9B07BD
:10D210009B0B9A18069B1B195B5C9B071B0B9A18B0
:10D22000059B1B195B5C9B079B0A9A18049B1B19A7
:10D230005B5C9B071B0A9A18039B1B195B5C9B0793
:10D240009B099A183B195B5C9B071B099A180319E9
:10D250005B5C9B079B089A183319595C89078918EE
:10D2600002C51034A0D102980078042101430E4871
:10D27000C1630025284611B0F0BD04200090084A83
:10D280002846294601F004FEF4E703200090044AF2
:10D290002846294601F0FCFDECE7C046389401021F
:10D2A000112B0100572B010000100040556E6465E2
:10D2B00066696E6564206D65616E2050524620255A
:10D2C000640D0A00496E76616C6964206D65616E5B
:10D2D000205052462025640D0A0000007047704718
:10D2E00080B50E490E480246083A1268920000D4F2
:10D2F000603142680A4342600A490A6808239A4337
:10D300000A60091F012252040A600321890402688D
:10D310008A430260FBF782FA80BDC046200000808D
:10D320002800004004020040B0B5032000072D494A
:10D330000A68824301256807101808600024204607
:10D34000FFF7CDFF2046FFF7C9FFEFF3108028401D
:10D3500002D1EFF3108172B68021C943224A53688B
:10D360000B40536093680B409360D3680B40D360CD
:10D3700013690B40136153690B405361002800D1BE
:10D3800062B6B0BD70B50C4603210907154A136893
:10D390000B4313600122EFF31081114002D1EFF330
:10D3A000108272B68025EA430F4B5E6816405E60BD
:10D3B0009E682E439E60DD681540DD601D69154046
:10D3C0001D615D6915405D61002900D162B60028CC
:10D3D00002D00120FFF783FF002C02D00120FFF7CD
:10D3E0007DFF70BD00040040989501020D4A0029A0
:10D3F00007D001290BD101218140106888431060BA
:10D4000007E00121814010680843106001E001211C
:10D410008140101F02680A430121C90711430160BE
:10D420007047C04644000040032804D84000064925
:10D43000085A00B27047002000B27047032802D893
:10D440004000014A1152704712D001029E490870F3
:10D450007047C04670B58AB00C460546FF20FC30C8
:10D46000A8490E68315C59208000335CB27830786E
:10D4700008AE069609AE05960C4E04962126760651
:10D4800003960B4E0296012601960E2600965B1C13
:10D49000DBB2F8F765FA0998F3F704FA28700898F0
:10D4A000F3F700FA20700AB070BDC04600002041BA
:10D4B00000000443F0B58BB00446457C82480078F8
:10D4C0008249002822D000200880814A1080814BA8
:10D4D00001269E761E830A907F4800787F4E36781C
:10D4E0006DB205957E4D04957E4D03950AAD02956E
:10D4F0007D4D01950096F7F771FF0A9D112020568A
:10D500007A497B4A00F0D0FB064626E000260E80D2
:10D510006F4A16806F4B01209876188309966E48E3
:10D5200000786E4F3F786DB205956D4D04956D4D49
:10D53000039509AD02956C4D01950097F7F74EFFE5
:10D54000099D112021567F20C00500900190029670
:10D55000664A674B3046F9F795F84320010628469E
:10D56000F2F72CFFF3F79EF9089062480078002844
:10D5700024D05120800060494A7D42438D185F4885
:10D580000068A8642F46403750480078B874504867
:10D590000078F874554800783875554800787875E3
:10D5A00057480078F87550480069F3F77BF9B8756B
:10D5B00052484069E8644C4800686864FF20FE30C7
:10D5C00050490968085C3922D2008918022812D310
:10D5D00003D04E48007801280DD14B4806604348DF
:10D5E00000883A4A108042480088394A1080092051
:10D5F0000790089605E04448089A02603548C08BB9
:10D6000007900B780022002B01D0114600E0D14397
:10D610000125002B01D0042300E0EB43A67AAD1BCB
:10D62000EE175B1971416568AE0F277AAD00ED19F1
:10D630005641677A3F1FF817ED1970414000EE0F11
:10D6400080196D00EB1848418001990E411898012E
:10D6500027239B02C31A91411D4805881B48008857
:10D66000854201D00798421B10202056C001194D59
:10D670002D8C032D07D1E468E5176D0A6419E415B4
:10D680000519EC170FE0E468E5176D0A6519EC174A
:10D69000ED15C6174519744197B2002F00D03446D6
:10D6A000002F00D00546581BA141130409D012B227
:10D6B000D2015242D31780185941089BDA17C01A79
:10D6C00091410BB0F0BDC046BA930102E0AA01023D
:10D6D000DEAA010290940102B9900102B890010201
:10D6E000CCA00102C89E0102E4AA01022EAB0102F5
:10D6F0002CAB010298A40102D0A1010264200040D9
:10D70000DCAA010238940102D8AA010240AB01024E
:10D71000C10D4002803070470120C0071B490860DE
:10D720007047C04610B519480068C10710D181077D
:10D7300011D4410712D4010713D4C10614D48106B1
:10D7400015D4410616D48021084016D031A215E028
:10D7500001240FA213E0022411A210E0032414A25A
:10D760000DE0042416A20AE0052419A207E006240D
:10D770001CA204E0072421A201E0254A040902209A
:10D78000032101F085FB204610BDC0465C0000402F
:10D79000526573657420627920504F520D0A000063
:10D7A000526573657420627920424F520D0A000061
:10D7B00052657365742062792050494E0D0A00004D
:10D7C0005265736574206279205744540D0A000035
:10D7D0005265736574206279204C4F434B55500D50
:10D7E0000A00000052657365742062792053572047
:10D7F0005265626F6F740D0A000000005265736518
:10D8000074206279205359535245510D0A0000008B
:10D810003E1E0100526573657420627920445644AF
:10D82000440D0A0001218140044A1F2802D01068DB
:10D830008843106010680843106070471C00004067
:10D84000F0B583B0029104469949F2F743FC0546CE
:10D85000984901942046F2F73DFC974946189749AC
:10D86000714300956F189649441864212046F2F7D9
:10D8700031FC3818A108471A92492046F2F740FCBB
:10D88000381891494518914F05D464213046F2F774
:10D8900021FC0C4614E0A6B264213046F2F71AFCD3
:10D8A000B7204000A20701D1002907D1884B73435C
:10D8B0000422D341874A934200D3401E0C464519A7
:10D8C0000098474302980680192001013046F2F77C
:10D8D00001FC2A461F3A284600DB1046019BFF1830
:10D8E000B30705D1002C03D01F2D05DA0120C5E0B8
:10D8F0001F2D0BDA0120C1E005461D3D034600DB6C
:10D900002B461C2808DC02201546B7E000290CD065
:10D910001C21451A0CD50CE019461F39184600DBAE
:10D9200008461F2B1DDA0320A8E01D21451A00D44C
:10D930002846002D08D401461F39024600DB0A465E
:10D940001F2804DA032099E00220154696E01546C8
:10D950001E3D104600DB28461E2A0CDA04200D4628
:10D960008CE005461E3D024600DB2A461E280BDAE7
:10D9700004200D4682E001461F39024600DB0A46BC
:10D980001F280ADA052079E011461F39104600DB0E
:10D9900008461F2A0BDA052070E015461E3D10468A
:10D9A00000DB28461E2A0CDA06200D4666E00546F6
:10D9B0001E3D024600DB2A461E280BDA06200D46D5
:10D9C0005CE001461F39024600DB0A461F280ADADE
:10D9D000072053E011461F39104600DB08461F2A76
:10D9E0000BDA07204AE015461F3D134600DB2B46A5
:10D9F0001F2A0CDA08200D4640E005461F3D02466E
:10DA000000DB2A461F280BDA08200D4636E01946AF
:10DA10001E39184600DB08461E2B0ADA09202DE0C5
:10DA200011461E39104600DB08461E2A0BDA092073
:10DA300024E01F28054601DB05461F3D1F280CDAA0
:10DA40000A200D461AE01F28054601DB05461F3D4A
:10DA50001F2806DA0A200D4610E01E2D05DB0C20DB
:10DA600004E01E2D06DB0C2005E00B201E2D05DB3F
:10DA70001E3D03E00B201E2D00DB1E3D029EB070FC
:10DA8000681CF070E12001013846F2F723FB307189
:10DA9000C0B211494143CC193C212046F2F71AFB90
:10DAA00070713B21C94341430819B07103B0F0BD07
:10DAB000805101008033E101B207000093FEFFFFB7
:10DAC000B107000070FEFFFFA7FA0A0080AEFEFF5C
:10DAD000295C8FC20BD7A300F0F1FFFF70B504469D
:10DAE000FFF722FCA08A00280AD01F480ECC0EC0E7
:10DAF0000ECC0EC00ECC0EC01C480021018170BDA2
:10DB0000E08A1A4E3081A16932891948F2F70CFB7C
:10DB1000154D28460ECC0EC00ECC0EC00ECC0EC03D
:10DB2000FFF704FAF0606C68FFF796F9201A70624C
:10DB30002846FFF7BFFC05460C460E48007BFFF762
:10DB400073FC0121B1700C4900220A70316C491C30
:10DB5000316481B2C90B401800B2C1174010281AB5
:10DB600030658C41746570BD7097010208960102A2
:10DB70001CD00102BA9001021AD00102F0B581B0A6
:10DB8000EFF3108072B600200146FBF727FF044632
:10DB9000002803D062B6204601B0F0BD01273A0349
:10DBA0000025074E28463146FBF772FEBB02054AA8
:10DBB00028463146FCF74AFB62B6204601B0F0BD6C
:10DBC00000E00204D6A6010280B5F6F7C8FCF9F71A
:10DBD0003FFC0A49012048728A7A531C8B72034623
:10DBE00093434B710A7A0B78134304D0CA79501CC3
:10DBF000C871012090430249087080BDC897010296
:10DC00002094010270B514460D4606461120FAF71D
:10DC100083FF2248042101600C4804601E4805600F
:10DC20008660002E0DD0FF20000609490A68824355
:10DC30000120C00710180860064808210160064846
:10DC400001601A200221FFF7D1FB70BD1CD1010237
:10DC500000E400E080E200E000E100E00C49086040
:10DC60007047C04610B5044609480068604309493A
:10DC7000F2F746FA00190849486008480022026095
:10DC800002460C3A4B6813600968016010BDC0463B
:10DC900018D1010240420F000C9001022C100140EB
:10DCA00000480047C100000080B582B013460A4614
:10DCB00000900348011D0348F8F790FC02B080BDB6
:10DCC0005CD10102009E010210B50C498A1C9042F1
:10DCD0000DD2401E0D4A50600D4803680B400321D1
:10DCE0008C071B19036000209060116010BD044870
:10DCF0000449E622044B00F06FF8C046FFFFFF0026
:10DD0000151E01002F1E0100FB1D010010E000E0A8
:10DD100020ED00E0B0B50120EFF31081014002D109
:10DD2000EFF3108272B6124A1368124C22686468CC
:10DD30008506114800682840850E5D192923DB00FF
:10DD40006B43002C1D4606D1002809D11E206843D4
:10DD500000290AD0B0BD121BD218551C0028F5D0DE
:10DD60001D461E2068430029F4D162B6B0BDC046EE
:10DD70008CDC010214E000E004ED00E080B500203E
:10DD8000FBF7D6F8404280BDB0B586B01048694672
:10DD90000A4638C838C238C838C200242046FBF7C3
:10DDA000CDF803992046FBF763F90198012803D0C9
:10DDB0000824002804D102E00424002800D10446ED
:10DDC0000220FAF7B1FEE0400249086006B0B0BD9B
:10DDD000C00E0100A0DC010290B01C4605AB07C3D9
:10DDE000EFF31080C00702D1EFF3108072B6EFF3AB
:10DDF00010800B9068460E907046089010AB0F9301
:10DE0000CF4F3E1D01200490C502304629462246D0
:10DE100000F0B8FC00213154EFF303800990EFF3D8
:10DE200008800C90EFF309800D90EFF314800A90B6
:10DE300000F02CFC3868012833D80028C14F00D0EE
:10DE4000C14F2A20C1497A69920703D50A783A60FE
:10DE5000401E491C0028F6D1B948041D2046F2F79F
:10DE600091F9002807D079698907FAD521783960B6
:10DE7000401E641CF5E70220B5497A69920703D574
:10DE80000A783A60401E491C0028F6D12A20AF4982
:10DE90007A69920703D50A783A60401E491C002827
:10DEA000F6D1FFF737FF0346AA4A30462946FDF769
:10DEB00029FF04463018291B089F3B1F049A9343EF
:10DEC000A5A2FDF71FFF9E490968012966D8001920
:10DED00000299C4C00D09C4C00280AD09849091D70
:10DEE0006269920703D50A782260401E491C002807
:10DEF000F6D10A209F496269920703D50A78226009
:10DF0000401E491C0028F6D10598F2F73BF900287D
:10DF100009D061698907FAD5059A11782160401EF8
:10DF2000521C0592F3E7022089496269920703D5E2
:10DF30000A782260401E491C0028F6D10A208EA1D2
:10DF40006269920703D50A782260401E491C0028A6
:10DF5000F6D10698F2F716F9002809D06169890709
:10DF6000FAD5069A11782160401E521C0692F3E7FA
:10DF7000022077496269920703D50A782260401E21
:10DF8000491C0028F6D10A207EA16269920703D5B8
:10DF90000A782260401E491C0028F6D17CA2304637
:10DFA0002946079BFDF7AEFE6549096801290E9BCE
:10DFB0001BD80029634900D0634900280AD0604A71
:10DFC000121D4C69A40703D514780C60401E521C26
:10DFD0000028F6D102205E4A4C69A40703D51478C4
:10DFE0000C60401E521C0028F6D16AA23046294619
:10DFF000FDF788FE04463018291B694A3B46FDF7A9
:10E0000081FE4F490968012911D8001900294D499D
:10E0100000D04D4900280AD0494A121D4B699B0780
:10E0200003D513780B60401E521C0028F6D15D4AC0
:10E0300030462946099F3B46FDF764FE0446F8003A
:10E04000C00FB900C90F7A00D20F0092019102905F
:10E050003019291BFB0F544AFDF754FE04193019DF
:10E06000291B3F233B40514AFDF74CFE34490968C8
:10E07000012911D820180029324900D0324900283E
:10E080000AD02F4A121D4B699B0703D513780B60EA
:10E09000401E521C0028F6D1454A304629460B9BAB
:10E0A000FDF730FE04463018291B424A0A9BFDF753
:10E0B00029FE23490968012911D80019002921499D
:10E0C00000D0214900280AD01D4A121D4B699B0728
:10E0D00003D513780B60401E521C0028F6D1364A37
:10E0E000304629460C9BFDF70DFE04463018291BCF
:10E0F000324A0D9BFDF706FE114909680129114AB4
:10E100000DD80019002908D00F4A06E05169890787
:10E1100003D531781160401E761C0028F6D12849BD
:10E120000E98091AA94200D32946890800F03AFE40
:10E1300024480068002800D0804700F045F8C04619
:10E14000A8DC01020090014000A001406F1E010008
:10E150007B2B0100581E01000D0A2323232041536D
:10E1600053455254204020307825303858202323FE
:10E17000230D0A00321F010046554E4354494F4EAD
:10E180003A2000004C494E45202020203A20000033
:10E19000256400000D0A53503D253038580D0A0003
:10E1A000F71E01000D1F0100191F0100011F0100D2
:10E1B000B61E0100C51E0100D41E0100DF1E0100B5
:10E1C00000F80202A4DC0102F7480068012811D817
:10E1D000002801D00B4800E0FC480C210A4A01E06D
:10E1E000002907D043699B07FAD513780360491EBD
:10E1F000521CF5E71E20FFF715FB00BF00BF00BF54
:10E2000000BFFAE700A00140621E01008AB0064686
:10E21000E448B06600F03AFAFFF77CFD0346E248B6
:10E22000041D01200590C502E04A20462946FDF75D
:10E2300069FD074608942018DB4C0995E91BF36C2F
:10E240003F2206921340DAA2FDF75CFD2168012906
:10E2500010D8C0190029DD4900D0DD49002809D0B7
:10E26000221D4B699B0703D513780B60401E521C7F
:10E270000028F6D1F36BD7A2089C2046099D2946B9
:10E28000FDF740FD0746291A2018336C069A134003
:10E2900007D1D8A2FDF736FDC34C2168012907D963
:10E2A00017E0CEA2FDF72EFDBF4C2168012910D842
:10E2B000C0190029C54900D0C549002809D0221D30
:10E2C0004B699B0703D513780B60401E521C002836
:10E2D000F6D10027CBA5B8003058009008980999CE
:10E2E0002A463B46FDF70EFD216801290FD800297B
:10E2F000B64900D0B649002809D0221D4B699B07BA
:10E3000003D513780B60401E521C0028F6D17F1CE9
:10E310000D2FE0D1736BBFA2089C2046099D2946B2
:10E32000FDF7F0FC074620189F4CE91BB36BBC4A75
:10E33000FDF7E8FC2168012910D8C0190029A3497C
:10E3400000D0A349002809D0221D4B699B0703D5A3
:10E3500013780B60401E521C0028F6D1336CB14A72
:10E36000089C2046099D2946FDF7CCFC0746326CE7
:10E37000D000C00F9100C90F5300DB0F0093019133
:10E380000290E019E91BD30FA74AFDF7BBFC324608
:10E39000C619A019A91B1546136C069A1340A34A67
:10E3A000FDF7B0FC80490968012911D880190029BE
:10E3B000864900D0864900280AD07B4A121D4B6945
:10E3C0009B0703D513780B60401E521C0028F6D122
:10E3D0002E466B6C964A089C2046099D2946FDF7FF
:10E3E00091FC07462018E91B0796B36C914AFDF78C
:10E3F00089FC6D4A1168012910D8C0190029734998
:10E4000000D07349002809D0121D4B699B0703D522
:10E4100013780B60401E521C0028F6D10798426EFC
:10E42000042360215C2004931A400B4600D003466D
:10E430000693002A00D00846079E33587E4A089C5F
:10E440002046099D2946FDF75DFC0746069833588E
:10E45000E019E91B794AFDF755FCC619A019A91B5B
:10E46000079A536E76A2FDF74DFC4F4909680229C1
:10E4700011D280190029554900D0554900280AD0E9
:10E48000494A121D4B699B0703D513780B60401E48
:10E49000521C0028F6D10798C36C06466DA2089C52
:10E4A0002046099D2946FDF72DFC07462018E91B4B
:10E4B000336D6B4AFDF726FCC619A019A91B079FEF
:10E4C0007B6D68A2FDF71EFC8619A019A91BBB6D08
:10E4D00067A2FDF717FC344909680129059C11D88A
:10E4E00080190029394900D0394900280AD02E4A1C
:10E4F000121D4B699B0703D513780B60401E521CFD
:10E500000028F6D10798476B5D4A974237D203201F
:10E5100087430026059CB00039580246049B1A43E5
:10E52000BA5808230343FB580C2505437D59009135
:10E530000192029303953B1808980999514AFDF7F7
:10E54000E1FB1949096801290FD800291F4900D0AA
:10E550001F49002809D0089A4B699B0703D51378F7
:10E560000B60401E521C0028F6D11B2E444A06D8D0
:10E570000798406B361DB10040189042CBD30798E6
:10E58000406B111A099A914201D8890800E0610292
:10E5900000F008FC3C480068002800D08047FFF7E6
:10E5A00013FEC04622224B4DA8DC0102581E01007A
:10E5B0000D0A0D0A23232320455843455054494F43
:10E5C0004E202564202323230D0A000000900140E3
:10E5D00000A0014050433D25303858002C2045789C
:10E5E00063657074696F6E4E756D6265723D25640A
:10E5F0000D0A00002C205468726561644D6F6465DB
:10E600000D0A000052252D32643D253038580D0A80
:10E610000000000053503D253038580D0A0000001E
:10E62000F71E01000D1F0100191F0100011F01004D
:10E63000B61E0100C51E0100D41E0100DF1E010030
:10E640004558435F52455455524E3D253038580D7C
:10E650000A000000494353523D253038580D0A0046
:10E66000EA1E01005343523D253038580D0A000080
:10E670004343523D253038580D0A0D0A0000000072
:10E6800000F802029A1E0100A4DC0102F0B583B07A
:10E69000344D2C68012C06D8601E8441204601F0C0
:10E6A00047FB0028FAD10120EFF3108101400191CE
:10E6B00002D1EFF3108072B62B48285A2B49695AC1
:10E6C000814245D02A68002A01D02A4E00E0284E17
:10E6D0001F23DB020293284C022A27D205E01046B2
:10E6E000214AA85282B2914232D087B2B9420A4638
:10E6F00000D8621C131A21482B5218040DD0E819B7
:10E70000001D9FB201E0002F07D073699B07FAD567
:10E71000037833607F1E401CF5E7A242DFD90298E0
:10E720001018DDE7304683B299420CD0024680B221
:10E7300081420E4600D8661CA642F3D902983018D2
:10E7400083B29942F2D108496852B01A0B49685213
:10E750000B48002129540198002800D162B603B06B
:10E76000F0BDC046A8DC01020A080000080800004D
:10E770000090014000A00140FF0700000C080000CD
:10E780000F080000F0B58DB00793174600240C94D5
:10E7900009AA13C215E006986849F1F70FFEF2F7CF
:10E7A00081F8C117401848406549F1F793FC00957E
:10E7B00009A806223346F9F72FFCBDE0002C00D54E
:10E7C000BEE138787F1C25280DD0002800D1B7E1A4
:10E7D0000B9A511C0A9B9942F0D8099B9854641CCF
:10E7E0000C940B91EAE708940025397823390D2918
:10E7F00014D801207944097949008F44090F0F0F7B
:10E800000F0F0F0F0B0F060F0F0D05437F1CECE7CB
:10E810000820FAE70420F8E70220F6E738780146F6
:10E8200030390024092902D9264639460BE0002652
:10E830000A2171430E18303E791C78780246303A2E
:10E840000A2A0F46F4D32E2817D14A1C48780146CD
:10E850003039092905D911464F1C2538532811D9BB
:10E860006AE000240A2161430C18303C511C5078A6
:10E870000246303A0A2A0A46F4D34F1C2538532858
:10E8800000D959E04000C046784480884000874461
:10E89000A000530053005300530053005300530093
:10E8A00053005300530053005300530053005300D0
:10E8B00053005300530053005300530053005300C0
:10E8C00053005300530053005300530053005300B0
:10E8D0005300600053005300530053005300530093
:10E8E0005300530053005300530053005300530090
:10E8F000530053005300980053005300530053003B
:10E90000530053005300530053005300AD00B600B2
:10E910005300600053005900530053005300590046
:10E92000530053005300DE0053005300BD0053005A
:10E93000D3005300530098000C9C3FE70024744917
:10E9400040420F00791C38780F4625385328F3D8F9
:10E9500098E70799C91D072081430868079149680E
:10E96000F2F706F800210690F1F752FF00280BD1CC
:10E970000B99481C0A9A904206D8099A2D235354A1
:10E980000899491C0C910B9007980830079006983D
:10E99000F1F788FF0095C2178118514009A8224657
:10E9A0003346F9F739FB0B98411C0A9A914200D97A
:10E9B000F1E6099A2E2313540B910C98401C0C90ED
:10E9C000E9E6079802C807900096019509A8102269
:10E9D00039E00B98411C0A9A9142ADD8099A252337
:10E9E00013540B910C98401C0C90A5E70B9A511CEA
:10E9F000079C201D0A9B994239D907909CE70798EC
:10EA000002C80790009509A82246D3E6079901C9D4
:10EA1000079109990A9A089E02E0401C002E8BD4A7
:10EA20000378002B88D00B9D6C1C9442F5D84B5575
:10EA3000761C0C960B94F0E7079802C80790009696
:10EA4000019509A80A222346F9F784FB74E7079B7E
:10EA500010CB102C079308D300202146401C0A0934
:10EA6000FF291146FAD806280AD8082009E02368A9
:10EA7000099CA354089A521C0C920B9107905BE7D7
:10EA8000401C069009230C980B9D099905910A9E3C
:10EA900004940DE0202104463046059E715506463B
:10EAA0002046049C401C15460146089100290AD4C2
:10EAB0005B1E0699994206D26A1CB242EAD90899AD
:10EAC00008910029F4D50C900B950898002800D5E2
:10EAD00032E70126082501E06D1E3601022DFBD22A
:10EAE00020463146F1F7F6FA0F28F6D80C98059033
:10EAF000099803900A9806900B9D20463146F1F73D
:10EB0000E9FA691C069A914204D9089908910029EA
:10EB10000CD511E00C4A125C039B5A55089A521C02
:10EB20000D46059211460891002905D47043241A18
:10EB30003009102E0646E0D205980C900B95FBE6A6
:10EB400020460DB0F0BDC046B411010070B588B0CC
:10EB50000022032803D9D243104608B070BD7F4C71
:10EB6000C34D2A510F4B104EEE5081231E0101233D
:10EB7000AB5528602C1962600128EDD8079300225C
:10EB8000069205920492032303930292019200914C
:10EB9000411E8841694600F0FBFC0246104608B061
:10EBA00070BDC04604080000FFC0FFC0F0B583B0D0
:10EBB0000C460023D943012C56DB0746029101265F
:10EBC000EFF31085354002D1EFF3108072B658494B
:10EBD000584A505C002800D0A3E056545E48115AB1
:10EBE0005E48105A0196F202161A814240D8324607
:10EBF0005218A24240DB00930295A642354600DB44
:10EC000025464C490818001D39462A46F1F78CFA6A
:10EC1000A642484E04DA7919621B301DF1F784FAD6
:10EC20004E48305A001981B24D4A914201D94D499E
:10EC30004018029D009B4949705230464A4E805D03
:10EC4000002865D1EFF310850198054002D1EFF35C
:10EC5000108072B6374A4048115A4048105A8842CC
:10EC600032D1424813524FE00C46204603B0F0BD6B
:10EC700042425218A242BEDA3B4A2E4EB25C002AF1
:10EC80000CD03A4AB25A51188AB2354CA242284C9A
:10EC9000029F01D9334A8918304A02E0244C2F4A96
:10ECA000029F3355B152421A89B2884202D22C488F
:10ECB0008018421C93B22F4801212FA200F0E8F8DF
:10ECC0003C46002DD1D128E0019F9755884201D8BC
:10ECD0002348401C421A90B2800A01D00198820257
:10ECE0002248144F3A52386801280DD8431E9841E3
:10ECF000104B5918091D92B21D4B00F05FFE009B8E
:10ED0000002801D00B488355002D029D00D162B62A
:10ED1000074808490B54002DA7D162B6204603B01E
:10ED2000F0BD21200201044804A108A3FFF754F814
:10ED30000E080000A8DC0102AE1F010074726163BE
:10ED4000655F6F7574707574000000005452414324
:10ED500045204255535900000A08000008080000E9
:10ED6000FF07000000F8FFFF0F0800000C0800007C
:10ED7000BDEF000002FF00000D0A547261636520C0
:10ED80006275666665722069732066756C6C2C20EE
:10ED90006469736361726473202575206279746598
:10EDA000730D0A00F0B587B0054600260696059655
:10EDB000049603960296800701D007B0F0BD01913A
:10EDC00002A8142126A2FCF79DFF29490968012900
:10EDD00011D80029274900D0274900280BD002AAC2
:10EDE00001E0002807D04B699B07FAD513780B6028
:10EDF000401E521CF5E701990029DED0204C374611
:10EE0000B8002B58D80724D0581EA04204D31B4862
:10EE100018181C4A90421CD802A814211AA2FCF708
:10EE200071FF13490968012911D80029114900D03F
:10EE3000114900280BD002AA01E0002807D04B6935
:10EE40009B07FAD513780B60401E521CF5E7761C21
:10EE500001997F1C8F42B0D2322ED1D3ADE7C0468C
:10EE60000D0A4261636B74726163653A200D0A009A
:10EE7000A8DC01020090014000A00140FFFFFFFC60
:10EE8000FFFF0200FEFF0100253038580D0A000088
:10EE900081B0F0B5C4B00E46074649938120000109
:10EEA0002F49085C002845D002920120050204A8E1
:10EEB0002946F1F752F9FCB20021C8430C2C3AD88C
:10EEC000721E032A37D82748005DB042084632D365
:10EED000F80535D50021B8050DD404A801904018D7
:10EEE000691AA20022A39B582E4AFCF70BFF019837
:10EEF000F1F748F9014678050ED404AF7818691A7D
:10EF0000B20029A3D218121F1368264AFCF7FAFE92
:10EF10003846F1F737F90146029A04AE70180C46EC
:10EF2000691A49AB0393FFF72DFC01193046FFF72F
:10EF30003DFE00E0002044B0F0BC02BC01B0084738
:10EF4000FEF7E8FE034604A8019007A22946FCF755
:10EF5000D9FE0198F1F716F90146B805BDD5CAE703
:10EF6000A8DC01025E37010025313075207C2000CD
:10EF7000521F0100A81F0100A21F0100811F0100F4
:10EF80004C1F01006D1F01009B1F0100941F010019
:10EF90008F1F0100451F0100581F0100681F01005D
:10EFA0003D1F0100DF270100871F0100731F0100C3
:10EFB0007A1F01005E1F010000000000F0B581B063
:10EFC0000B460120EFF31084044002D1EFF31081CF
:10EFD00072B6990F07D0022001212DA2FFF758FF2A
:10EFE000002C3DD141E02249224D00276F54224A96
:10EFF000AB5A224AAE5AF3189EB2F60A01D0204EFE
:10F000009B19AB52EFF31086064002D1EFF3108349
:10F0100072B6AA5A1C4BEB5A934202D116482F5291
:10F020001AE06854934201D8164B5B1C9B1A99B2A4
:10F03000890A00D0830210482B52286801280BD877
:10F04000411E8841A918091D9AB2104B00F0B6FC68
:10F05000002801D006482F54002E03D0002C04D0E5
:10F0600001B0F0BD62B6002CFAD162B601B0F0BDBD
:10F070000F080000A8DC01020C0800000A080000CC
:10F0800000F8FFFFFF07000008080000BDEF0000C8
:10F0900055415254204572726F722025780D0A0036
:10F0A00010B50446FEF740F9A08A002800D010BD34
:10F0B000FDF73CFF0349C861C860486C401C4864C8
:10F0C00010BDC04608960102B0B50A2000242146B2
:10F0D000FBF796FD09202146FBF792FD012420460F
:10F0E00000F02CF80E2004252946FBF789FD0D20A1
:10F0F0002946FBF785FD1049204600F049FAB0BDCE
:10F10000B0B50E2000242146FBF77AFD0D202146E4
:10F11000FBF776FD0124204600F010F80A200425B4
:10F120002946FBF76DFD09202946FBF769FD0249D9
:10F13000204600F02DFAB0BD2090010270B50128E4
:10F1400001D9012070BD48224243734B9C58A569E8
:10F150001F218D43A5610625A5600F2525629C18FA
:10F16000A27C002A05D1627C002A02D1227C002ADE
:10F1700014D06368002B11D4251D0B4001221646C4
:10F180009E400C4B1E60BFF34F8FBFF36F8F2B68F9
:10F19000002B03D40B409A4007490A60002803D093
:10F1A000012804D1092000E00820F9F7ADFC002077
:10F1B000A06170BD80E100E080E200E0F0B585B0C4
:10F1C0000D460278E348C368934219D0446D9442D7
:10F1D00016D08368934203D0016D914200D07FE046
:10F1E0009B1A591E8B41049348215943032D46D144
:10F1F0004418E16900294ED01C34002020606DE0E5
:10F200009B1A5A1E93410493032D1AD10395482249
:10F210005A438418A26B0121EFF310850D4002D1EF
:10F22000EFF3108772B6A7691026B743A761A669E6
:10F23000002E01D118342160002D00D162B6039D4B
:10F240000CE048215943421891691832302902D004
:10F25000116810294CD180211160002248215943A6
:10F260004018002181630162816224300021016025
:10F27000002A33D004A82946904705B0F0BD4218B3
:10F2800091691832302902D01168202939D18021A2
:10F290001160002216E00395E26B0126EFF3108562
:10F2A000354002D1EFF3108172B6A1692027B9432E
:10F2B000A161A169002901D118342660002D00D177
:10F2C00062B6039D4821594340180021C163C162C1
:10F2D0004163303000210160002ACBD105B0F0BD80
:10F2E00000920E4A2E329C480D490E4BFEF774FDDB
:10F2F00010680093019098480949084A0A4BFEF7A4
:10F300006BFD106800930190044A2432924804492E
:10F31000054BFEF761FDC046D4940102B102000026
:10F320002A200100FF1F0100E31F0100F0B585B096
:10F33000049048210A464243864B9C58E6690F25B3
:10F3400035409A18167C002E31D04F20400261695A
:10F35000014200D185E0A06904218843A061022018
:10F360002062012081076918D161D36BEFF310840B
:10F37000044002D1EFF3108572B695692026B5439B
:10F3800095619569002D00D173E010463C30002C4A
:10F3900000D162B600240460D4625463303200208D
:10F3A0001060002B63D004A8984705B0F0BD0C2D69
:10F3B0005DD8C0467D442D796D00AF4467586B58C9
:10F3C0000658A1635858585806009569202D04D056
:10F3D000154618352D68302D49D1156B566B3432D2
:10F3E000AE4217D26669360714D5646815686E1C7C
:10F3F000166048431818C06A445504980C464443A4
:10F400001A19156B566B3432AE4203D21C59666919
:10F410003607EAD41268AA4229D141435858826972
:10F420000524A24382615A18D36B0121EFF31080A7
:10F43000084002D1EFF3108472B694692025AC43E2
:10F4400094619469002C02D114461834216014464A
:10F450003C34002800D162B600212160D1625163A2
:10F460009CE70C2D00D176E7012D00D173E705B0A4
:10F47000F0BD15461835286010463C30002C00D1F0
:10F4800087E787E70420206205B0F0BD01202062F5
:10F4900005B0F0BD08252562164618369569102D71
:10F4A00002D03568302D4BD10396566A1546283563
:10F4B000976AB74228D1A06902218843A061936B63
:10F4C0000121EFF31080084002D1EFF3108472B6EF
:10F4D000039E34681027BC4334603468002C00D18C
:10F4E000316014463834002800D162B60021216012
:10F4F00029601162243200201060002BB7D052E73F
:10F500000220206205B0F0BD2A68B242AFD2626923
:10F510009207ACD52A68561C2E6048431818006A1A
:10F52000805C206004980A4642439D18AC6A6E6A6B
:10F53000B4429CD228359C5862699207EAD496E777
:10F54000316800900191044804A1094A09A3FEF71B
:10F5500043FCC046D4940102C91F01007561727456
:10F560005F6972715F68616E646C657200000000B3
:10F570003D0300005561727420256420737461742A
:10F580006520676F65732077726F6E672025640052
:10F59000F0B585B00E460546022804D3002E02D1F0
:10F5A000012005B0F0BD002D03D0012D08D10924A4
:10F5B00000E008242046F9F7AFFA2046FEF732F9BA
:10F5C00048216943E74A505883691F240294A343A2
:10F5D0008361062383600F2301930362571800237E
:10F5E000BB62BB63FB633B627B62FB623B63317F5D
:10F5F0003974727F7A74B27FBA7404937B637368D0
:10F60000B268F468920022435B1E032B0ED8C046FA
:10F610007B441B795B009F4401050307082304E03A
:10F62000282302E0182300E038231A43C260C907E8
:10F63000090F72699201D2B28918B2699207920ECB
:10F640008918491C816079613169012901D1222120
:10F650000161012D5CD831680E2959D2384612302B
:10F6600003900324002D01D0204600E004204C43E9
:10F670002D490E19B178F9F7DFFA3968CA68802583
:10F6800010462843C8602848005D73781B0218188C
:10F69000C862AA43CA60F9F717FB039800780028EC
:10F6A00009D1384611300078002804D1384610308E
:10F6B0000078002827D07868002815D40321024656
:10F6C0008A431B4953588407E40EFF26A640B343E0
:10F6D000A5401D4355500299014001208840A24990
:10F6E0000860144908600EE08107C90EFF228A40B5
:10F6F000019C0440083C032084430C482358934356
:10F700008D401D4325500120B861049805B0F0BD1F
:10F7100002480349DA22034BFEF75EFBC91F0100D2
:10F720003C20010019200100480F01001CED00E001
:10F7300000E400E000E100E0F0B58FB00E9001259C
:10F74000002900D14BE0039304910592002A00D1D7
:10F7500045E00121EFF3108201910A4002D1EFF35D
:10F76000108172B64827029747437E49CE19B56982
:10F770000023302D23D831461831C0467D442D79E1
:10F780006D00AF4420242626262626262626262659
:10F79000262626265E2626262626262626262626D1
:10F7A0002626262618262626262626262626262607
:10F7B0002626262618000223002A0CD00CE0402D15
:10F7C00001D0802D05D10123002A04D004E020249B
:10F7D0000C60002A00D162B61D46002B02D02846DC
:10F7E0000FB0F0BD002575630399F1630499F162D0
:10F7F000059931635B4CE35959691322D2021142D6
:10F8000005D0062199600F21196271699960317CD8
:10F8100000290CD0F56109950895079506950D9579
:10F820000B9502210A91012810D017200FE0717C5E
:10F830009A6900292CD0952002439A6128460FB07E
:10F84000F0BD30240C60002AC5D0C5E71920049F04
:10F850000C907068002805D41F2108400199814050
:10F860004148016014209861B06806A9F9F79CFA34
:10F870000E98029941436018806861583B4A009293
:10F88000091D3A46059BF9F7FFFA28460FB0F0BD6F
:10F890003436110602D580218A439A6131680025E9
:10F8A000059A91422DD205955D694F214A02154274
:10F8B0001BD1E90502D4029CF24F0AE05968336873
:10F8C0005C1C3460029C6043EE4F3818C06AC1541F
:10F8D0000E98214641437E18736B346BA34238D295
:10F8E00034367B585D691542E3D002211962019ECE
:10F8F000B10729433546E34CEFF31082324006D07E
:10F9000008E02946019EEFF31082324002D1EFF366
:10F91000108372B6029B4343E01883692024A343FB
:10F9200083618369002B05D0002A08D0C26B002AAE
:10F930000AD154E7034618331E60002AF6D162B696
:10F94000C26B002A00D14AE70EA8904728460FB0A4
:10F95000F0BD2946059D019E3C46EFF310823240E2
:10F96000D5D0D7E7D494010280E200E0BDF10000D9
:10F9700080B5012082020249024BFFF7DDFE80BD07
:10F9800088CB010271F90000B0B582B07920840003
:10F99000E54D285D01A90870652080002818F3F75F
:10F9A000EDFE2F20C000285829190122024BFFF735
:10F9B000C3FE02B0B0BDC04689F90000F0B591B0F9
:10F9C00010900126002900D19BE003930591002AA5
:10F9D00000D196E007900121EFF3108002910840DA
:10F9E00002D1EFF3108172B604924823069307996F
:10F9F0004B43D649C9188D690026302D6ED80C4668
:10FA00001834AD00374602A675593E46AF46C0468B
:10FA1000E5FA0000EDFA0000F1FA0000F1FA00004A
:10FA2000F1FA0000F1FA0000F1FA0000F1FA00002A
:10FA3000F1FA0000F1FA0000F1FA0000F1FA00001A
:10FA4000F1FA0000F1FA0000F1FA0000F1FA00000A
:10FA5000D5FA0000F1FA0000F1FA0000F1FA000016
:10FA6000F1FA0000F1FA0000F1FA0000F1FA0000EA
:10FA7000F1FA0000F1FA0000F1FA0000F1FA0000DA
:10FA8000F1FA0000F1FA0000F1FA0000F1FA0000CA
:10FA900083FB0000F1FA0000F1FA0000F1FA000027
:10FAA000F1FA0000F1FA0000F1FA0000F1FA0000AA
:10FAB000F1FA0000F1FA0000F1FA0000F1FA00009A
:10FAC000F1FA0000F1FA0000F1FA0000F1FA00008A
:10FAD000D5FA0000022600280CD00CE0402D01D001
:10FAE000802D05D10126002804D004E010252560D2
:10FAF000002800D162B6002E069D944F049C079802
:10FB000002D0304611B0F0BD00268E62039A8A639F
:10FB1000059A0A624C620A7C002A0BD00C960B965E
:10FB20000A96099608960E9602220D9201282DD06B
:10FB300018202CE08A7C2831002A3BD00A68A24297
:10FB400016D22B464343FA585469A40710D50868C7
:10FB5000441C0C60F918096A085C1060109829466A
:10FB600041437A1811462831936A526A9342E8D386
:10FB700045437859816982220A438261304611B037
:10FB8000F0BD302525600028B4D0B4E71A200F90CE
:10FB9000C86808A9F9F708F9109845437A597819FF
:10FBA000C0683949009105992346F9F76DF9304647
:10FBB00011B0F0BDFB589A69140602D58024A24307
:10FBC0009A610A680026049882422ED25D694F220B
:10FBD0005202154207980AD002211962029EB1070B
:10FBE00029431FE028315D6915423E46F4D137466E
:10FBF0005C69A40702D40699544E0AE00C68661C9E
:10FC00000E6006994843514E3018006A005D186036
:10FC100010984143735871188C6A4E6AB442E1D30C
:10FC200029463E46069D494F01E0314607985A6AEB
:10FC3000002AFCD1EFF31082029B1A4002D1EFF3AD
:10FC4000108372B64543781983691024A3438361F6
:10FC50008369002B05D0002A09D0826B002A0BD1C2
:10FC60004FE703461833029C1C60002AF5D162B6A8
:10FC7000826B002A00D144E710A89047304611B0AB
:10FC8000F0BDC046D4940102BDF10000B0B52649D4
:10FC900000684A68824202D10D1D002016E08022D1
:10FCA0008A58824203D10D46803501200EE0FC22A5
:10FCB0008A58824203D10D46FC35022006E02F22ED
:10FCC000D2008B5883422ED18D1803207C224243D0
:10FCD0008C18A068012814D0002824D14034204674
:10FCE000F4F701F901462046F4F7D3F82046F4F77B
:10FCF000FAF8002817D006C828680C4BFFF75EFEFC
:10FD0000B0BD40342046F4F7EEF801462046F4F743
:10FD1000C0F82046F4F7E7F8002804D006C82868A1
:10FD2000024BFFF74BFEB0BD00BC01028DFC000092
:10FD300048214143054842189269D20601D4002067
:10FD4000704740584169012008407047D49401022F
:10FD500080B511480078C001104909788901014334
:10FD60000F480078400108430E4909780901014312
:10FD70000D480078C00008430C4909788900014308
:10FD80000B480078400008430A4909780143C8B28B
:10FD9000F4F75AFB80BDC0464C9D01026E970102EC
:10FDA00020940102BEE4010241AB01024D9D01021B
:10FDB000C8A00102C9A00102F0B587B00146012721
:10FDC000022505283A4600D02A4600200929014686
:10FDD00000D01146C900374A54180E210591615EC2
:10FDE000FDF72CFB1026A15F3846FDF727FB1227F5
:10FDF000E15F2846FDF722FB06951425615F03208D
:10FE00000490FDF71BFB0598235EA05FE15F625F36
:10FE100000AD07C528A2069F3846049D2946FFF776
:10FE200037F82046263004263146FBF7D9FF262036
:10FE3000235E2820205E2A21615E2C22A25E009093
:10FE40000191029224A238462946FFF721F827465D
:10FE50003E3738463146FBF7E1FF3E20235E0698E9
:10FE60003C5EB95F0622BA5E00940191029221A223
:10FE700007462E462946FFF70BF856240D4D285FFE
:10FE8000FBF7C0FF2B5F2C4621A238463146354692
:10FE9000FEF7FEFF264658363046FBF79FFF5820F8
:10FEA000235EF05F00901FA238462946FEF7F0FF60
:10FEB00007B0F0BD689E0102546F4620616E742049
:10FEC00064656C6179732025642025642025642095
:10FED00025640D0A0000000050446F412064656CE9
:10FEE0006179732025642025642025642025640D14
:10FEF0000A00000050446F41206761696E7320253D
:10FF0000642025642025642025640D0A000000007B
:10FF100050446F4120616E742073706163652025C9
:10FF2000640D0A0050446F4120616E676C65206F5C
:10FF30006666736574732025642025640D0A0000CD
:10FF4000F0B587B015467A4B1A680F24A2432F7874
:10FF50003A431A60774C23462C3B774A1A60049048
:10FF600003462246283A12681207FAD5734E092F23
:10FF7000029306D9754A326072600C2F09D1754818
:10FF80000FE0042F07D9704A3260704A7260092F5F
:10FF900006D3714805E06A4830607060694800E047
:10FFA0006B486E4A1060EB7AFF2B039102D1002060
:10FFB000B0620AE003210B406948C05C4022024362
:10FFC000B2620220674AFEF763FF029F00213846B3
:10FFD00005952A460B46FBF77BFF064602250321C3
:10FFE00061A2284601913346FEF752FF069630463D
:10FFF000FCF742FC01210498009108402CD13D40BF
:020000040001F9
:1000000033D1604900283AD1002D1ED06548A06246
:10001000E0622063606364486062644808601520A1
:1000200085046E1C8E608D60642420460F46F8F7B0
:100030004BFE3E603D602046F8F746FE281D3860C6
:1000400003215BA24E48FEF723FF0598007BFBF7D8
:100050009DF8069807B0F0BD2E4605460698FCF7B9
:1000600097FF284635463D40CBD02E46054606989C
:10007000FCF70AFC2846354642490028C4D04248CD
:10008000086142484861424888611520C86141487A
:10009000016840220A43026007210803274B5A697E
:1000A0008243009840031018586105220398424388
:1000B0002A4803689818334E766B47780F40995C4E
:1000C0000907490EC919CA03334B33409A18C901AD
:1000D0005118324A89182B4A51632A49896B3822B0
:1000E000914382785207920E891804220A432549C7
:1000F0008A63124B19690279019E3240C078400729
:10010000C00E80181F229143081818615520400323
:10011000411C216020606420F8F7D6FD204A184871
:100120003146039BFEF7B4FE1649002D8DD06DE7D6
:10013000040400402C6000400004008000060040E1
:100140000F040F04D1190100030403040004000488
:10015000021B0100A0180100331C01003C940102A5
:10016000641D0100682001005048592070617261CF
:100170006D73207365747320253038780D0A000084
:10018000020800009060004012A83E009DD79B5AD4
:10019000D579BD49340200403F0080FF4040000057
:1001A0004A2001002008820002D50F0002025500FB
:1001B0007577625F72785F696E69740D0A0000007E
:1001C00080B522480021017022480078C0012049F2
:1001D00009788901014320480078400108431F49FC
:1001E0000978C90001431E480078800008431D4972
:1001F0000978490001431C4800780843C0B2F4F76D
:1002000023F980BD80B511480121017010480078A4
:10021000800110490978C90101430F480078400165
:1002200008430E490978C90001430D480078800051
:1002300008430C490978490001430B4800780843FA
:1002400010210143C8B2F4F7FFF880BDBEE40102FB
:100250006E9701024C9D01022094010241AB010204
:100260004D9D0102C8A00102C9A00102F0B581B0F4
:100270001820FDF7D7FA1920FDF7D4FA00242046FC
:100280002146F8F739F920462146FAF703FF0126FF
:1002900003257F23304629462A46FBF70DF83046D2
:1002A000FBF7B2F902273846FBF7F2FD304631463C
:1002B000FCF740FE03A238462946FEF7E9FD20463A
:1002C00001B0F0BD7577625F6F70656E0D0A00005A
:1002D000F0B581B01646009104460020012739464A
:1002E000FDF750F8EFF310853D4002D1EFF3108099
:1002F00072B62720400170430A21EFF7EBFE024659
:10030000002C02D00020009901E002200021FBF720
:1003100081F90446FBF748FA002D00D162B6204669
:1003200001B0F0BDF0B581B01D460E460446022A6C
:1003300009D1012738463946FDF724F800960022F6
:10034000384629460FE0174601200021FDF71AF82C
:10035000012F04D1009600202946024603E00096B2
:10036000022000210A462346FBF736FA0446FBF733
:100370001BFA204601B0F0BD7047000070B50028A0
:1003800001D0012070BD0325A9020F4802680F4B60
:10039000535000249460012253030D4E3360BFF389
:1003A0004F8FBFF36F8F0B4E336003685A508472C8
:1003B00004811020F8F7A8FB022007A22946FEF7C7
:1003C00067FD204670BDC0466495010251E5CC1A18
:1003D00080E100E080E200E057445420636C6F73DA
:1003E000650D0A000FB47CB50C0009AD01D0611E8B
:1003F00000E0002101910090074B6A4629460898C9
:1004000000F012F9002C02D0009A002111707CBC7F
:1004100008BC04B018470000610D01007CB51D4602
:1004200016460C0001D0611E00E0002101910090F1
:10043000054B6A462946304600F0F6F8002C02D0FB
:10044000009A002111707CBD610D01002021020C79
:1004500001D010211046020A01D0104608390209C5
:1004600001D01046091F820801D01046891E42089B
:1004700001D0881E7047081A704700000048704776
:100480000890010202E008C8121F08C1002AFAD130
:1004900070477047002001E001C1121F002AFBD104
:1004A00070470000F0B51FB486B00998089A030D94
:1004B0000021024314D05148514A181850430514E2
:1004C0001198012810981AD0281A401C00264D4F68
:1004D0004D49009601910490002812DA444211E03F
:1004E0001198012449A3012801D11098C14306980D
:1004F000119A84600360C26041600BB0F0BD40425D
:10050000E4E70446210500203F4A001C51410391C5
:10051000029012E0E00707D032463B46019900986E
:10052000F0F77AF80191009032463B4610461946A2
:10053000F0F772F806460F466410002CEAD10498D2
:10054000039B0028029A0999089806DAF0F764F8E4
:10055000019B009AF0F760F805E0F0F7C5F8019B01
:10056000009AF0F7C1F804460E460022284BF0F737
:1005700009FC03D80020C043014607E00022254BB8
:1005800020463146EFF796FFF0F7DCFB102409E038
:10059000002C0ADB0A220023F0F706FA079B303210
:1005A0001A55641E02460A43F2D11122641C079BAD
:1005B000121B1C19119B012B03D0012308430ED1E0
:1005C0000AE0084304D0112010900020119077E732
:1005D0001098151A6D1E0BE01098824202DD002360
:1005E0006D1C03E0824201DA00236D1E002BEED069
:1005F000069811998260C16030C07EE701FCFFFF60
:10060000104D0000000014400000F03F30000000DA
:100610000000F0430000E03F30380A2801D20120FA
:100620007047002070470000FFB597B006460025D0
:1006300018E2252877D100242746FD49049400E0DC
:100640000443761C32780120203A90400842F7D1CA
:1006500030782A280ED00222307801463039092914
:1006600016D804990A235943303940181443761C8C
:100670000490F1E7189802C804911890002904DA50
:100680000120400304434842049002200443761CA6
:1006900030782E2814D1042004437078761C2A2840
:1006A00009D11898761C80C8189009E00A214F4398
:1006B000303FC719761C3078014630390929F5D901
:1006C00030786C2810D006DC4C281AD068280ED060
:1006D0006A2817D104E0742813D07A2812D110E0C8
:1006E0000120400504430CE00121090501E003213C
:1006F00009050C437178814203D1012000052418BB
:10070000761C761C3078119066280BD013DC5828A4
:100710007DD009DC00287BD04528F6D04628F4D0CF
:1007200047281AD1A5E118E0632835D0642870D095
:10073000652812D19DE170286CD008DC6728F1D0C3
:1007400069287BD06E280DD06F2806D1BAE07328B7
:100750002ED0752871D0782859D01A9A19999047B7
:100760006D1C7EE16002400F022809D003280DD0E5
:100770000428189801680DD00D60001D189070E1D4
:100780001898EA1701680D604A60F6E71898016842
:100790000D80F2E70D70F0E718986A460178117243
:1007A000001D18900020507202A80090012005E062
:1007B000189802C8189000200091C04361070DD519
:1007C000002101E00199491C0191B94212DA8142EC
:1007D000F8DB009A515C0029F4D10BE0002101E024
:1007E0000199491C01918142FADB019A0099895CC7
:1007F0000029F5D1019904981A9B471A21463846D9
:10080000199A00F097FA0199401945180BE04FE04A
:100810002CE113E04EE0009800990078491C00910B
:100820001A9A199990470198401E0190401CF2D1E4
:10083000214638461A9B199A10E137E00A20002118
:10084000009001916002410F022907D0189A01CA55
:100850001892C2179446032908D00AE01898C01DC0
:10086000C108C90005C91891944607E000B2C21733
:100870009446042902D140B2C1178C460022614639
:10088000944506DA0A460021404291418C462D21CA
:1008900002E0210504D52B216A461173012103E0F2
:1008A000E10701D02021F7E7029155E00A200AE094
:1008B000102008E010200090002104200443019142
:1008C000082703E008200021019100906002410FF9
:1008D000022907D0189A01CA1892002294460329C7
:1008E00008D008E01898C01DC108C90005C91891B2
:1008F000944603E080B2042900D1C0B200210291E5
:10090000210729D51199702906D0009A1021019B41
:100910004A401A4305D00EE040216A461173012176
:1009200008E06146014306D030216A4611731199EF
:10093000517302210291009A0821019B4A401A43F7
:100940000AD16146014301D1610705D530216A46CC
:10095000117301217F1E02911199582904D035A1EC
:100960000E910DA90D910DE037A1F9E76146019BAC
:10097000009AF0F719F80E9B8C469B5C0D9A521E5C
:100980000D92137061460143F0D10D9805A9081A24
:1009900020300190600703D501200004844300E06B
:1009A00001270198874201DD381A00E000200199F3
:1009B00000904118029809180498401A0490E00326
:1009C00006D421461A9B199A049800F0B3F94519E8
:1009D000002706E003A81A9AC05D199990476D1C7C
:1009E0007F1C02988742F5DBE0030CD521461A9B59
:1009F000199A049800F09EF9451904E01A9A3020DB
:100A0000199990476D1C0099481E00900029F5DC4B
:100A100008E00D980D990078491C0D911A9A1999C2
:100A200090476D1C0199481E01900029F1DC63E19B
:100A300009280100303132333435363738396162B4
:100A40006364656600000000303132333435363778
:100A500038394142434445460000000000F05AF94D
:100A60004519761C3078002800D0E2E528461BB0F6
:100A7000F0BD600700D406271898C01DC108C90042
:100A800048680A680831C30FDB071891190001D0C4
:100A90009CA108E0210501D59BA104E0E10701D05C
:100AA0009AA100E09AA1430011985B081091652873
:100AB0000CD006DC452809D046281DD0472841D156
:100AC00041E0662818D067283CD13CE00021112F76
:100AD00001DB112000E0781C0191009008A911A809
:100AE000FFF7E0FC139905910021119A15927F1CE4
:100AF00012980197009150E00120C0070390012057
:100B0000019008A9009711A8FFF7CCFC139A14993B
:100B100005920022119B009212981593059A01925A
:100B2000002901D0104602E0791C40180190381AC3
:100B300001D5019804E04042401E0090781C0190CD
:100B4000C01B029043E0012F00DA01270021112F82
:100B500001DD112000E038460191009008A911A89C
:100B6000FFF7A0FC13990591119A00211298159294
:100B70000091019721070CD40599B94201DB019935
:100B800000E00191012904DD159A491E515C3029CC
:100B900006D0B84201DA011D05DA0121029115E003
:100BA0000199491EEDE7002805DC009941180091E4
:100BB0000199091A03E0019A411C914200DD01915B
:100BC0000099401A401C02900120C00703902007A2
:100BD00006D402990198814202DB0020C0430290B2
:100BE00000206946C87707AF012103980337C9077A
:100BF000884224D0022011902B20129003980028C4
:100C00000CDA404203902D20129007E00A2103984D
:100C1000EFF760FA30317F1E039039701199481E4A
:100C200011900029F2DC03980028EFD1791E129868
:100C300008703078202108404530BF1E387006A863
:100C4000C01BC01D039010980078002800D0012020
:100C5000019941180298C0170918039809180498B7
:100C6000401A401E0490E00306D421461A9B199AAC
:100C7000049800F05FF8451910980078002803D018
:100C80001A9A199990476D1CE00324D521461A9BA6
:100C9000199A049800F04EF845191CE000980028B5
:100CA00007DB00990598884203DD1598405C199987
:100CB00001E0199930201A9A904700986D1C401C49
:100CC00000900298401E0290002804D11A9A2E200B
:100CD000199990476D1C0199481E01900029DDDC8F
:100CE00005E038781A9A7F1C199990476D1C039972
:100CF000481E03900029F4DC21461A9B199A049897
:100D0000ACE600002D0000002B00000020000000D9
:100D100000000000F8B5044600251E46174688046A
:100D200004D405E039462020B0476D1C641EF9D577
:100D30002846F8BDFFB50446002581B01E46C8030D
:100D400001D5302700E02027880404D505E0384687
:100D50000399B0476D1C641EF9D5284605B0F0BD57
:100D60004A68002A06D00A68531C0B601070486855
:100D7000401E4860704700B50A4683B000210091CC
:100D80000191014601236846EFF7CAFE01990098D8
:100D900003B000BD00404040404040404040414121
:100DA0004141414040404040404040404040404040
:100DB00040404040400502020202020202020202DA
:100DC00002020202022020202020202020202002D7
:100DD0000202020202029090909090901010101067
:100DE0001010101010101010101010101010101003
:100DF0000202020202028888888888880808080897
:100E00000808080808080808080808080808080862
:100E10000202020240000000950D0100642801005A
:100E2000881300000100000054280100881300000E
:100E3000010000004A2801008813000001000000A2
:100E40005E28010088130000010000000C2801004A
:100E500088130000010000001A2801008813000018
:100E600001000000E227010060EA0000030000002A
:100E70006E28010060EA00000300000079280100EC
:100E8000E803000005000000F727010088130000B8
:100E900005000000000084C1000008C10000C03F40
:100EA000000038410000AC410000D441280004009B
:100EB0000000084008000008100804081020000086
:100EC000000000000000000001000000FFFFFFFF25
:100ED000000000000000000000000000B00400005E
:100EE000010000006009000002000000C0120000C4
:100EF000030000008025000004000000004B0000FB
:100F000005000000009600000600000000E100005F
:100F10000700000000C20100080000000084030078
:100F200009000000000807000A00000000100E0081
:100F30000B00000000201C000C00000040420F00CD
:100F40000D00000080841E00590620140321450175
:100F5000288200324100321900411300390300B5E4
:100F600006002D03002D02002201002201003E0197
:100F7000002000008009EE4D5048504F80096E4F10
:100F800058E5854F80096E4FB867C14F5048D04F24
:100F9000B867C14FE828DF4F8009EE4F18EAFC4FD1
:100FA0008009EE4F58E50550A4550D50F0C514507A
:100FB000A4550D5000002110422063308440A550FC
:100FC000C660E770088129914AA16BB18CC1ADD18F
:100FD000CEE1EFF13112100273325222B552944237
:100FE000F772D662399318837BB35AA3BDD39CC3DF
:100FF000FFF3DEE36224433420040114E664C77483
:10100000A44485546AA54BB528850995EEE5CFF52E
:10101000ACC58DD55336722611163006D776F666D6
:101020009556B4465BB77AA719973887DFF7FEE77E
:101030009DD7BCC7C448E5588668A77840086118A2
:1010400002282338CCC9EDD98EE9AFF948896999CE
:101050000AA92BB9F55AD44AB77A966A711A500A76
:10106000333A122AFDDBDCCBBFFB9EEB799B588B1E
:101070003BBB1AABA66C877CE44CC55C222C033CC2
:10108000600C411CAEED8FFDECCDCDDD2AAD0BBD6E
:10109000688D499D977EB66ED55EF44E133E322E16
:1010A000511E700E9FFFBEEFDDDFFCCF1BBF3AAFBE
:1010B000599F788F8891A981CAB1EBA10CD12DC11C
:1010C0004EF16FE18010A100C230E32004502540B2
:1010D00046706760B9839893FBA3DAB33DC31CD312
:1010E0007FE35EF3B1029012F322D2323542145202
:1010F00077625672EAB5CBA5A89589856EF54FE55E
:101100002CD50DC5E234C324A01481046674476451
:1011100024540544DBA7FAB79987B8975FE77EF7B1
:101120001DC73CD7D326F2369106B01657667676A1
:10113000154634564CD96DC90EF92FE9C899E9897D
:101140008AB9ABA94458654806782768C018E108F1
:101150008238A3287DCB5CDB3FEB1EFBF98BD89B51
:10116000BBAB9ABB754A545A376A167AF10AD01A41
:10117000B32A923A2EFD0FED6CDD4DCDAABD8BAD9D
:10118000E89DC98D267C076C645C454CA23C832C91
:10119000E01CC10C1FEF3EFF5DCF7CDF9BAFBABFF1
:1011A000D98FF89F176E367E554E745E932EB23EE1
:1011B000D10EF01E303132333435363738394142B2
:1011C0004344454610004000800000010002000436
:1011D00000080010100018002000300040006000DF
:1011E00080000001FFFFFFFF01FF01FFFF0101FF82
:1011F000FF010000020000000100000002000000EA
:101200000200000002000000000000001B000000BF
:1012100000000000000000000000000000000000CE
:1012200000000000000000000200000000000000BC
:10123000140000000200000007000000020000008F
:10124000020000000000000002000000000000009A
:101250001400000002000000010000000200000075
:101260000200000002000000000000001400000066
:1012700000000000FFFFFFFFFFFFFF01FFFF01FF76
:10128000FF01FF01FF01FFFFFF0101FFFFFF01FF62
:101290000101FFFF000100FF010000FF00006400EA
:1012A0009E00C800E800020119012C013D014C011B
:1012B0005A01660172017D01870190019901A10126
:1012C000A901B001B701BE01C401CA01D001D60114
:1012D000DB01E101E601EB01EF01F401F801FD01A1
:1012E0000102050209020D021102140218021B027A
:1012F0001F022202250228022B022E023102340292
:1013000037023A023D023F024202450247024A02C8
:101310004C024F0251025302560258025A025C021A
:101320005F02610263026502670269026B026D027D
:101330006F02710273027502760278027A027C02F1
:101340007E027F0281028302840286028802890271
:101350008B028C028E028F029102920294029502FD
:10136000970298029A029B029D029E029F02A1028E
:10137000A202A302A502A602A702A902AA02AB0228
:10138000AD02AE02AF02B002B102B302B402B502C6
:10139000B602B702B902BA02BB02BC0200000000EA
:1013A000000000000200000004000000001003EB39
:1013B0000000000001000000010000000400000027
:1013C00000010032000000000000000000000000EA
:1013D0000100000001000005000000000000000006
:1013E00000000000010000000100003500000000C6
:1013F00001000000000000000400000000000020C8
:1014000000000000010000000000000004000000D7
:10141000000000D8000000000100000000000000F3
:1014200001000000000000060000000001000000B4
:1014300000000000010000000200000100000000A8
:101440000000000000000000010000000300009FF9
:10145000000000000100000000000000010000008A
:10146000000000B9000000000100000000000000C2
:1014700001000000000000AB842801000000000013
:1014800008150100C922000036290100E8140100F6
:10149000000000005D18000047290100E814010069
:1014A000000000009D1A0000282901001815010005
:1014B00000000000551D0000D6280100C8140100DE
:1014C00000000000391F0000652901001815010007
:1014D000B8140100F11F0000A228010078140100D7
:1014E00000000000812000001C2901007814010088
:1014F000081501002D210000AE280100781401001C
:1015000000000000A1210000E4280100E81401000F
:1015100000000000F52100005829010078140100A6
:1015200028150100B5230000BE2801001815010090
:101530000000000021240000AB290100C8140100B4
:101540000000000029260000EE290100C814010057
:101550000000000029270000BE290100C814010076
:1015600000000000FD280000D7290100C814010078
:10157000000000007529000095290100C814010031
:1015800000000000052A000074290100E814010091
:1015900000000000112D0000C9270100FA260100FB
:1015A0004325010037260100602701001E260100A7
:1015B00032250100AA240100BD24010031270100C9
:1015C0000C260100F1250100C82501004527010076
:1015D000A327010076250100E7240100622601000F
:1015E0004B2601007323010059230100F62301005B
:1015F000B5250100092401001C2501005E2501001C
:1016000080240100E3230100CD260100052701000D
:101610008A250100E326010019270100CB230100E0
:101620001C240100382401009F230100F92401003B
:101630003E230100B62601009F2501006924010018
:10164000DB250100B52301008A2301007826010073
:101650008C27010076270100D1240100A02601007B
:10166000B72701008D2601005424010094240100B5
:1016700022210100362101004A2101005E210100E2
:1016800072210100862101009A210100AE21010092
:10169000C2210100D62101005125010002000000F5
:1016A0001425010002000000DA22010003000000FE
:1016B0004526010003000000792201000700000018
:1016C00080220100080000001F2301000900000023
:1016D000CD2201000A000000022201000B000000E0
:1016E000BC2201000C0000003C230100100000009F
:1016F0009222010011000000D3220100120000001C
:101700000C250100180000005425010019000000FC
:10171000A9220100160000000821010014000000A9
:10172000F62001001A000000352201001700000019
:101730003E2201001B000000DB2601001C0000000F
:101740000B2301001D000000A02201001E0000006C
:10175000002301001F0000001323010020000000EF
:101760002222010021000000452201002200000089
:1017700055220100230000000E2201002400000079
:101780009922010025000000EA2101002600000046
:10179000E320010027000000B22201002800000021
:1017A0006E22010029000000C32201002A0000006F
:1017B000182201002B000000F92101002C0000007C
:1017C000E62201002D000000312301002E00000060
:1017D000272301002F0000008822010030000000B4
:1017E000F6220100310000002E2201001500000049
:1017F000C527010032000000EF2201003300000085
:1018000065220100340000001821010035000000AD
:10181000342101003600000048210100370000009B
:101820005C21010038000000702101003900000037
:10183000842101003A000000982101003B000000D3
:10184000AC2101003C000000C02101003D0000006F
:10185000392A01003E000000E82101003F0000009D
:10186000000100FF010000FF000100FF010000FF78
:10187000FF00000100FF00010001000000FF00FF69
:1018800000FF00000100FFFF00FF01000000000159
:10189000010000FFFFFF01FF010100000000010146
:1018A0000003020100000502010000010301000025
:1018B0000303010001000301000102030100020013
:1018C00003010002020301000302030100030403F9
:1018D00001000402030100000003020000030302F0
:1018E00000000603020001000302000103030200DE
:1018F00001060302000201030200020403020002C7
:1019000007030200030303020000010703000006AF
:10191000070300010004030001000703000104079E
:101920000300010707030002000703000204070386
:101930000002070703000302070300030607030072
:101940000402070300040607030005010403000561
:10195000020703000506070300060007030006044C
:10196000070300060707030007030703000707072D
:101970000300080207030008060703000902070323
:101980000009060703000A020703000A070703000D
:101990000B050703000C030703000C070703000DEA
:1019A000070703000E070703000E060704000E07D3
:1019B0000704030E070704030E070704030E0707B7
:1019C00004030E070704030E070704030E070704AA
:1019D00003000700020201000002020004010202EB
:1019E00000070102020202000202010101020201DB
:1019F00006010202030500020204020002020206BE
:101A000001020203000102020305010202050300B4
:101A1000020204050102020204020202020702029B
:101A2000020503010202050601020206000102028C
:101A3000060301020202050302020206030202017A
:101A40000604020201060702020203040202020364
:101A50000702020206070202030207020203050749
:101A6000020203070702020407040202050104023E
:101A7000020501070202050307020205060702022A
:101A80000602070202060507020207010702020713
:101A90000407020208010402020802070202080504
:101AA000070202090304020209040702020A0007EE
:101AB00002020A020702020A050702020A070702D7
:101AC000020B030702020B060702020C01070202C7
:101AD0000C040702020D010702020E000702020EAB
:101AE000040702020F010702020F050702020E049B
:101AF0000703030F030703030F070703030F07077A
:101B000003030000000202000000020200000002C5
:101B100002000000020200000002020000000202B7
:101B2000000100020200040002020007000202019C
:101B30000100020201040002020107000202020386
:101B40000002020104010202010601020203050073
:101B50000202020401020203010102020303010264
:101B6000020401010202040401020202060202024E
:101B70000302020202010603020202020302020140
:101B80000207020201040702020303030202020425
:101B90000402020205070202030107020203050410
:101BA00002020401070202040307020205060302FF
:101BB00002050007020205020702020504070202ED
:101BC00006000702020602070202060507020206D5
:101BD00007070202070407020207070402020802BD
:101BE00007020208050702020901070202090407A9
:101BF00002020A000702020A030702020A0607029B
